:020000040800F2
:10000000B0D10320A1D20508793105087B3105085C
:100010007D3105087F3105088131050800000000A9
:10002000000000000000000000000000CD73000888
:100030008331050800000000717300088531050850
:10004000C9F00508CDF00508D1F00508D5F0050880
:10005000D9F00508DDF00508E1F00508E5F0050830
:10006000E9F00508EDF00508F1F00508F5F00508E0
:10007000F9F00508FDF0050801F1050805F105088E
:1000800009F105080DF1050811F1050815F105083C
:1000900019F105081DF1050821F1050825F10508EC
:1000A00029F105082DF1050831F1050835F105089C
:1000B00039F105083DF1050841F1050845F105084C
:1000C00049F105084DF1050851F1050855F10508FC
:1000D00059F105085DF1050861F1050865F10508AC
:1000E0008F31050869F105086DF1050871F1050802
:1000F00075F1050879F105087DF1050881F105081C
:1001000085F1050889F105088DF1050891F10508CB
:1001100095F1050899F105086DD902089DF10508CA
:10012000A1F10508A5F10508A9F10508ADF105083B
:1001300097310508000000000000000000000000EA
:10014000000000000000000000000000B1F1050800
:10015000B5F105089F310508B9F10508BDF105089D
:10016000C1F10508C5F10508C9F10508CDF105087B
:10017000D1F10508893105080000000000000000E9
:10018000D5F10508D9F10508DDF10508E1F105080B
:10019000E5F10508E9F1050800000000EDF10508AA
:1001A000000000000000000000000000F1F1050860
:1001B000F5F10508F9F10508000000000000000055
:1001C000000000000000000000000000000000002F
:1001D000000000000000000000000000FDF1050824
:1001E000000000000000000000000000000000000F
:1001F00000000000000000000000000000000000FF
:1002000000000000000000000000000000000000EE
:1002100000000000000000000000000000000000DE
:10022000000000000000000000000000000003804B
:10023000000380000380000380000380000380002F
:100240000380000380000380000100000100000023
:100250000000000000038000038000000000000098
:10026000000000000000000000000000000000008E
:100270000000000000000000000E70000E70000E74
:10028000700004200004200004200004200000006E
:10029000000000000000000000000000000000005E
:1002A000000000000000000000000000000000004E
:1002B00000000000000000000000000000000660D8
:1002C000000660000660000660000660003FF8005F
:1002D0003FF8000660000CC0003FF8003FF8000C3B
:1002E000C0000CC0000CC0000CC0000CC00000001E
:1002F00000000000000000000000000000000000FE
:1003000000000001800001800007B0000FF000181D
:1003100070001870001C00000F800007E00000F063
:10032000001830001C30001C70001FE0001BC000D3
:1003300001800001800001800001800000000000B9
:100340000000000000000000000000000000078026
:10035000000FC0001CE0001860001860001CE000E6
:100360000FF80007E0001FF000073800061800062D
:10037000180007380003F00001E000000000000052
:10038000000000000000000000000000000000006D
:1003900000000000000000000000000003F0000763
:1003A000F0000C60000C00000C00000600000700CC
:1003B000000F9C001DFC0018F0001870000FFC00DE
:1003C00007DC00000000000000000000000000004A
:1003D000000000000000000000000000000000001D
:1003E0000003800003800003800001000001000082
:1003F00001000001000000000000000000000000FB
:1004000000000000000000000000000000000000EC
:1004100000000000000000000000000000000000DC
:10042000000000000000001800003800007000000C
:10043000F00000E00000E00001C00001C00001C0C9
:100440000001C00001C00001C00000E00000E000A9
:10045000007000007000003800001800000000006C
:100460000000000000000000000000000000180074
:10047000001C00000E00000E000007000007000036
:1004800003800003800003800003800003800003DA
:1004900080000700000700000F00000E00001C0095
:1004A0000018000000000000000000000000000034
:1004B0000000000000000180000180000180001D9C
:1004C000B8001FF80007E00003C00003C00006608A
:1004D00000066000000000000000000000000000B6
:1004E000000000000000000000000000000000000C
:1004F00000000000000000000000000000000000FC
:1005000000000000018000018000018000018000E7
:100510000180003FFC003FFC0001800001800001E1
:100520008000018000018000000000000000000049
:1005300000000000000000000000000000000000BB
:1005400000000000000000000000000000000000AB
:10055000000000000000000000000000000000009B
:100560000000000000000000000000E00000C000EB
:1005700001C00001800001800003000003000000B2
:10058000000000000000000000000000000000006B
:10059000000000000000000000000000000000005B
:1005A0000000001FF8001FF800000000000000001D
:1005B000000000000000000000000000000000003B
:1005C000000000000000000000000000000000002B
:1005D000000000000000000000000000000000001B
:1005E000000000000000000000000000000000000B
:1005F0000000000000000000000003C00003C00075
:1006000003C0000000000000000000000000000027
:100610000000000000000000001800001800003872
:100620000000300000700000600000600000C000AA
:1006300000C00001800001800003000003000006EC
:1006400000000600000E00000C00001C0000180056
:100650000018000000000000000000000000000082
:1006600000000000000003C00007E0000C30000C98
:10067000300018180018180018180018180018185A
:10068000001818001818000C30000C300007E000AB
:1006900003C0000000000000000000000000000097
:1006A00000000000000000000000000000000080CA
:1006B000000780001F80001D800001800001800075
:1006C00001800001800001800001800001800001A4
:1006D00080000180001FF8001FF8000000000000EB
:1006E000000000000000000000000000000000000A
:1006F00000000000000007C0001FF000383000308C
:10070000180030180000180000300000600001C020
:10071000000380000600000C00001800003FF800F5
:100720003FF8000000000000000000000000000092
:10073000000000000000000000000000000003C0F6
:10074000000FE0000C70000030000030000060007E
:1007500003C00003E0000070000018000018000053
:1007600018001838001FF0000FC000000000000043
:100770000000000000000000000000000000000079
:1007800000000000000000E00001E00001E00003C4
:1007900060000660000660000C60000C60001860DD
:1007A000003060003FF8003FF80000600003F800F0
:1007B00003F800000000000000000000000000003E
:1007C00000000000000000000000000000001FF01A
:1007D000001FF0001800001800001800001BC000E7
:1007E0001FF0001C30000018000018000018000066
:1007F00018003030003FF0000FC000000000000083
:1008000000000000000000000000000000000000E8
:1008100000000000000000F80003F8000700000ED0
:1008200000000C00001800001BC0001FF0001C306E
:10083000001818001818001818000C38000FF000E5
:1008400003E00000000000000000000000000000C5
:1008500000000000000000000000000000001FF881
:10086000001FF80018180018380000300000300091
:1008700000700000600000600000E00000C00000A8
:10088000C00001C0000180000180000000000000E5
:100890000000000000000000000000000000000058
:1008A00000000000000007E0000FF0001C380018F6
:1008B00018001818000C300007E00007E0000C30AA
:1008C000001818001818001818001C38000FF00045
:1008D00007E0000000000000000000000000000031
:1008E000000000000000000000000000000007C041
:1008F000000FF0001C30001818001818001818001D
:100900000C38000FF80003D8000018000030000079
:10091000700000E0001FC0001F0000000000000089
:1009200000000000000000000000000000000000C7
:1009300000000000000000000000000000000000B7
:10094000000003C00003C00003C00000000000005E
:100950000000000000000000000003C00003C00011
:1009600003C00000000000000000000000000000C4
:100970000000000000000000000000000000000077
:100980000000000000000000000000F00000F00087
:1009900000F0000000000000000000000000000067
:1009A000E00001C00001800001800003000002009F
:1009B0000000000000000000000000000000000037
:1009C000000000000000000000000000001C00000B
:1009D0003C0000F00003C0000F00003C0000F000ED
:1009E000003C00000F000003C00000F000003C00CD
:1009F000001C0000000000000000000000000000DB
:100A000000000000000000000000000000000000E6
:100A1000000000000000000000000000007FFC005B
:100A20007FFC000000000000007FFC007FFC000055
:100A300000000000000000000000000000000000B6
:100A400000000000000000000000000000000000A6
:100A500000000000000000000000000070000078AE
:100A600000001E000007800001E000007800001E6A
:100A70000000780001E0000780001E000078000000
:100A800070000000000000000000000000000000F6
:100A90000000000000000000000000000000000056
:100AA0000007C0000FE00018700018300018300078
:100AB00000700000E00003C000038000030000009D
:100AC0000000000000070000070000000000000018
:100AD0000000000000000000000000000000000016
:100AE00000000000000003E00007F0000E38000CDA
:100AF000180018780018F80019D8001998001998EB
:100B00000019980018F8001878001800000C000070
:100B10000E180007F80003E00000000000000000CD
:100B200000000000000000000000000000000000C5
:100B3000001F80001FC00001C000036000036000B0
:100B40000630000630000C30000FF8001FF80018C7
:100B50000C00300C00FC7F00FC7F00000000000057
:100B60000000000000000000000000000000000085
:100B70000000000000000000007FE0007FF000188F
:100B800038001818001818001838001FF0001FF857
:100B900000181C00180C00180C00180C007FF8003E
:100BA0007FF00000000000000000000000000000D6
:100BB0000000000000000000000000000000000035
:100BC0000003EC000FFC001C1C00180C00300C0093
:100BD000300000300000300000300000300000180D
:100BE0000C001C1C000FF80003F0000000000000C7
:100BF00000000000000000000000000000000000F5
:100C00000000000000000000007FC0007FF000181E
:100C10003800181800180C00180C00180C00180CDC
:100C200000180C00180C001818001838007FF0008D
:100C30007FE0000000000000000000000000000055
:100C400000000000000000000000000000000000A4
:100C5000007FF8007FF80018180018180019980095
:100C60001980001F80001F8000198000199800184B
:100C700018001818007FF8007FF80000000000003E
:100C80000000000000000000000000000000000064
:100C90000000000000000000003FFC003FFC000CD2
:100CA0000C000C0C000CCC000CC0000FC0000FC0DE
:100CB000000CC0000CC0000C00000C00003FC00085
:100CC0003FC0000000000000000000000000000025
:100CD0000000000000000000000000000000000014
:100CE0000003EC000FFC001C1C00180C00300C0072
:100CF00030000030000030FE0030FE00300C0038C4
:100D00000C001C1C000FFC0003F0000000000000A1
:100D100000000000000000000000000000000000D3
:100D20000000000000000000007E7E007E7E0018B3
:100D300018001818001818001818001FF8001FF8DD
:100D4000001818001818001818001818007E7E00E7
:100D50007E7E000000000000000000000000000097
:100D60000000000000000000000000000000000083
:100D7000001FF8001FF800018000018000018000C2
:100D800001800001800001800001800001800001DD
:100D900080000180001FF8001FF800000000000024
:100DA0000000000000000000000000000000000043
:100DB00000000000000000000007FE0007FE000029
:100DC00030000030000030000030000030003030D3
:100DD000003030003030003030003060003FE00044
:100DE0000F80000000000000000000000000000074
:100DF00000000000000000000000000000000000F3
:100E0000007F3E007F3E0018300018600018C000D0
:100E10001980001B80001FC0001CE0001870001823
:100E200030001838007F1F007F1F00000000000006
:100E300000000000000000000000000000000000B2
:100E40000000000000000000007F80007F80000C98
:100E500000000C00000C00000C00000C00000C0056
:100E6000000C0C000C0C000C0C000C0C007FFC00A7
:100E70007FFC0000000000000000000000000000F7
:100E80000000000000000000000000000000000062
:100E900000F00F00F81F00381C003C3C003C3C00F8
:100EA000366C00366C0033CC0033CC00318C003013
:100EB0000C00300C00FE7F00FE7F000000000000F0
:100EC0000000000000000000000000000000000022
:100ED00000000000000000000078FE0078FE001C0A
:100EE00018001E18001F18001B18001B980019D8A6
:100EF0000018D80018F8001878001838007F18007B
:100F00007F1800000000000000000000000000004A
:100F100000000000000000000000000000000000D1
:100F20000003C0000FF0001C3800181800381C0027
:100F3000300C00300C00300C00300C00381C001855
:100F400018001C38000FF00003C000000000000073
:100F50000000000000000000000000000000000091
:100F60000000000000000000003FF0003FF8000C0F
:100F70001C000C0C000C0C000C0C000C18000FF8E2
:100F8000000FE0000C00000C00000C00003FC0004F
:100F90003FC0000000000000000000000000000052
:100FA0000000000000000000000000000000000041
:100FB0000003C0000FF0001C3800181800381C0097
:100FC000300C00300C00300C00300C00381C0018C5
:100FD00018001C38000FF00007C00007CC000FFC01
:100FE000000C3800000000000000000000000000BD
:100FF0000000000000000000007FE0007FF000180B
:1010000038001818001818001838001FF0001FC00A
:101010000018E0001870001830001838007F1E001B
:101020007F0E000000000000000000000000000033
:1010300000000000000000000000000000000000B0
:101040000007D8000FF8001C380018180018180006
:101050001E00000FC00003F00000780018180018F0
:1010600018001C38001FF0001BE00000000000000A
:101070000000000000000000000000000000000070
:101080000000000000000000003FFC003FFC0031B9
:101090008C00318C00318C00318C0001800001808B
:1010A000000180000180000180000180000FF0003D
:1010B0000FF0000000000000000000000000000031
:1010C0000000000000000000000000000000000020
:1010D000007E7E007E7E0018180018180018180088
:1010E00018180018180018180018180018180018F8
:1010F00018000C30000FF00003C0000000000000DA
:1011000000000000000000000000000000000000DF
:101110000000000000000000007F7F007F7F0018BB
:101120000C000C18000C18000C18000630000630DB
:101130000003600003600003600001C00001C00004
:10114000008000000000000000000000000000001F
:10115000000000000000000000000000000000008F
:1011600000FE3F80FE3F80300600300600308600E3
:1011700019CC0019CC001B6C001B6C001E7C000EEF
:1011800038000E38000C18000C1800000000000099
:10119000000000000000000000000000000000004F
:1011A0000000000000000000007E7E007E7E00182F
:1011B00018000C300006600003C0000180000180B0
:1011C0000003C0000660000C30001818007E7E008E
:1011D0007E7E000000000000000000000000000013
:1011E00000000000000000000000000000000000FF
:1011F000007C7E007C7E001818000C300006600029
:1012000006600003C0000180000180000180000131
:1012100080000180000FF0000FF0000000000000CF
:1012200000000000000000000000000000000000BE
:101230000000000000000000001FF8001FF8001868
:10124000180018300018600018C00001800003006A
:10125000000618000C18001818003018003FF8009D
:101260003FF8000000000000000000000000000047
:10127000000000000000000000000000000001F07D
:101280000001F00001800001800001800001800069
:1012900001800001800001800001800001800001C8
:1012A000800001800001800001800001800001F0C9
:1012B0000001F0000000000000000000000000003D
:1012C0001800001800001C00000C00000E000006B2
:1012D0000000060000030000030000018000018000
:1012E0000000C00000C0000060000060000070004E
:1012F0000030000038000018000018000000000056
:1013000000000000000000000000000000000F804E
:10131000000F80000180000180000180000180003A
:101320000180000180000180000180000180000137
:1013300080000180000180000180000180000F809A
:10134000000F80000000000000000000000000000E
:1013500000000000800001C00003E00007700006EC
:1013600030000C1800180C001004000000000000F1
:10137000000000000000000000000000000000006D
:10138000000000000000000000000000000000005D
:10139000000000000000000000000000000000004D
:1013A000000000000000000000000000000000003D
:1013B000000000000000000000000000000000002D
:1013C000000000000000000000000000000000001D
:1013D00000000000000000000000FFFF00FFFF0011
:1013E00000000003000003800000E0000060000037
:1013F00000000000000000000000000000000000ED
:1014000000000000000000000000000000000000DC
:1014100000000000000000000000000000000000CC
:1014200000000000000000000000000000000000BC
:10143000000000000000000000000FC0001FE000DE
:1014400000300000300007F0001FF000383000309E
:1014500030003070001FFC000FBC000000000000D6
:10146000000000000000000000000000000000007C
:10147000000000000000780000780000180000184C
:1014800000001BE0001FF8001C1800180C00180CCE
:1014900000180C00180C00180C001C18007FF80035
:1014A0007BE00000000000000000000000000000E1
:1014B000000000000000000000000000000000002C
:1014C0000000000000000000000003EC000FFC0022
:1014D0001C1C00380C00300C0030000030000038BC
:1014E0000C001C1C000FF80003F0000000000000BE
:1014F00000000000000000000000000000000000EC
:1015000000000000000000780000780000180000D3
:10151000180007D8001FF8001838003018003018DD
:10152000003018003018003018001838001FFE0076
:1015300007DE0000000000000000000000000000C6
:10154000000000000000000000000000000000009B
:101550000000000000000000000007E0001FF8008D
:10156000181800300C003FFC003FFC003000003039
:101570000000180C001FFC0007F000000000000035
:10158000000000000000000000000000000000005B
:1015900000000000000001FC0003FC000600000643
:1015A00000003FF8003FF8000600000600000600BB
:1015B000000600000600000600000600003FF000E4
:1015C0003FF00000000000000000000000000000EC
:1015D000000000000000000000000000000000000B
:1015E0000000000000000000000007DE001FFE00F9
:1015F000183800301800301800301800301800304B
:1016000018001838001FF80007D80000180000184C
:10161000000038000FF0000FC000000000000000C4
:10162000000000000000780000780000180000189A
:1016300000001BE0001FF0001C38001818001818EC
:10164000001818001818001818001818007E7E00DE
:101650007E7E00000000000000000000000000008E
:1016600000000000000000000000000000000180F9
:10167000000180000000000000001F80001F8000AB
:1016800001800001800001800001800001800001D4
:1016900080000180003FFC003FFC000000000000D3
:1016A000000000000000000000000000000000003A
:1016B00000000000000000C00000C00000000000AA
:1016C00000001FF0001FF00000300000300000306C
:1016D000000030000030000030000030000030001A
:1016E0000030000030000030000070001FE0001FDC
:1016F00080000000000000000000000000003C002E
:10170000003C00000C00000C00000CF8000CF8007D
:101710000CC0000D80000F80000F00000F80000D36
:10172000C0000CE0003C7C003C7C0000000000009D
:1017300000000000000000000000000000000000A9
:101740000000000000001F80001F800001800001D9
:101750008000018000018000018000018000018084
:10176000000180000180000180000180003FFC003A
:101770003FFC00000000000000000000000000002E
:101780000000000000000000000000000000000059
:1017900000000000000000000000F77800FFFC00DF
:1017A00039CC00318C00318C00318C00318C00310F
:1017B0008C00318C00FDEF00FDEF00000000000008
:1017C0000000000000000000000000000000000019
:1017D0000000000000000000000000000000000009
:1017E00000007BE0007FF0001C380018180018187B
:1017F000001818001818001818001818007E7E002D
:101800007E7E0000000000000000000000000000DC
:1018100000000000000000000000000000000000C8
:101820000000000000000000000003C0000FF000F6
:101830001C3800381C00300C00300C00300C003814
:101840001C001C38000FF00003C000000000000066
:101850000000000000000000000000000000000088
:101860000000000000000000000000000000000078
:1018700000007BE0007FF8001C1800180C00180C1A
:1018800000180C00180C00180C001C18001FF800A1
:101890001BE0001800001800001800007F00007F07
:1018A0000000000000000000000000000000000038
:1018B0000000000000000000000007DE001FFE0026
:1018C0001838003018003018003018003018003078
:1018D00018001838001FF80007D80000180000187A
:1018E0000000180000FE0000FE00000000000000E4
:1018F00000000000000000000000000000000000E8
:1019000000003E78003EFC0007CC00070000060007
:10191000000600000600000600000600003FF00080
:101920003FF0000000000000000000000000000088
:1019300000000000000000000000000000000000A7
:101940000000000000000000000007F8000FF80091
:101950001818001818001F80000FF00000F8001879
:1019600018001838001FF0001FE000000000000001
:101970000000000000000000000000000000000067
:101980000000000000000C00000C00000C00000C27
:1019900000003FF0003FF0000C00000C00000C00C5
:1019A000000C00000C00000C00000C1C0007FC00E8
:1019B00003F0000000000000000000000000000034
:1019C0000000000000000000000000000000000017
:1019D0000000000000000000000078780078780027
:1019E00018180018180018180018180018180018EF
:1019F00018001838000FFE0007DE0000000000008D
:101A000000000000000000000000000000000000D6
:101A100000000000000000000000000000000000C6
:101A200000007C3E007C3E001818001818000C30A6
:101A3000000C300006600006600007E00003C000F4
:101A400003C00000000000000000000000000000D3
:101A50000000000000000000000000000000000086
:101A600000000000000000000000783C00783C000E
:101A70003118003398003398001AB0001EF0001E91
:101A8000F0001C60000C60000C6000000000000012
:101A90000000000000000000000000000000000046
:101AA0000000000000000000000000000000000036
:101AB00000003E7C003E7C000C300006600003C04D
:101AC0000001800003C0000660000C30003E7C0076
:101AD0003E7C00000000000000000000000000004C
:101AE00000000000000000000000000000000000F6
:101AF000000000000000000000007E1F007E1F00AC
:101B0000180C000C18000C180006300006300003FA
:101B1000600003E00001C00000C0000180000180FF
:101B2000000300003FC0003FC000000000000000B4
:101B300000000000000000000000000000000000A5
:101B400000001FF8001FF80018300018600000C0E7
:101B5000000180000300000618000C18001FF800A8
:101B60001FF800000000000000000000000000005E
:101B7000000000000000000000000000000000E085
:101B80000001E00001800001800001800001800070
:101B90000180000180000380000700000380000135
:101BA000800001800001800001800001800001E0D0
:101BB0000000E00000000000000000000000000045
:101BC0000000000000000180000180000180000191
:101BD0008000018000018000018000018000018000
:101BE0000001800001800001800001800001800070
:101BF00001800001800001800001800000000000E1
:101C000000000000000000000000000000000700CD
:101C10000007800001800001800001800001800039
:101C200001800001800001C00000E00001C000014F
:101C30008000018000018000018000018000078099
:101C4000000700000000000000000000000000008D
:101C50000000000000000000000000000000000084
:101C600000000000000000000E00001F18003BB83C
:101C70000031F00000E00000000000000000000063
:101C80000000000000000000000000000000000054
:101C90000000000000000000000000000000000044
:101CA0000000000000000000000000000000000034
:101CB0000000000000000000000000000000000024
:101CC00000000700070007000700070007000700E3
:101CD00002000200000000000700070000000000F2
:101CE0000000000000000000000000001CE01CE0FC
:101CF0001CE0084008400840000000000000000010
:101D000000000000000000000000000000000000D3
:101D10000CC00CC00CC00CC00CC03FF03FF00CC09D
:101D20000CC03FF03FF00CC00CC00CC00CC00CC08D
:101D300000000000000000000300030007E00FE0C7
:101D4000186018001F000FC000E0186018601FC066
:101D50001F800300030003000000000000000000DB
:101D600000001C002200220022001C6001E00F8005
:101D70003C0031C002200220022001C0000000000F
:101D8000000000000000000000000000000003E070
:101D90000FE00C000C0006000F301FF019E018C017
:101DA0001FF007B00000000000000000000000006D
:101DB0000000000003800380038001000100010097
:101DC0000000000000000000000000000000000013
:101DD0000000000000000000000000C000C0018002
:101DE00001800180030003000300030003000300DF
:101DF00001800180018000C000C0000000000000E0
:101E000000000C000C0006000600060003000300A2
:101E100003000300030003000600060006000C0098
:101E20000C0000000000000000000300030003009D
:101E30001B601FE0078007800FC00CC0000000007F
:101E40000000000000000000000000000000000092
:101E500000000000000003000300030003003FF047
:101E60003FF0030003000300030000000000000037
:101E70000000000000000000000000000000000062
:101E800000000000000000000000000000000380CF
:101E9000030003000600060004000000000000002C
:101EA00000000000000000000000000000003FE013
:101EB0003FE0000000000000000000000000000003
:101EC0000000000000000000000000000000000012
:101ED000000000000000000000000000000003807F
:101EE00003800380000000000000000000000000EC
:101EF0000060006000C000C000C0018001800300DD
:101F00000300060006000C000C000C00180018006E
:101F1000000000000000000000000F801FC018C07B
:101F2000306030603060306030603060306018C0E9
:101F30001FC00F8000000000000000000000000033
:101F4000000003001F001F00030003000300030044
:101F500003000300030003001FE01FE00000000077
:101F6000000000000000000000000F801FC038E0EB
:101F70003060006000C00180030006000C00180003
:101F80003FE03FE000000000000000000000000013
:101F900000000F803FC030E0006000E007C007C0D5
:101FA00000E00060006060E07FC03F800000000053
:101FB0000000000000000000000001C003C003C0DA
:101FC00006C00CC00CC018C030C03FE03FE000C0ED
:101FD00003E003E00000000000000000000000003B
:101FE00000001FC01FC0180018001F801FC018E08D
:101FF00000600060006030E03FC01F800000000013
:102000000000000000000000000003E00FE01E00E0
:102010001800380037803FC038E03060306018E08A
:102020001FC007800000000000000000000000004A
:1020300000003FE03FE03060006000C000C000C032
:102040000180018001800300030003000000000004
:10205000000000000000000000000F801FC038E0FA
:10206000306038E01FC01FC038E03060306038E0BA
:102070001FC00F80000000000000000000000000F2
:1020800000000F001FC038C03060306038E01FE033
:102090000F6000E000C003C03F803E000000000071
:1020A0000000000000000000000000000000000030
:1020B0000000038003800380000000000000038014
:1020C000038003800000000000000000000000000A
:1020D0000000000000000000000001C001C001C0BD
:1020E000000000000000038003000600060004005A
:1020F00000000000000000000000000000000030B0
:1021000000F003C007001C0078001C00070003C09B
:1021100000F000300000000000000000000000009F
:10212000000000000000000000007FF07FF00000D1
:1021300000007FF07FF000000000000000000000C1
:10214000000000000000000000000000000030005F
:102150003C000F00038000E0007800E003800F00E7
:102160003C00300000000000000000000000000003
:10217000000000000F801FC018601860006001C0E0
:1021800003800300000000000700070000000000BB
:102190000000000000000000000003800C800840E8
:1021A0001040104011C012401240124011C01000E7
:1021B0000800084007800000000000000000000048
:1021C000000000001F801F80038006C006C00CC0F6
:1021D0000C601FE01FE03030787878780000000055
:1021E0000000000000000000000000003F803FC031
:1021F0001860186018E01FC01FE018701830183001
:102200003FF03FE000000000000000000000000080
:102210000000000007B00FF01C70383030003000B4
:102220003000300038301C700FE007C000000000A4
:102230000000000000000000000000007F807FC060
:1022400030E030703030303030303030307030E0AE
:102250007FC07F8000000000000000000000000040
:10226000000000003FF03FF01830183019801F8048
:102270001F801980183018303FF03FF00000000038
:102280000000000000000000000000003FF03FF0F0
:102290001830183019801F801F801980180018000E
:1022A0003F003F00000000000000000000000000B0
:1022B0000000000007B01FF0187030303000300010
:1022C00031F831F8303018301FF007C0000000003E
:1022D0000000000000000000000000003CF03CF0A6
:1022E0001860186018601FE01FE018601860186020
:1022F0003CF03CF000000000000000000000000086
:10230000000000001FE01FE00300030003000300C3
:1023100003000300030003001FE01FE000000000B3
:1023200000000000000000000000000003F803F8B7
:10233000006000600060006030603060306030E05D
:102340003FC00F80000000000000000000000000FF
:10235000000000003EF83EF818E019801B001F0046
:102360001D8018C018C018603E783E38000000007C
:102370000000000000000000000000003F003F00DF
:102380000C000C000C000C000C000C300C300C305D
:102390003FF03FF0000000000000000000000000DF
:1023A000000000007878787838703CF034B037B0AE
:1023B00037B03330333030307CF87CF80000000028
:1023C00000000000000000000000000039F03DF0B7
:1023D0001C601E601E601B601B6019E019E018E0A5
:1023E0003EE03E6000000000000000000000000031
:1023F0000000000007800FC01CE038703030303023
:102400003030303038701CE00FC007800000000012
:102410000000000000000000000000003FC03FE09E
:1024200018701830183018701FE01FC018001800FE
:102430003F003F000000000000000000000000001E
:102440000000000007800FC01CE0387030303030D2
:102450003030303038701CE00FC0078007B00FF00C
:102460000CE0000000000000000000003FC03FE062
:102470001870183018701FE01FC018E0186018702E
:102480003E383E1800000000000000000000000080
:10249000000000000FB01FF03870303038001F808F
:1024A00007E00070303038703FE037C000000000B7
:1024B0000000000000000000000000003FF03FF0BE
:1024C00033303330333003000300030003000300D4
:1024D0000FC00FC00000000000000000000000005E
:1024E000000000003CF03CF01860186018601860B4
:1024F0001860186018601CE00FC007800000000022
:1025000000000000000000000000000078F078F0FB
:102510003060306018C018C00D800D800D8007003D
:10252000070007000000000000000000000000009D
:10253000000000007C7C7C7C301833983398339802
:1025400036D816D01C701C701C70183000000000AB
:1025500000000000000000000000000078F078F0AB
:10256000306018C00D80070007000D8018C0306073
:1025700078F078F00000000000000000000000008B
:10258000000000003CF03CF018600CC007800780A1
:1025900003000300030003000FC00FC00000000091
:1025A0000000000000000000000000001FE01FE02D
:1025B000186018C001800300030006000C6018605A
:1025C0001FE01FE00000000000000000000000000D
:1025D000000003C003C00300030003000300030066
:1025E000030003000300030003000300030003C013
:1025F00003C0000000000000180018000C000C00D0
:102600000C0006000600030003000180018000C0EA
:1026100000C000C00060006000000000000000007A
:1026200000000F000F00030003000300030003007D
:1026300003000300030003000300030003000F0076
:102640000F000000000000000000020007000D80E5
:1026500018C03060202000000000000000000000D2
:10266000000000000000000000000000000000006A
:10267000000000000000000000000000000000005A
:10268000000000000000000000000000000000004A
:1026900000000000FFFCFFFC0000040003000080BD
:1026A000000000000000000000000000000000002A
:1026B000000000000000000000000000000000001A
:1026C000000000000000000000000FC01FE00060DC
:1026D0000FE01FE0386030E03FF01F7000000000A6
:1026E00000000000000000000000700070003000DA
:1026F000300037803FE03860303030303030386084
:102700007FE0778000000000000000000000000073
:102710000000000000000000000007B01FF01830AB
:1027200030303000300038301FF00FC000000000A3
:102730000000000000000000000000700070003089
:10274000003007B01FF01870303030303030387043
:102750001FF807B8000000000000000000000000A3
:102760000000000000000000000007801FE018606B
:102770003FF03FF0300018301FF007C000000000AD
:102780000000000000000000000003F007F0060059
:1027900006001FE01FE00600060006000600060017
:1027A0001FE01FE00000000000000000000000002B
:1027B0000000000000000000000007B81FF81870BB
:1027C00030303030303018701FF007B000300070FB
:1027D0000FE00FC0000000000000380038001800B3
:1027E00018001BC01FE01C6018601860186018609B
:1027F0003CF03CF000000000000000000000000081
:10280000000003000300000000001F001F00030081
:1028100003000300030003001FE01FE000000000AE
:1028200000000000000000000000030003000000A2
:1028300000001FC01FC000C000C000C000C000C01A
:1028400000C000C000C001C03F803F000000000089
:10285000000038003800180018001BE01BE01B00C7
:102860001E001E001B00198039F039F00000000026
:10287000000000000000000000001F001F00030017
:102880000300030003000300030003000300030030
:102890001FE01FE00000000000000000000000003A
:1028A000000000000000000000007EE07FF03330F8
:1028B00033303330333033307BB87BB80000000026
:1028C0000000000000000000000000000000000008
:1028D00000003BC03FE01C60186018601860186082
:1028E0003CF03CF000000000000000000000000090
:1028F0000000000000000000000007801FE01860DA
:1029000030303030303018601FE0078000000000A9
:1029100000000000000000000000000000000000B7
:10292000000077807FE03860303030303030386001
:102930003FE03780300030007C007C000000000069
:102940000000000000000000000007B81FF8187029
:1029500030303030303018701FF007B000300030A9
:1029600000F800F800000000000000000000000077
:1029700000003CE03DF00F300E000C000C000C009D
:102980003FC03FC000000000000000000000000049
:102990000000000000000000000007E01FE01860D9
:1029A0001E000FC001E018601FE01F800000000043
:1029B0000000000000000000000000000C000C00FF
:1029C0000C003FE03FE00C000C000C000C000C3051
:1029D0000FF007C000000000000000000000000031
:1029E0000000000000000000000038E038E018603F
:1029F00018601860186018E01FF00F7000000000E9
:102A000000000000000000000000000000000000C6
:102A1000000078F078F0306018C018C00D800D808C
:102A20000700070000000000000000000000000098
:102A30000000000000000000000078F078F0326034
:102A4000326037E01DC01DC018C018C00000000073
:102A50000000000000000000000000000000000076
:102A600000003CF03CF00CC00780030007800CC065
:102A70003CF03CF0000000000000000000000000FE
:102A80000000000000000000000078F078F03060E6
:102A900018C018C00D800F800700060006000C004B
:102AA0007F007F0000000000000000000000000028
:102AB00000001FE01FE018C00180030006000C604A
:102AC0001FE01FE000000000000000000000000008
:102AD000000001C003C00300030003000300030063
:102AE00007000E000700030003000300030003C0FB
:102AF00001C000000000000000000300030003000C
:102B000003000300030003000300030003000300AD
:102B100003000300030003000300000000000000A6
:102B200000001C001E00060006000600060006004D
:102B300007000380070006000600060006001E00CE
:102B40001C00000000000000000000000000000069
:102B5000000000000E003F3033F001E000000000F4
:102B60000000000000000000000000000000000065
:102B70000000000000000000000000000010101025
:102B80001010000010000000006C48480000000019
:102B900000000000001414287C287C2850500000FD
:102BA00000103840403848701010000000205020BD
:102BB0000C70081408000000000000182020544881
:102BC0003400000000101010100000000000000091
:102BD0000008081010101010100808000020201025
:102BE000101010101020200000107C102828000069
:102BF000000000000000101010FE10101000000077
:102C0000000000000000001810302000000000004C
:102C1000007C000000000000000000000000003008
:102C200030000000000404080810102020400000BC
:102C3000003844444444444438000000003010103C
:102C4000101010107C0000000038440408102044CC
:102C50007C000000003844041804044438000000DC
:102C6000000C141424447E040E000000003C2020BC
:102C70003804044438000000001C204078444444D8
:102C800038000000007C4404080808101000000010
:102C90000038444438444444380000000038444478
:102CA000443C040870000000000000303000003098
:102CB000300000000000001818000018302000004C
:102CC00000000C10608060100C000000000000008C
:102CD0007C007C00000000000000C02018041820C8
:102CE000C00000000000182404081000300000009C
:102CF0003844444C54544C404438000000301028B0
:102D000028287C44EE00000000F844447844444401
:102D1000F8000000003C44404040404438000000BF
:102D200000F0484444444448F000000000FC445093
:102D300070504044FC000000007E222838282020EB
:102D400070000000003C4440404E44443800000005
:102D500000EE44447C444444EE000000007C10102B
:102D6000101010107C000000003C0808084848487B
:102D70003000000000EE444850704844E600000077
:102D800000702020202024247C00000000EE6C6CC9
:102D900054544444EE00000000EE64645454544C17
:102DA000EC0000000038444444444444380000002F
:102DB0000078242424382020700000000038444487
:102DC00044444444381C000000F8444444784844D7
:102DD000E200000000344C40380404645800000055
:102DE00000FE9210101010103800000000EE444455
:102DF000444444443800000000EE4444282828108D
:102E00001000000000EE44445454545428000000C4
:102E100000C6442810102844C600000000EE4428D4
:102E20002810101038000000007C440810102044C6
:102E30007C000000003820202020202020203800A6
:102E40000040202020101008080800000038080862
:102E5000080808080808380000101028440000007E
:102E6000000000000000000000000000000000FE64
:102E70000010080000000000000000000000003802
:102E8000443C44443E00000000C040586444444474
:102E9000F80000000000003C4440404438000000BE
:102EA000000C04344C4444443E0000000000003850
:102EB000447C40403C000000001C207C202020205E
:102EC0007C000000000000364C4444443C043800C0
:102ED00000C0405864444444EE00000000100070FC
:102EE000101010107C00000000100078080808087E
:102EF0000808700000C0405C48705048DC000000CA
:102F000000301010101010107C000000000000E8CD
:102F100054545454FE000000000000D8644444445B
:102F2000EE00000000000038444444443800000033
:102F3000000000D8644444447840E00000000036BB
:102F40004C4444443C040E000000006C302020201F
:102F50007C0000000000003C44380444780000007D
:102F60000000207C202020221C000000000000CC5B
:102F70004444444C36000000000000EE444428283D
:102F800010000000000000EE4454545428000000DB
:102F9000000000CC48303048CC000000000000EEBB
:102FA00044242818101078000000007C48102044A9
:102FB0007C000000000810101010201010100800F5
:102FC0000010101010101010101000000020101031
:102FD00010100810101020000000000000245800FD
:102FE000000000004178007807E08278C17842EA6A
:102FF00001224178007841EA022140EA012070472D
:103000000170090A417070470170090A4170090A8C
:103010008170090AC17070472AB111F8013B521E34
:1030200000F8013BF9D17047521E00F8011BFBD19B
:10303000704702781AB18A4218BF401CF9D1104675
:103040007047002800D1704780B5006901F0F1FF9A
:1030500000B1012002BD002882B018BF0C2907D0A2
:103060000B2918BF0F2903D0006902B001F0EBBF94
:1030700002B07047F0B5024600230024854D05EBF1
:103080000416306880B11768B84202BF706897684C
:10309000B84202BFB0685669B04206D1022C0AD1CC
:1030A00093B9022905D10FE00123641C022CE6D359
:1030B000F4E71220F0BD29B905EB04108289B2F5BE
:1030C000807F01D11020F0BD0020F0BDF8B50022B6
:1030D0004369856806686F4F140157F804C0B4450A
:1030E00002BF07F1040C5CF804C0AC4502BF07F155
:1030F000080C5CF804409C4202D0521C012AEBD917
:10310000022A11D13C680022002C1EBF01223B691B
:10311000002B0ED11301FC1826606560406907F191
:103120000805E8500020A08107EB0213988929B117
:1031300008B10020F2BD4FF4807000E0401C98817F
:10314000501CF2BD401E022818B513D2000151498F
:103150000A189389B3F5807F01D01C0002D10023A7
:10316000938103E05B1E93819BB20BB900220A504E
:10317000002012BD022012BD10B50021454A0B01EE
:10318000D458844204BF0024D450491C0129F6D9E4
:1031900010BDF8B505460024E878F0B16E6B68788C
:1031A000012305F13801324601F074FF08B1012412
:1031B00013E0A86A296AEC70301A88420DD2AF7801
:1031C00009E0286A012305F138017F1E8619687815
:1031D000324601F05FFF012FF3D82046F2BD70B5F3
:1031E00004460D46606B0026854210D02046FFF74E
:1031F000D0FF06000BD1607801232A4604F1380184
:1032000001F042FF10B14FF0FF35012665633046F3
:1032100070BD38B50446FFF7BCFF050037D12078F4
:10322000032804BF217901292AD101F0E1FE04F12C
:103230003800FFF7F9FE4AF6552104F23620FFF771
:10324000DFFE154904F13800FFF7DEFE134904F5EF
:103250000770FFF7D9FEA16904F50870FFF7D4FEE7
:10326000616904F50970FFF7CFFE626A6078012397
:1032700004F13801521C626301F00CFF0020207140
:1032800060780022002101F013FF00B101252846DB
:1032900032BD00007CAE0320525261417272416126
:1032A000C269891E921E914201D300207047438952
:1032B000006B03FB0101084670472DE9F0410C4605
:1032C000022C05684CD3E869844249D228784FF033
:1032D000FF36012804D043D3032830D01FD33FE06A
:1032E000A96A04EB540700F0B5F8002839D105F1BC
:1032F0003800C7F3080110F80180A96A7F1C00F0AC
:10330000A9F870BB05F13800C7F30807C05DE107F5
:1033100048EA002654BFC6F30B06360921E0A96A25
:10332000284601EB1421FFF75AFFD0B905F1380008
:10333000240600EBD450FFF755FE064611E0A96ABB
:10334000284601EBD411FFF74AFF50B905F13800C8
:10335000640600EBD450FFF748FE20F0704600E012
:1033600001263046BDE8F0812DE9F0410E46022EDF
:10337000054614464FF0020869D3E869864266D2D2
:103380002878012804D062D3032844D031D35EE0EA
:10339000A96A06EB560700F05DF85FEA000856D10F
:1033A00005F13800C7F3080108447F1CF10743BF4B
:1033B000017801F00F0141EA04112146017001205A
:1033C000A96AE87000F046F85FEA00083FD105F10D
:1033D0003800C7F30807C019F10748BF240906D40D
:1033E0000178240A04F00F0401F0F0010C4304708A
:1033F0002BE0A96A284601EB1621FFF7F0FE5FEAF1
:10340000000824D105F13800360600EBD650A1B2F1
:10341000FFF7F6FD19E0A96A284601EBD611FFF780
:10342000DEFE5FEA000812D105F13800760600EBF7
:10343000D65624F070443046FFF7D7FD00F07040B8
:1034400040EA04013046FFF7DFFD0120E870404606
:10345000BDE8F081284601EB5721C0E6F8B50546E6
:103460000F46012F11462E6829D9F069874226D2CE
:1034700029B14FF0FF3200F078F801001ED1394633
:103480002846FFF71AFF040017D0012C17D014F1BB
:10349000010F16D0002200F067F801000ED1F0698C
:1034A000B169821E914205D2491CB161317941F066
:1034B0000101317127468742E1D30020F2BD02208D
:1034C000F2BD0120F2BD2DE9F0410C008046D8F894
:1034D000006006D1756915B1F06985420ED30125EA
:1034E0000CE0FFF7EAFE012898BF01203AD910F15D
:1034F000010F37D0F169884234D325462F46F06951
:103500007F1C874202D30227012D0BD93946404642
:10351000FFF7D3FE40B1012818BF10F1010F21D0F1
:10352000AF42ECD100201DE04FF0FF3200F01CF85C
:1035300020B924B13A46214600F017F860B9776106
:10354000F169B069891E814224BF401EB0613079A3
:1035500040F00100307104E001280CBF4FF0FF374C
:1035600001273846BDE8F08139463046FCE6C26A9C
:103570000068490A4389121DB1FBF3F003E0884259
:1035800006D3401A083211680029F8D1002070478C
:103590005168081870472DE9FC410E460546B6F5FE
:1035A000001F2F683AD216F01F0F37D1AC686E613A
:1035B0001CB93878032801DBFC6A2CB93889490921
:1035C00081422BD2F86A24E0B7F80A8006E0022C88
:1035D00024D3F869844221D2A6EB4826B6EB482FC3
:1035E000214614D32846FFF768FE044614F1010F64
:1035F000EDD1012009E000EB5620C6F30806E86192
:10360000B81900F1380100202962BDE8F68100F008
:1036100077F8E861E869AC610028ECD10220F4E7B2
:103620002DE9F04106460C467569F069376820358A
:1036300010B3B5F5001F1FD2E90556D1B169401C82
:10364000F06121B93989680988424ED312E078893E
:10365000401E10EA552F48D13046FFF72EFE804617
:10366000B8F1010F16D918F1010F34D0F86980456F
:1036700036D31CB90020F06104203EE0B169304629
:10368000FFF721FF5FEA000808BF072035D0B8F137
:10369000010F01D1022030E018F1010F1BD0384694
:1036A000FFF777FDB8B901F0A3FC07F1380000245B
:1036B000FFF7BAFC00F023F802E0786B641C401CB2
:1036C000798978638C4208D201213846F970FFF776
:1036D00060FD0028F1D001200FE0786B041B7C63B3
:1036E000C6F8188000F00BF8F061756107F138003A
:1036F000C5F30805401930620020BDE8F08141465D
:103700003846CDE570B504460D4605F11A00FFF7C1
:1037100069FC21780646032905D105F11400FFF75D
:1037200061FC46EA0046304670BD70B504460D4661
:103730001646B1B205F11A00FFF762FC21780329A1
:1037400005D1310C05F11400BDE8704058E470BD9E
:103750007CB5164605461C460B22FFF75DFC062C81
:1037600014D310E036F8021B1020224601F00104A9
:1037700004EB42044908E20344BF84F4883484F033
:103780002104401EF1D130880028EBD1072004F03D
:103790000F023032D3B23A2BA8BFD21D0DF8002051
:1037A000401E2409F3D17E220DF80020002200E003
:1037B000521C824202D2AB5C202BF9D113465A1C18
:1037C00007289ABF1DF80040401C2024072AEC540B
:1037D000F4D973BD024600200B210306C00100EBA3
:1037E000536012F8013BC018491EF6D1C0B27047B1
:1037F0002DE9F34F81B004462068FF264FF00408FE
:103800000090B146E169002976D001F0FCFB002868
:10381000804671D1276A3878002846D0F97AE528A1
:1038200018BF2E2801F03F01A1715FD021F02002C6
:10383000082A029B14BF002201229A4256D10F2966
:1038400049D1410606D597F80D9000F0BF00616997
:1038500006462163F1B2884204BF797B894545D190
:103860000098D0F80C8007F11A00FFF7BBFB002886
:103870003CD13D780D204FF0010A4FF0000B25F0B0
:1038800040056D1E45430FF2C03010F80B00384460
:10389000FFF7A8FBBAF1000F0AD0FF2D3EBF82460A
:1038A00028F815A06D1C07D320E04FF0040826E08F
:1038B0004FF6FF71884219D10BF1010BBBF10D0FCF
:1038C000E1D33878410604D5FF2D0FD2002128F826
:1038D0001510761E0BE04FF0FF35F6B226B93846CC
:1038E000FFF778FF81450CD025630AE0FF2600F042
:1038F000B4F80028804685D0B8F1000F01D0002030
:10390000E0614046BDE8FE8F2DE9FE4F04460021F0
:10391000206801902046FFF73EFE5FEA00080BD1C9
:10392000FF214FF0FF300091FF252063E1690198EE
:10393000FFF755FC5FEA000877D1266A3078002847
:103940004AD0F17AE52801F03F01A17163D00A075E
:1039500045D50F295FD194F82F104A065FD442064F
:1039600006D5717B00F0BF000546009161692163B7
:10397000E9B2884202BF0098717B88426BD10198FE
:10398000D0F80C8006F11A00FFF72CFB002862D15A
:1039900037780D204FF0010B4FF0000907F03F077B
:1039A0007F1E47430FF2A02010F809003044FFF7B4
:1039B00019FBBBF1000F824638D0FF2F4BD201F02C
:1039C000A7FB834638F817007F1C01F0A1FB834555
:1039D00008BFD3462ED03EE04FF0040825E00F2963
:1039E000B9D0EDB22DB9009D3046FFF7F3FE854208
:1039F0001BD094F82F00C1070DD4226A04F12403D0
:103A00000B2112F8015B13F8010B281A491E01D093
:103A10000028F6D048B14FF0FF30FF25206300F0BA
:103A20001CF85FEA00083FF481AF6AE74FF6FF70C9
:103A3000824510D109F10109B9F10D0FB2D33178E6
:103A4000480606D5BBF1000F1CBF38F81700002848
:103A500001D16D1EE3E7FF25E1E700212046DFE508
:103A60002DE9F84F86B005462868009095F82F108C
:103A700011F0A00F18BF062040F0E2800027C168B7
:103A800000E07F1C31F817000028FAD10C2205F164
:103A9000240102A802ACFFF7BFFAE07AC10723D5E0
:103AA0004021012685F82F10DDF80080D8F80C2081
:103AB000334602A905F12400FFF74AFE2846FFF726
:103AC00023FF5FEA000902D1761C642EEED3642E38
:103AD000CDF8008008BF072000F0B280042840F035
:103AE000AE80E07A85F82F00E07A810705D50C37A3
:103AF0000D21B7FBF1F77F1C00E001272E680021A4
:103B00002846FFF748FD010016D10024E969304638
:103B1000FFF765FB01000FD1286A0078E5281CBF7C
:103B20000028002402D1641CBC4208D00121284690
:103B3000FFF776FD0100E9D0042908BF07215FEAFD
:103B4000010960D1B7F1010860D069692846A1EB8D
:103B50004811FFF720FD5FEA000954D105F1240068
:103B60004FF6FF77FFF736FE8DF8040001F04AFAB2
:103B70005FEA000947D100982C6AC1465FFA89F6CE
:103B8000761E4FF0000AC1680F2005919DF80410C1
:103B900061730021E0720020207304F11A00FFF726
:103BA0002FFA0D20464301E0BB4503D0059830F8BD
:103BB00016B0761C0FF29000594610F80A000AF170
:103BC000010A2018FFF71CFABBF1000F08BFBB4623
:103BD000BAF10C0FE8D9BB451DBF059830F81600A7
:103BE000002849F0400984F80090009A01212846F5
:103BF000D1700021FFF714FD5FEA000903D1B8F18D
:103C00000108B3D102E05FEA090018D101F0FAF926
:103C10005FEA000913D1286A20220021FFF704FA85
:103C2000286A0B2205F12401FFF7F6F995F82F0019
:103C3000296A012200F0180008730098C2704846F3
:103C400007B0BDE8F08F000001030507090E101250
:103C50001416181C1E00000070B50446216B256860
:103C6000666911F1010F0CBF0020FFF794FC010001
:103C700014D1E1692846FFF7B2FA01000BD1226A9C
:103C8000E52111700121E9706169B14206D2FFF7A7
:103C9000E4FE0100EDD0042808BF022070BD2DE92C
:103CA000F04104460D4626680020A875E06900280A
:103CB00041D0216B11F1010F46D00027B846F068C2
:103CC00030F817007F1C010039D0002101F000FA04
:103CD00098B3B8F1FF0F3EBF05F1160101F80800D7
:103CE00008F10108EBD328E0276A3F7B374218BF71
:103CF000203105F11606B154521C0B2B27D330B9D5
:103D000005F116018854216A087B00B900220023BE
:103D100005F109018B54206AC17A2972216A01F1E7
:103D20001C00FFF762F92860206A1630FFF75DF982
:103D3000E880000CA880BDE8F0814FF0000800206A
:103D400005F1160101F8080000220023A87D216A70
:103D5000C95C5B1C2029D0D0052908BFE521092BAF
:103D600009D118B92E2605F11607BE542E2605F1E5
:103D70000907BE54521C002805F10906B154BBD1F5
:103D8000A1F141061A2EB4D2092B2CBF1026082609
:103D9000AAE72DE9F34F81B080460E68D8F80010ED
:103DA000002500270FF2C01AD1F80C9015E0FF2D66
:103DB00080F0D8800121104601F08AF9040000F05B
:103DC000D180802C06DA21465046FFF732F90028D0
:103DD00040F0C88029F815406D1CF25D7F1C202A38
:103DE00009DB2F2A18BF5C2AE1D1F05D2F2814BF10
:103DF0005C287F1CF9D09BE008F124060B222021CF
:103E00003046FFF711F94FF00009504601E009F183
:103E1000010930F81910202918BF2E29F7D0B9F15F
:103E2000000FB84618BF44F00304811E31F8181083
:103E30002E2902D0B8F10108F7D14FF0000A002571
:103E400008270090A34600E08B46009830F8194000
:103E500009F1010974B1202C4BF00301F4D02E2C90
:103E600001D1C145F0D1BD4201D2C14534D10B2FA2
:103E700026D18B463178E52904BF05223270082F00
:103E800008BF4FEA8A0A0AF00C000C281ABF0AF091
:103E9000030103294BF0020B5FEA8B700BD40AF08D
:103EA000030001280AF00C0008BF4BF0100B042897
:103EB00008BF4BF0080B86F80BB00020BDE8FE8F62
:103EC000C14518BF8B46C84521BFC14608250B27F1
:103ED0004FEA8A0AB9D2CDE7802C0EDB00212046BA
:103EE00001F0F6F800284BF0020B1FBF0FF284011F
:103EF000081810F8804C002C05D00FF2F80021466D
:103F0000FFF797F818B15F244BF0030B0DE0A4F115
:103F100041001A2838BF4AF0020A06D3A4F1610111
:103F20001A293CBF4AF0010A203C74556D1C8CE7ED
:103F30000299F019202ACA4608602846ACBF00241E
:103F4000042440B1AAF1020131F81010202914BF55
:103F50002E29401EF5D007460020002F2AF8170012
:103F60007FF44AAF0620A9E7222A3A3C3E3F7C7FF5
:103F70000000000043554541414141434545454905
:103F8000494941414592924F4F4F5555594F554FD1
:103F90009C4F9E9F41494F55A5A5A6A7A8A9AAAB8E
:103FA000ACADAEAFB0B1B2B3B4414141B8B9BABB38
:103FB000BCBDBEBFC0C1C2C3C4C54141C8C9CACBD4
:103FC000CCCDCECFD1D145454549494949D9DADB98
:103FD000DCDD49DF4FE14F4F4F4FE6E8E8555555DF
:103FE0005959EEEFF0F1F2F3F4F5F6F7F8F9FAFBC0
:103FF000FCFDFEFF2B2C3B3D5B5D000033B581B02B
:104000000446256801E0511C0291029A10782F287D
:1040100018BF5C28F7D00020A06002980278202A00
:1040200016D28021204684F82F100021FFF7B3FA22
:10403000014622E008BBA079C1061DD5616928466A
:10404000C1F308016A1802F13801FFF75BFBA060B9
:1040500002A92046FFF79DFE01000ED12046FFF782
:1040600053FC014694F82F000A0000F00400E1D050
:10407000042908BF002800D1052108463EBD03469B
:104080004FF0FF301A68002A00D1704710B514466F
:104090002178202906D33A2918BF641CF8D101E001
:1040A000002010BD3A29FBD112F8011B30390A2932
:1040B000F7D2A24208BF0029F3D1611C0020196089
:1040C00010BD1CB504460020E0704FF0FF30606367
:1040D0002046FFF784F808B1042016BD04F236200C
:1040E000FEF780FF4AF65521884201D0032016BD15
:1040F00004F138000178E92904D0EB2904BF807865
:10410000902813D104F16E00FEF76FFF20F07F407E
:10411000DFF84815884207D004F18A00FEF765FFF2
:10412000DFF83C15884201D1002016BD022016BDE3
:104130002DE9FF410E46002114463160FFF79FFF35
:10414000070048BF0B2007D4DFF8188508F10400EA
:1041500050F827500DB90C200DE12846FEF771FFED
:1041600008B90F2007E13560287804F0FE0448B153
:10417000687800F071FFC10704D4002C01D040071B
:104180000DD4F7E0002028706F70687800F06DFFA4
:10419000C10748BF032003D41CB1400701D50A2042
:1041A000E9E0002128460026FFF78BFF02281ED1F8
:1041B000002405EB041101F5FB71087918B101F138
:1041C0000800FEF712FF4DF82400641C042CF0D305
:1041D0005DF8264024B121462846FFF772FF00E033
:1041E0000320022802DB761C042EF1D32646042885
:1041F00008BF0120D4D0022880F2818005F143005D
:10420000FEF7F0FEB0F5007F79D105F14E00FEF724
:10421000E9FE040004D105F15C00FEF7E6FE044669
:104220002C6205F14500C1780129A97018BF022947
:1042300065D14C4300780100688160D0411E08427E
:104240005DD105F14900FEF7CDFE10F00F0F28817A
:1042500055D105F14B00FEF7C5FE070004D105F16D
:104260005800FEF7C2FE074605F14600FEF7BAFE0B
:10427000002844D02989231803EB11139F423ED311
:104280006A89FF1AB7FBF2F2002A38D003274FF6EB
:10429000F67C624540F6F67C38BF0227624538BF9F
:1042A0000127921C8019EA619B19032F6E62A86294
:1042B0002B6310D105F16200FEF794FE002804BFC5
:1042C000288900281BD105F16400FEF78EFE044604
:1042D000E86980000CE091B1A86A2418E869022F0F
:1042E0000FBF400000EB400100F0010000EB510067
:1042F0002A6A00F2FF10EC62B2EB502F01D20D20BF
:1043000039E04FF0FF30A86168618020032F2871E9
:1043100026D105F16800FEF765FE012820D1711C49
:104320002846FEF75CFFD8B9287105F23620FEF763
:1043300059FE4AF65521884212D105F13800FEF7A0
:1043400054FEC94988420BD105F50770FEF74DFEB2
:10435000C649884204D105F50970FEF746FE68613A
:104360002F70B8F80000401CA8F80000E88028462C
:10437000FEF702FF002004B0BDE8F08138B504006C
:104380000D461CBF216800290AD0087840B1CA88B0
:10439000A3889A4204D1487800F05EFEC10703D595
:1043A00000210920296032BD206828602068FEF7BE
:1043B00048FE08B90F2032BD002032BDF3B581B0F0
:1043C000154600916846FFF75AFE060001D50B20FE
:1043D000FEBDA44901EB86077C6844B12046FEF788
:1043E000CBFE206900F020FE78B1002020700198FB
:1043F00010B90021796010E000210170019800F1EE
:104400001001F0B200F002FE08B90220FEBD0198D2
:104410007860019808B1012D01D00020FEBD002276
:1044200001A902A8FFF784FE044601982146FEF781
:1044300012FE2046FEBD2DE9F24304008EB008BFF7
:10444000092013D002F03F06324669460EA8FFF756
:104450006FFE050040F0F7800098019000F09DFC91
:104460005FEA000803D100F0A0FC1120F3E00098FF
:10447000C0F80C800E9901A8FFF7C0FD05000DD112
:104480009DF83300010648BF062507D416F0FE014B
:1044900001A818BF0121FEF7EDFD054616F01C0F1F
:1044A00000F0AC80280000F09F80042D4AD17048B5
:1044B000016800291EBF00690028122503D101A848
:1044C000FFF7CEFA0546280046F0080639D1300736
:1044D0003DD500F0FBFD0746099839460E30FEF742
:1044E00093FD099A394602F11600FEF78DFD0999F0
:1044F0002020C872DDF8249000984946FFF702F9A1
:104500000746009800224946FFF70FF90998002155
:104510001C30FEF779FD009A0121D1709FB10098FF
:1045200000223946D0F8349001A8FEF797FF050025
:1045300007D1009849467F1EFEF751FE05460098B8
:10454000476128007CD1310748BF46F040060098FB
:10455000416B6162099816F0FE01A06201A818BFC4
:104560000121FEF7B3FD002820613BD0099F009890
:104570003946FFF7C7F8A06007F11C00FEF735FDCC
:10458000E0600020E0620098206000984FF4007224
:10459000C18804F13000A180002126756175216277
:1045A000A161FEF741FDB0064AD5E768002F47D06C
:1045B000A7610098A16846897602BE420CD22046C7
:1045C000FEF77BFE0146022926D311F1010F26D00A
:1045D000BF1B2800F1D020E0F805E16130D000F0E9
:1045E000D7F908BB02252BE09DF80A0010F0110F47
:1045F00010D171077FF56BAF082521E02800A0D10D
:104600009DF80A00C10648BF042519D4B1079AD500
:10461000C00798D5072513E00225E16110E04FF0AF
:10462000FF300125E0610BE000EB57200123206201
:1046300004F130010246009800F0AFF900B1012505
:10464000404600F004FD280029461CBF00202060E1
:1046500000F006FB28460FB0BDE8F0834641540049
:104660004641543398B00320525261417272416105
:104670007CAE03202DE9FC470646994600208A4679
:10468000C9F80000154669463046FFF777FE04007A
:1046900002D1747D200005D000982146FEF7DBFC96
:1046A00020468CE0307DC10703D400F06CF9072070
:1046B00085E0F068B469041BAC423ED92C463CE06E
:1046C000F1693046FEF7F9FD02287AD310F1010FA7
:1046D0007DD0F061F16900F05BF9010071D0670AEB
:1046E00005EB00083BD00098791942464089884282
:1046F000514638BF471B009D3B46687800F0C4FC1C
:10470000002864D1307D01060CD5316AA1EB080385
:10471000BB4207D20AEB43204FF4007206F130018E
:10472000FEF77AFC7F02B069BA44E41B3818B06126
:10473000D9F800003818C9F80000002C3CD0B16945
:10474000C80528D100F019F9C4D109B9B068BBE790
:10475000F06A0028B4D03046FEF709FFB4E7326AA9
:10476000424516D0307D01060BD50098012306F195
:104770003001407800F08EFC48BB307D00F07F00B7
:10478000307500980123424606F1300100F005F92A
:10479000E8B9C6F82080B1692746C1F30801C1F520
:1047A0000070844288BF074606F1300001443A4653
:1047B0005046FEF731FCB6E700F052F90020BDE8A4
:1047C000F6870220022100F04AFA0220F7E70120D2
:1047D000012100F044FA0120F1E72DE9FC470746EA
:1047E000984600208946C8F80000144669463846B5
:1047F000FFF7C4FD050002D17D7D280003D000F045
:10480000D8FA2846A9E0387D810703D400F0BBF828
:104810000720A2E0B869211881425DD24FF0FF3134
:104820000C1A59E0F9693846FEF74DFE002854D0BD
:1048300001281CD010F1010F00F09880B968F861D0
:1048400001B9B860387D01060DD500983A6A012398
:1048500007F13001407800F01DFC00281AD1387DA6
:1048600000F07F003875F96900F092F8002876D0E2
:10487000660A05EB000A43D0009871195246408938
:104880008842494638BF461B009D3346687800F091
:1048900001FC00286AD1386AA0EB0A00B0420BD2B2
:1048A00009EB40214FF4007207F13000FEF7B4FB32
:1048B000387D00F07F0038757602F968B869B14438
:1048C00030188842B86138BF0846F860D8F8000050
:1048D000A41B3018C8F80000002C37D0B969C805EF
:1048E0001FD100F04AF8ADD119B9B86800289DD1A0
:1048F00099E7F86A002895D03846FEF738FE95E724
:10490000396A51450BD0B869F968884207D20098D6
:104910000123524607F1300100F03FF830BBC7F8E1
:1049200020A0BB6926464946C3F30803C3F50070BF
:10493000844288BF064607F1300032461844FEF72D
:104940006BFB387D40F080003875B6E7397D41F06B
:104950004001397500F084F80020BDE8F687022098
:104960000221787500F07CF90220F6E70120012190
:10497000787500F075F90120EFE7009845896D1E04
:1049800015EA5125704700980721FEF764BB0146E0
:104990000098FEF785BC04F13001407800F074BB4C
:1049A0007CB500F0C0F9050037D1207D410634D533
:1049B00000060AD500F035F828B100980121FEF76D
:1049C0004AFB012076BD00F045F900F07FFB06466A
:1049D000616A00F018FB05001FD1A56AE87A40F073
:1049E0002000E872A26820682946FEF79EFEE16872
:1049F00005F11C00FEF708FB314605F11600FEF735
:104A000003FB002105F11200FEF7FAFA00F0F4FAB8
:104A10000546207D00F0BF00207500F0CAF9284649
:104A200076BD0098226A012304F13001407800F03D
:104A300031BB38B50446FFF7B3FF05000ED1694618
:104A40002046FFF79BFC050008D12069FEF77AFBA2
:104A5000050004BF0020206000F002F8284632BDA7
:104A600000980021FEF7F7BA2DE9F84F0D4600F047
:104A70005AF95FEA000808BF94F815805FEA080059
:104A800032D1E06A002860D015F1010F2DD1074620
:104A9000A06857F8049B4FF0020AE0B18346002556
:104AA0000AF1020A0646014620466D1CFEF705FC87
:104AB000012840F29B8010F1010F6ED0761CB042AD
:104AC000F0D0D14503D33D60C7F804B00837009952
:104AD000CA699042E2D3E06AD145C0F800A032BF73
:104AE0004FF0110800203860ADE0E668AE4288BFA4
:104AF0002E46002EA661F7D0761E31462046FEF7E0
:104B000036FDE061FFF743FF05006FD00098A26912
:104B10004189491E01EA56214D19D0051CBF226A60
:104B2000954211D0207D010606D50098FFF77BFF46
:104B3000002807D100F08EF8009801232A46FFF7DD
:104B40002AFF002878D125627DE0E068A84203D2E0
:104B5000217D8A0758BF0546A0690026002DA66161
:104B60004DD000994F897F0268B1401E6A1EB0FB8C
:104B7000F7F1B2FBF7F28A4205D3791E8843A061B0
:104B80002D1AE0690CE0A06848B900212046FEF724
:104B90009AFC01282AD010F1010F4DD0A060E061ED
:104BA00060B92CE0FEF789FB10F1010F44D0012819
:104BB0001CD90099CA69904218D2E061AF420DD267
:104BC000A269217DED1BBA18A2618A070146204621
:104BD000E8D5FEF778FC0028E6D10025A169691820
:104BE000A161E9050BD0FFF7D2FE30B90220022106
:104BF000607500F035F802202AE000EB5526A06928
:104C0000E168814204D2217DE06041F040012175DC
:104C1000C0051CBF226A964215D0207D010605D52D
:104C20000098FFF700FF38B900F014F8009801234E
:104C30003246FFF7B0FE28B10121617500F010F88F
:104C4000012005E0266200984146FEF704FA40463E
:104C5000BDE8F28F207D00F07F00207570477075F1
:104C60000098FEF7F8B973B5040001D1092076BDAC
:104C70000022694601A8FFF75BFA06003AD10098C6
:104C8000206000F08AF8050003D100F08EF81120B2
:104C900076BD0098C56001992046FFF7AFF9060080
:104CA00021D194F82F00010607D4A179C80617D5A1
:104CB000216A0098FEF726FDA0600098C188204672
:104CC000A1800021FEF767FC06000CD1A06848B166
:104CD00000212046FEF7FAF9206120B9122602E0F1
:104CE000052600E02061284600F0B1F9042E08BF37
:104CF000052601D0300001D00020206000F051F8DE
:104D0000304676BD38B500F00EF8050009D12069AF
:104D100018B1FEF717FA050001D100202060FFF757
:104D20009FFE284632BD04466946FFF727BBF8B50B
:104D30000D4606466946FFF721FB070027D12DB92E
:104D400000213046FEF727FC074620E000F025F85A
:104D5000040003D100F029F81120F2BD00980021D1
:104D6000C4603046FEF744FD0428074601D03800F1
:104D70000BD129463046FEF792FF00213046FEF760
:104D80004FFC0746042808BF002700F075F800987C
:104D90003946FEF760F93846F2BD4FF4007000F076
:104DA00054B900983146FEF756B900981121FEF724
:104DB00052B900982946FEF74EB971B59BB0022250
:104DC00069461BA8FFF7B4F90600009B01934ED17A
:104DD000FFF7E3FF040003D1FFF7E7FF112049E0ED
:104DE0000098C4601B9901A8FFF708F9060004D1D8
:104DF000022101A8FEF73EF90646300035D19DF8A4
:104E00003300010648BF06262FD49DF80A60F0073C
:104E100015D409990098FEF775FC0546F00612D5E1
:104E2000009810950E9000210EA8FEF7B4FB060026
:104E30001BD100210EA8FEF7DBFC060001D10726DE
:104E400013E0042811D101A8FEF706FF060006D1E1
:104E50003DB10022294601A8FEF700FB06463000BE
:104E600003D10098FEF7D5F9064600F005F8FFF7E4
:104E700098FF30461CB070BD204600F0E8B82DE920
:104E8000F1478FB0022269460FA8FFF751F90700DA
:104E9000009B019340F0A480FFF77FFF5FEA0009C9
:104EA00003D1FFF782FF11209FE00098C0F80C901B
:104EB0000F9901A8FFF7A2F8070008BF082700F024
:104EC0008C80042840F08980002101A8FEF7FBFABD
:104ED000064600984189490204910EB907270CE063
:104EE000012E08BF022708D016F1010F08BF0127C5
:104EF00003D00098FEF74DF9074600F0E7F880462A
:104F000038004CD100983146FEF7CAF905460098A2
:104F100000F06EF800F1380A5046FEF785F80B22D3
:104F200020215046FEF780F82E2041468AF80000E6
:104F300010208AF80B000AF11600FEF765F80098B9
:104F400032465146FEF7F1FB202251460AF120007D
:104F5000FEF762F82E208AF821000098039A017863
:104F600003290AF1200102BFC06A82420022009890
:104F7000FEF7DBFB0098448905E000F039F8504665
:104F8000641EFEF751F864B1012100984563009A50
:104F90006D1CD1700098FEF7FCF80700EDD03800CA
:104FA00003D101A8FEF75CFD0746380010D1099C2B
:104FB000414604F11600FEF727F8009832462146D4
:104FC000FEF7B3FB1020E07200F016F8074604E08D
:104FD0000022314601A8FEF741FA484600F037F8B2
:104FE00000983946FEF737F8384610B0BDE8F0872C
:104FF0004FF400720021704700990120C87000989A
:10500000FEF707B9E9690098FEF7E9B81CB50FF299
:1050100044020C46136801210093684600F02CFB03
:10502000206000B1012016BD80B500F08DFB01208D
:1050300002BD10B54FF47A71002400F033FB00B9C3
:105040000124204610BD00F061BB00F021BC00F03F
:10505000A7BC00000000000001461B4A501802EBEC
:105060008101007A4A6853681847174B0246995CD9
:10507000002041B901209854981803EB8202007A6D
:1050800051680B681847704770B500F009F8AE68B2
:10509000B04770BD70B500F003F8EE68B04770BD62
:1050A0000446094D281905EB8404007A65687047A9
:1050B00038B50346044CE01804EB8303007A5C68BF
:1050C0002569A84732BD000048B003200020704782
:1050D000802800DA704718B50FF2AC0351B1B0F573
:1050E000807F01DB002012BD03EB4000A0F5807142
:1050F000088812BD8CB233F81440A04203D0491C7A
:105100008AB2802AF6DB01F1800000F0FF0012BDB8
:10511000B0F5805F70B5ACBF0FF260340FF2681469
:1051200002E00AB904EB4504218851B3884228DB28
:105130006588241D2A0205F0FF05120C6E18B04286
:10514000EFDA082A1DD8DFE802F005090E10121464
:1051500016181A00431A34F8130012E0411A01F02D
:105160000101401A0DE010380BE0203809E030381A
:1051700007E01A3805E0083003E0503801E0A0F5F8
:10518000E35080B270BD0000C700FC00E900E200FF
:10519000E400E000E500E700EA00EB00E800EF00D3
:1051A000EE00EC00C400C500C900E600C600F40033
:1051B000F600F200FB00F900FF00D600DC00F8006A
:1051C000A300D800D7009201E100ED00F300FA003F
:1051D000F100D100AA00BA00BF00AE00AC00BD00D3
:1051E000BC00A100AB00BB009125922593250225B0
:1051F0002425C100C200C000A90063255125572500
:105200005D25A200A5001025142534252C251C257C
:1052100000253C25E300C3005A2554256925662551
:10522000602550256C25A400F000D000CA00CB00FA
:10523000C8003101CD00CE00CF0018250C258825EF
:105240008425A600CC008025D300DF00D400D20046
:10525000F500D500B500FE00DE00DA00DB00D90065
:10526000FD00DD00AF00B400AD00B1001720BE00AE
:10527000B600A700F700B800B000A800B700B9005A
:10528000B300B200A025A00061001A03E0001703DC
:10529000F8000703FF00010078010001300132012E
:1052A0000601390110014A012E0179010601800130
:1052B0004D00430281018201820184018401860143
:1052C0008701870189018A018B018B018D018E0184
:1052D0008F0190019101910193019401F6019601D2
:1052E0009701980198013D029B019C019D012002BC
:1052F0009F01A001A001A201A201A401A401A60195
:10530000A701A701A901AA01AB01AC01AC01AE0143
:10531000AF01AF01B101B201B301B301B501B501F4
:10532000B701B801B801BA01BB01BC01BC01BE01A3
:10533000F701C001C101C201C301C401C501C4011B
:10534000C701C801C701CA01CB01CA01CD011001C3
:10535000DD0101008E01DE011201F3010300F10104
:10536000F401F401F8012801220212013A020900B5
:10537000652C3B023B023D02662C3F02400241028B
:10538000410246020A015302400081018601550292
:1053900089018A0158028F015A0290015C025D0264
:1053A0005E025F029301610262029401640265027F
:1053B00066026702970196016A02622C6C026D0216
:1053C0006E029C01700271029D01730274029F01C2
:1053D00076027702780279027A027B027C02642CE0
:1053E0007E027F02A60181028202A9018402850257
:1053F00086028702AE014402B101B20145028D026C
:105400008E028F0290029102B7017B030300FD031D
:10541000FE03FF03AC0304008603880389038A03A9
:10542000B1031103C2030200A303A303C4030803CF
:10543000CC0303008C038E038F03D8031801F203FF
:105440000A00F903F303F403F503F603F703F70384
:10545000F903FA03FA033004200350041007600430
:1054600022018A043601C1040E01CF040100C004E8
:10547000D004440161052604000000007D1D0100E8
:10548000632C001E9601A01E5A01001F0806101F63
:105490000606201F0806301F0806401F0606511F7B
:1054A0000700591F521F5B1F541F5D1F561F5F1FB0
:1054B000601F0806701F0E00BA1FBB1FC81FC91F40
:1054C000CA1FCB1FDA1FDB1FF81FF91FEA1FEB1FD4
:1054D000FA1FFB1F801F0806901F0806A01F080662
:1054E000B01F0400B81FB91FB21FBC1FCC1F0100A2
:1054F000C31FD01F0206E01F0206E51F0100EC1FBC
:10550000F21F0100FC1F4E21010032217021100208
:10551000842101008321D0241A05302C2F04602C13
:105520000201672C0601752C0201802C6401002DFC
:10553000260841FF1A03000001460020842918BFF5
:10554000C81C704780B500F058FC002002BDEFF386
:105550000580002818BF00F0D2BC00F0CCBC3EB5DE
:1055600004460D46B4F90800FFF7E6FF02A90090D3
:1055700001912269216860682B4692B200F064FABA
:10558000012801D000203EBD02983EBD00F055BE6E
:1055900080B500F01DFB002002BD80B500B90120E0
:1055A00000F052FB002002BD0129134680B50068BF
:1055B0000CBF012200220090012150A000F072FFD8
:1055C00002BD1CB500240A46019402B90122EFF382
:1055D000058159B1009401AB092100F097FF012822
:1055E0000BD1019850B100F07EF807E000230421B0
:1055F000009300F08BFF012800D0FF24204616BD49
:10560000012001F054B980B50022009208B9802031
:1056100002BD11F1010F08BF4FF0FF3200F070F82A
:1056200059B16A46002101F057FB01280AD10098C0
:1056300008B100F058F8002002BD002301F098FAEC
:105640000128F8D0FF2002BD1CB500F077F849B161
:10565000694601F049FA01280CD1009840B100F0E8
:1056600042F805E0002301F05AF9012818BFFF2491
:10567000204616BDFF2016BD012910B50DD103220D
:105680000021012001F0E8F8040004D000230022EA
:10569000002101F044F9204610BD0846BDE8104045
:1056A00001F021B980B50022009208B9802002BD26
:1056B00011F1010F08BF4FF0FF3200F021F859B18E
:1056C0006A46002101F008FB01280AD1009808B1C0
:1056D00000F009F8002002BD002301F049FA01287A
:1056E000F8D0FF2002BD4FF08051DFF89421116007
:1056F000BFF34F8FBFF36F8F7047000000000000B3
:1057000001D001B10A46EFF3058170471CB500F0E6
:1057100015F849B1694601F0E7F901280CD1009864
:1057200040B1FFF7E0FF05E0002301F0F8F80128A1
:1057300018BFFF24204616BDFF2016BD00220024FE
:105740000092EFF30581704780B5EFF3058109B151
:10575000822002BD01F004FB002002BD4168006808
:10576000002201F079B803B581B00021009102B99F
:105770000122EFF3058149B100F045F801280BD172
:10578000009808B1FFF7AFFF00200EBD002302A96B
:1057900001F0C5F80128F7D0FF200EBD38B5054649
:1057A00084B0084600210290019110B900F03BF846
:1057B00027E0002412F1010F039108BF4FF0FF34DE
:1057C00000F02BF851B103AA01A901F085FA0128D4
:1057D00007BF102000900022009206E000F018F8A9
:1057E000012807D11021009109E0039838B1FFF793
:1057F0007AFF04E0002C0CBF00204020009000F055
:1058000041F805B030BD00236A4602A901F01EB977
:105810000023224601A901F0ABB901D002B1144620
:10582000EFF30581704780206946009091E81C00E5
:1058300085E81C00704780B500F003FD012803D007
:10584000BDE8014001F0FCBB01BD80B500F010FADD
:10585000002002BD80B5EFF3058169B100F0A1FA27
:10586000012807D14FF0805005490860BFF34F8FE2
:10587000BFF36F8F002002BD00F05EFAFAE7000070
:1058800004ED00E0684690E80E0085E80E007047E1
:105890002DE9F84304466A4F00F0DFFAB8684FF08C
:1058A00000090025F0B967494FF40C4011F0070FCB
:1058B0000B4605D0CB1DDB08DB00C3F50C400818F8
:1058C000C0180838C008C0003B60C11A7D60B860CD
:1058D000456005605960186058683861F8604FF09D
:1058E0000040786178694FF05008044233D194B396
:1058F000083414F0070F1FBF04F1080004F0070478
:10590000041B14F0070F02D000F041F8FEE714B3B7
:10591000F868A0421FD339463E687068A04223D27F
:10592000306800281CBF31460646F6D11CE0301D09
:1059300002510846746000F05FF83A697168F868CF
:10594000401A9042F86038BF38617869014371604D
:10595000356009F0070500F086FA15B100F017F878
:10596000FEE74846BDE8F283B8688642F3D0326865
:1059700008680A607268121B112A00F10809DCD35A
:10598000311911F00700D2D000F001F8FEE772B62D
:1059900088F31188BFF34F8FBFF36F8F62B67047E4
:1059A000002800D1704738B5A0F10804244D616883
:1059B0006A695023114202D100F015F8FEE7206811
:1059C00010B100F010F8FEE79143616000F045FA75
:1059D000E968606841182046E96000F00DF8BDE80C
:1059E000314000F040BA72B683F31188BFF34F8F95
:1059F000BFF36F8F62B67047114930B50A4600E0B9
:105A0000224614688442FBD35368D418844203D1DD
:105A10004068C3181046536043681468C518A5420F
:105A200008D189688C4204D06168CB18436024682F
:105A300000E00C468242046018BF106030BD0000D8
:105A400064AF0320680D02202DE9F843064617468F
:105A500084B088469946B800FFF71AFF05001AD0AF
:105A60005C20FFF715FF040012D00D990C982563F8
:105A7000002203924B4601913A460090414602941F
:105A8000304600F00DF8204600F050F8012004E008
:105A90002846FFF785FF4FF0FF3005B0BDE8F083E3
:105AA0002DE9F0470A9D81460C4617469846A522E7
:105AB000286BB90001F020FB286B00EB87010F1F5A
:105AC000FF08FF000021625C681880F83420605CE9
:105AD00010B1491C1029F6D3089E002085F8430018
:105AE000099C05F14C0A0B2E88BF0B26EE62CAF802
:105AF0000400281DCAF80060C6F10C0601F026FB60
:105B000005F1180001F022FB2D610020AE61424634
:105B10006D624946CAF808008AF80C00384601F060
:105B2000FBF9286004B12560BDE8F0872DE9F0415C
:105B300000F085F8E86C1426DFF83C88401CE86427
:105B4000A86A28BBAC62E96C012929D1002706FBB1
:105B500007F07F1C404401F0ECFA0C2FF7D305F15D
:105B6000740005F1880701F0E4FA384601F0E1FA23
:105B7000284601F0DEFA05F1140001F0DAFA05F129
:105B8000380001F0D6FA05F17400E8622F6307E0EF
:105B9000A86D28B9E16AAA6AD06A814228BFAC62BE
:105BA000A86E0122401CA8666064E06A696D8240AC
:105BB000464311436965211D08EB060001F0C9FA4F
:105BC00001F02BFAA86D08B100F0E3FBBDE8F0810D
:105BD00070B500F034F804B9AC6A00F08AFA00F04D
:105BE00086F808B100F079F8A96E491CA966A86A80
:105BF000844208D1211D05F1140001F0AAFA686B56
:105C0000401C686307E0E96C2046491EE96400F027
:105C1000FCFA00F004FB01F000FAA86D70B1A96A6B
:105C20008C420BD1296F11B100F0D1FBFEE74FF090
:105C30008050DFF85027106000F054F870BD044623
:105C4000DFF8445701F0CCB980B570B1DFF86027B8
:105C5000116F11B100F0BBFBFEE7136F5B1C136704
:105C600000F0CBFB00F0FFF808B900F084F801BDAC
:105C700070B5FFF7E4FF04B9AC6A00F03AFA00F03F
:105C800036F808B100F029F8211D05F1380001F0BF
:105C900060FA01F0C2F9A86D28B101F0A1F900F095
:105CA000BEFA01F0BAF9A86A844215D1A96D49B1CA
:105CB000286F00F08AF94FF08051DFF8C82600F015
:105CC00010F870BDA86BEA6C904202D10020A86267
:105CD00070BDBDE8704084E170BD04F1180001F0B2
:105CE0005DBA1160BFF34F8FBFF36F8F704768B914
:105CF000E16A1422DFF880064A43805830B96B6DA0
:105D0000012606FA01F123EA01016965A06A7047DC
:105D10000146002010B511B900F059FBFEE74B69B0
:105D2000DFF88C2602F13804A34204D1896A91423B
:105D300001D001B9012010BD38B5040000F025F8EC
:105D4000DFF86C56A86A844214D001F049F9204665
:105D5000FFF7DEFF50B100F0CCF900F0CDF9E16AB9
:105D6000AA6AD06A814201D300F005F8BDE831404B
:105D700001F053B931BD4FF08050DFF8E4160860F0
:105D8000BFF34F8FBFF36F8F704709D172B65020AA
:105D900080F31188BFF34F8FBFF36F8F62B6FEE7BA
:105DA0007047F8B504460025502724B900F00BFBD6
:105DB00000F011FBFEE701F059F900F002FB00F0E2
:105DC0000AFB2046FFF7A4FF98B1DFF89876386FFA
:105DD00050B9E16ABA6AD06A814228BF012500F051
:105DE00088F900F0FEFA02E004F11801384601F0EB
:105DF000B0F986F311882846F2BD7CB5DFF8644619
:105E0000002604F19C0500960195002380220FF2E4
:105E10005C610FF29130FFF717FE012808BF00F018
:105E200029FB502101280FD172B681F3118800F0AF
:105E3000D2FA4FF0FF30E0660120A0652665BDE88C
:105E4000734001F094B873BD10F1010FFBD172B62D
:105E500081F3118800F0BFFAFEE7DFF80806016F52
:105E6000491C0167704770B5DFF844650024306F46
:105E7000002500F0DFF801F0B3F8326F521E3267F0
:105E8000316F002936D1F06CD8B933E0F168CC68B5
:105E9000FFF723FF00F02DF9E06A716D0122142352
:105EA000824058431143DFF8C0257165211D10441D
:105EB00001F04FF9E06AB16ACA6A904224BF01203A
:105EC000306630680028E1D10CB100F0A8F9F46D1B
:105ED0003CB100F01BF808B101203066641EF8D117
:105EE000F565306E30B14FF08051DFF87425012533
:105EF000FFF7F7FE42E2DFF86C05006D704780B5F2
:105F000001F0B4F8DFF85C05006D02BD2DE9F8433F
:105F1000DFF89C740026386F00284DD13C6D641C5E
:105F20003C650CD1F96A086800F04FF8F86A396BE3
:105F3000F9623863786E401C786600F070F9F86E8C
:105F40004FF01408DFF82095844225D31AE0281D6D
:105F500001F024F9A86A18B105F1180001F01EF942
:105F6000E86A796D0122824008FB00F011437965EF
:105F7000291D484401F0EDF8E86AB96ACA6A9042FE
:105F800028BF0126FA6A106890B1F96ACA68D56814
:105F900068688442DBD2F866B86AC16A08FB01F01F
:105FA00059F80010F86D022928BF012648B906E00B
:105FB0004FF0FF31F966EFE7F96D491CF96501F023
:105FC00045F9386E00B10126E0E148B172B65022C1
:105FD00082F31188BFF34F8FBFF36F8F62B6FEE776
:105FE00070471CB5DFF8A043206F10B10121216676
:105FF00013BD0021216601F051F9606DDFF86824BE
:10600000B0FA80F1C1F11F0114204143505800F053
:1060100011F8501800F10802416849684160914246
:1060200004BF496841604068C168A162BDE813408F
:1060300001F029B948B972B6502181F31188BFF334
:106040004F8FBFF36F8F62B6FEE7704710B50C46F7
:1060500000F017F801F089F820460121BDE8104052
:1060600000F0CBB938B50D46144600F00AF801F03F
:1060700070F80CB14FF0FF3521462846BDE834409A
:10608000BBE148B972B6502080F31188BFF34F8F3F
:10609000BFF36F8F62B6FEE7DFF8C823936A03F1A0
:1060A0001801704738B5C168CC6814B900F08FF991
:1060B000FEE704F11800DFF8D05201F06FF8296F05
:1060C00051B900F016F8E26A696D0120DFF89833E3
:1060D000904000F06FF902E004F11801284601F049
:1060E00038F8A96AE26AC86A904200D212E0002039
:1060F00032BD201D01F052B8E26A696D0120DFF85F
:10610000683390400143142042436965211D98186B
:1061100001F01FB80120286632BD48B972B6502080
:1061200080F31188BFF34F8FBFF36F8F62B6FEE726
:10613000DFF830134A6E0260096D4160704770B538
:1061400004460D4650201CB972B600F042F9FEE735
:106150001DB972B600F03DF9FEE700F041FFDFF82F
:106160000403016D2A6812F1010F0FD06368406EBD
:106170002668B04201D099420AD2C81A904207D28A
:10618000511A591829602046FFF7C7FF002400E084
:10619000012400F042FF204670BD0120DFF8C41248
:1061A000086670472DE9F041DFF8D8514FF080566E
:1061B000DFF8C481DFF8F8711AE0386F401C3867E7
:1061C00079694C1EA441E40FFFF74DFE84B900F03D
:1061D00007FF386AC468FFF78CFFF86C401EF8644C
:1061E000796B491E796300F018FF204600F00DF826
:1061F000786B0028E1D1D8F80010012902D92E606F
:10620000FFF770FD01F01AF8F2E710B50446206BB5
:10621000FFF7C6FB2046BDE81040FFF7C1BB64494D
:10622000CA6A106818B94FF0FF33CB667047CA6A64
:10623000D068C3685A68CA667047DFF82802806A67
:106240007047DFF82002816D09B901207047006FA7
:1062500008B902207047002070472DE9F041040082
:106260002FD0494DE06AA96ACA6A904229D2A06932
:10627000002804D4A96AC86AC0F10C00A061E16AD0
:1062800014276069DFF8E08179434144884215D1E1
:10629000201D012600F082FF002801BFE16A79433A
:1062A00058F80110002900F055F8A86AC06AE062A9
:1062B00000F047F8BDE8F04100F04BBFA86AC16AA2
:1062C000E162BDE8F0812DE9F04104460021002C97
:1062D00034D02D4D5022A86A844205D072B682F384
:1062E000118800F078F8FEE7206D28B972B682F3C5
:1062F000118800F070F8FEE7E26A401EE36C20654A
:106300009A421BD0D0B9201D01261427DFF85881EE
:1063100000F044FF002801BFE16A794358F80110FA
:10632000002900F017F8E06CE062C0F10C00A061F9
:10633000E06A00F006F800F00CFF01210846BDE815
:10634000F081696D474386400E43211D6E6508EB61
:106350000700704705D1686DE26A06FA02F29043C1
:1063600068657047DFF8FC10886A18B1886A026DAA
:10637000521C0265886A704764A3032000F04DFE3A
:10638000284670BD04ED00E060A603203046BDE85D
:10639000F283A96AE06ACA6A824207D24FF080504B
:1063A0002F490860BFF34F8FBFF36F8F7047000016
:1063B00060A603200143142042436965211D9818FB
:1063C0007047EFF3118672B687F31188704772B683
:1063D000502080F31188BFF34F8FBFF36F8F62B6E9
:1063E0007047E26A796D01201F4B904001431420F1
:1063F00042437965211D98187047F8B5194D0C4630
:106400002F6DA96A0646081D00F0C8FE30B9A86ABB
:10641000696D0122C06A82409143696516F1010FDE
:1064200008D13CB1A86A011D05F13800BDE8F4406F
:1064300000F08FBEA96AF619BE424E60A86A05D266
:10644000011D286BBDE8F44000F08FBE011DE86A15
:1064500000F08BFEE86E864238BFEE66F1BD0000AC
:1064600004ED00E060A6032064A3032049444C45EA
:1064700000000000E0B500F084F9DFF84C138868F4
:1064800060B10C31042201910023009280220FF2AE
:1064900040310FF2C100FFF7D7FA10B900F067F9E9
:1064A000FEE70EBD2DE9FC4105460E46174698460F
:1064B0002C20FFF7EDF9040008D008980194009013
:1064C00043463A463146284600F003F82046BDE8E8
:1064D000F6812DE9F8430D0006469146984602D113
:1064E00000F045F9FEE7099C74B1089F00F049F9F6
:1064F0002660201DA561C4F81C90C4F82080676246
:10650000BDE8F24300F022BEBDE8F183FEB50446CB
:106510001E46002014B900F02AF9FEE7AA4FBD6814
:10652000BDB106290091019202940CDAFFF789FEB1
:106530000228B868694607BF089A00230023002292
:1065400000F0EDF9FEBD002332466946284600F012
:106550007DFAFEBD80B59C490A68106800281DBF01
:106560000021D2681068012100F003F800F0A2F8C1
:10657000F1E7FEB506460C46FFF76FFC01A800F0F8
:1065800044F80546019800283CD18F4F24BBB54202
:1065900027D3FFF768FC3968C868C468201D00F07D
:1065A000FDFDE069012813D1A16933462A46204642
:1065B000891900F065F858B1002000230090324698
:1065C00000212046FFF7A2FF10B900F0C6F8FEE751
:1065D000616A20468847F7BD786801684C1EA4416F
:1065E000E40FB8682246711B00F072FCFFF73BFC19
:1065F00050B94FF0805075490860BFF34F8FBFF31B
:106600006F8FF7BDFFF72FFCF7BD2DE9FC41044666
:106610006D4EFFF770FC0546306985420BD30020B4
:10662000206028463561BDE8F6817860391D3F61FC
:10663000306800F09AFD31680868E0B1C868C76842
:10664000D0F80080381D00F0A9FD796A38468847E7
:10665000F8690128EFD1B86940448045E5D30021AD
:106660000023009142463846FFF750FF0028E2D150
:1066700000F07DF8FEE77068716030600120CFE7C0
:1066800038B500248A4241604F4D006106D38169CC
:10669000D21A8A4206D2011D686807E09A4203D2E4
:1066A000994201D3012403E0011D286800F05DFD3B
:1066B000204632BD30B585B0434C04E013468918FE
:1066C0002846FFF7DDFFA0680023002202A900F0A2
:1066D0004FFA00283FD002980028F4D4049D68693E
:1066E00010B1281D00F05AFD01A8FFF78EFF0246E9
:1066F00002980928E7D8DFE800F006060605232AF5
:1067000006060523DFE70399A8690B4641182846CA
:10671000FFF7B6FF0028D6D0696A28468847E8699F
:106720000128D0D10021039A0091A8690023821882
:106730002846FFF7EBFE0028C5D100F00EF8FEE773
:106740000399A9610029B9D100F011F8FEE72846A4
:10675000FFF726F9B7E705B030BD72B6502181F3D7
:106760001188BFF34F8FBFF36F8F62B6704772B659
:10677000502080F31188BFF34F8FBFF36F8F62B645
:10678000704710B500F02CFC0F4CA068C0B904F1A4
:10679000140000F0CEFC04F1280000F0CAFC04F163
:1067A00014000022206004F1280060600C210A20FF
:1067B00000F052F8A06018B10FF21C0100F062FB6B
:1067C000BDE8104000F029BC1CAD032004ED00E042
:1067D000546D722053766300546D725100000000B6
:1067E00038B504000D4602D100F073F8FEE700F062
:1067F000F7FBE26B206C2168424388186060002040
:10680000A0632068E26BA060206C2168521E4243A6
:1068100088184FF0FF31E06004F1440001704170CE
:1068200075B92069A0B104F11000FFF73BFC78B105
:106830004FF08051DFF89006016000F03FFA07E06A
:1068400004F1100000F075FC04F1240000F071FC6C
:1068500000F0E3FB012032BDF8B506000D461746F7
:1068600002D100F036F8FEE7002D0EBF502005FBE8
:1068700006F05030FFF70CF8040007D000943B46B8
:1068800004F150022946304600F002F82046F2BDDD
:1068900038B51C46049D01B92A462A60E86328469B
:1068A00029640121FFF79CFF85F84C4031BD024669
:1068B000002110B50120FFF7CFFF040007D0002210
:1068C0000021626000232160E16000F028F820468A
:1068D00010BD72B6502080F31188BFF34F8FBFF305
:1068E0006F8F62B6704710B50C46502110B900F09A
:1068F0000DF8FEE7A04202D200F008F8FEE70222FF
:106900000021FFF7A9FF00B1846310BD72B681F3C7
:106910001188BFF34F8FBFF36F8F62B670472DE9B9
:10692000F64782B004461E46502714B900F0D3F84B
:10693000FEE75FEA010A01D1206C70B9022E02D194
:10694000E16B01290CD1FFF77CFC002861D1039891
:1069500000285ED000F0BFF8FEE700F0BCF8FEE7CC
:1069600000F0B9F8FEE7039907F11000FFF76EFB9E
:10697000384600F04AFAFFF776FA08B900F09CF9B9
:1069800000F02EFBB86BF96B884249D3022E47D03A
:10699000039800283AD01CB968460124FFF7BDFBD4
:1069A00000F03BFBFFF759FA00F01AFB07F1440037
:1069B00090F9001011F1010F04BF0022027090F94C
:1069C000012012F1010F04BF0021417000F025FBEE
:1069D00003A96846FFF7B3FB88BB00F001FBB86B67
:1069E000F96B884214BF0025012500F016FB002D2D
:1069F000B9D1384600F009FAFFF735FAC0E708B117
:106A000000F05AF900F009FB01201EE000F005FB40
:106A10001AE027460024DFF8B0844FF08059AFE732
:106A200032465146384600F0A8F9796A0029E6D086
:106A300007F12400FFF736FB0028E1D1E2E73846F2
:106A400000F0E3F9FFF70FFA002032E12DE9F843F7
:106A50000446884615461E46502714B900F03BF8F8
:106A6000FEE7B8F1000F01D1206C20BB022E02D14D
:106A7000E16B012922D100F0F9FAEFF3118900F05E
:106A80006BF801D3022E21D194F94570324641466C
:106A9000204600F072F917F1010F12D1606A98B127
:106AA00004F12400FFF7FEFA002818BF002D0BD0D8
:106AB0000120286008E000F00EF8FEE700F00BF877
:106AC000FEE77F1C84F84570012000E0002089F378
:106AD0001188BDE8F28372B687F31188BFF34F8F38
:106AE000BFF36F8F62B67047F8B504460D46502766
:106AF00014B9FFF7F0FFFEE7226C12B1FFF7EBFFCE
:106B0000FEE7216809B96068D0B900F0AFFAEFF389
:106B1000118600F021F81BD294F94510401CA063A7
:106B200011F1010F0FD1606A80B104F12400FFF769
:106B3000B9FA002818BF002D08D00120286005E010
:106B4000FFF7C9FFFEE7491C84F84510012000E06B
:106B5000002086F31188F2BD72B687F31188BFF367
:106B60004F8FBFF36F8F62B6A06BE16B88427047A7
:106B70002DE9F64782B0064699460024502516B9FD
:106B800000F0A1F8FEE75FEA010801D1316C39B9E4
:106B9000FFF757FB60B9039850B100F094F8FEE797
:106BA00000F091F8FEE7304600F02FF9FFF75BF9AF
:106BB00000F016FAB06BDFF810534FF0805720B991
:106BC000039858BB00F029FA72E00446D6F80CA0EE
:106BD0004146304600F005F9B9F1000F0ED1641EB0
:106BE000B463316811B9FFF7BDFB7060306988B1DB
:106BF00006F11000FFF756FA48B90BE0706AC6F8C4
:106C00000CA038B106F12400FFF74CFA10B12F6048
:106C100000F054F800F001FA01204AE01CB968467F
:106C20000124FFF77AFA00F0F8F9FFF716F900F0FF
:106C3000D7F906F1440090F9001011F1010F04BFDB
:106C40000022027090F9012012F1010F04BF00210F
:106C5000417000F0E2F903A96846FFF770FA0028D6
:106C600030461CD100F003F900289CD0306830B9C0
:106C700000F0B6F97068FFF7F0FA00F0CEF903996A
:106C800006F12400FFF7E2F9304600F0BEF8FFF706
:106C9000EAF800288CD12F6000F010F888E700F0A7
:106CA000B4F8FFF7E0F8304600F0E1F80028F5D03E
:106CB000002004B0BDE8F087C8F80090BFF34F8F04
:106CC000BFF36F8F704772B685F31188BFF34F8F94
:106CD000BFF36F8F62B670472DE9F84304460F4645
:106CE0001546502614B900F032F8FEE70FB9206CB3
:106CF00060B900F0BBF9EFF3118800F028F8A66B3B
:106D00003EB9002088F31188BDE8F28300F01FF837
:106D1000FEE794F9449039462046761E00F061F86B
:106D2000A66319F1010F0CD1206970B104F11000B4
:106D3000FFF7B8F9002818BF002D06D00120286001
:106D400003E009F1010084F844000120DAE772B69B
:106D500086F31188BFF34F8FBFF36F8F62B6704712
:106D600010B5040002D1FFF7B4FDFEE700F09AF879
:106D70002046BDE81040FEF713BEF8B5064615469E
:106D8000B46B326C002742B9316831BB7068FFF7D1
:106D90009AFA0022074672601FE065B9B06800F0F9
:106DA0008FFAB068316C08447168B060884214D3BF
:106DB0003068B06011E0F06800F082FA306CF16881
:106DC00040420144F1603268914202D27168084445
:106DD000F060022D01D104B1641E641C3846B46316
:106DE000F2BD026C0B46002A00D1704710B5446812
:106DF000C1681144C160A14224BF0168C160C1687B
:106E00001846BDE8104000F05BBAF8B5054605F13C
:106E1000440400F0E5F894F9016070B2012815DB34
:106E2000686A98B105F12400FFF73CF908B1FFF753
:106E3000B4F9761EF1E72869A0B105F11000FFF75B
:106E400031F908B1FFF7A9F97F1E08E04FF0FF36CE
:106E5000667000F0E2F800F0C3F894F9007078B2C0
:106E60000128E8DA2670BDE8F14000F0D6B810B588
:106E7000044600F0B5F8A06B441EA44100F0CDF824
:106E8000E00F10BD10B50023104C54F833201AB198
:106E90005B1C082BF9D310BD44F8331004EBC3017D
:106EA000486010BD10B50021084A02EBC1035C68C0
:106EB000844203D0491C0829F7D310BD002042F8B2
:106EC0003100586010BD000004ED00E09CAC0320D0
:106ED000F8B504460D46164604F1380700F080F870
:106EE00097F90C0010F1010F04BF0021397397F9D5
:106EF0000D1011F1010F04BF0020787300F08DF820
:106F0000386828B93246294604F12400FFF7AAF868
:106F10002046BDE8F24078E74908490010B5A0F1E5
:106F200020034FF0807499610FF2150159616FF0E1
:106F30000201DC611A6040F8241D203810BD0000F9
:106F40005D4950204A6812F1010F72B607D080F3F4
:106F50001188BFF34F8FBFF36F8F62B6FEE780F3E8
:106F60001188BFF34F8FBFF36F8F62B6FEE71CB57A
:106F70005248FF220178504C0191027002788DF83E
:106F800000209DF8001001F050012170072105E05C
:106F90009DF80020491E52008DF800209DF8003019
:106FA0001A06F5D4090201F4E061A16001990170AB
:106FB0004348016841F470010160026842F0704288
:106FC000026000F087F80020606000F019FA3D4888
:106FD000016841F04041016000F006FA002016BD52
:106FE00072B6502080F31188BFF34F8FBFF36F8FBD
:106FF00062B631494A68521C012A4A600CD13249B2
:107000000A68130608D072B680F31188BFF34F8F59
:10701000BFF36F8F62B6FEE770472749486848B9EB
:1070200072B6502080F31188BFF34F8FBFF36F8F7C
:1070300062B6FEE7401E486008BF80F311887047C3
:1070400080B572B6502080F31188BFF34F8FBFF325
:107050006F8F62B6FEF75AFF18B14FF080501A4991
:107060000860002181F3118801BD0000EFF3058065
:1070700050211028104A0DD3144B185C13789842F5
:1070800008D272B681F31188BFF34F8FBFF36F8FB1
:1070900062B6FEE790680E4A136803F4E063984214
:1070A00008D272B681F31188BFF34F8FBFF36F8F91
:1070B00062B6FEE7704700006800002000E400E0D0
:1070C00020ED00E034EF00E004ED00E0F0E300E04C
:1070D0000CED00E010B506494FF47A730A680548D4
:1070E0000724B2FBF3F35B1E4360046010BD00BFD6
:1070F0000001002010E000E062F30F2262F31F4263
:1071000000B500BF130096469446103928BFA0E88A
:107110000C50FAD85FEA417C28BF0CC048BF40F849
:10712000042BC90728BF20F8022B48BF00F8012B09
:1071300000BD00F1080141604FF0FF31816000F1B6
:107140000801C160016100210160704700210161F7
:10715000704742684A6093688B6093685960916099
:1071600008610168491C0160704730B50A6812F176
:10717000010F08BF036907D000F1080300E02346B0
:107180005C682568AA42FAD25A684A6091608B60AE
:10719000596008610168491C016030BD10B5436841
:1071A000016982689A608468426862604A688242C3
:1071B00004BF82684A60002202610868401E0860BD
:1071C00010BDF0B40246106895681318506803EBC0
:1071D0005004C00721D54D441FE0F0BC02F10C0063
:1071E000704713F8017B05F8017B491EF9D1A0B166
:1071F000B60813F8011B06F00306032E08BF13F8A8
:10720000016B01EB06214942801C294405D011F88D
:10721000016B05F8016B401EF9D1A342DDD013F8D4
:10722000016B16F0030104BF13F8011BC91C3009E0
:107230000F28DAD113F8010B0F30D6E710B51F4C29
:10724000206810B9FEF7F9FF206010BD10B51B498A
:1072500040F2E9334869421C984212DB0869002277
:107260004FF47A74B0F57A7F84BF4FF47A730B6170
:107270000B6964204343B3FBF4F4C4F164044C6031
:107280000A614A6110BD10B5FEF7D7FF0B4C2168AB
:10729000884202D1FEF733FEA06010BD10B5FEF7A4
:1072A000CCFF064C2168884207D1FEF728FEA16872
:1072B000401A2169E0604018206110BD4CAF0320E6
:1072C00062B38B0708D0521E11F8013B00F8013B56
:1072D00000F024808B07F6D1830740F0208000BFA8
:1072E000103A07D330B4B1E83810103AA0E838109B
:1072F000F9D230BC530724BFB1E80810A0E8081049
:1073000044BF51F8043B40F8043BD20724BF31F896
:10731000022B20F8022B44BF0B7803707047121F1A
:1073200017D35B0009D151F8043B20F8023B1B0C3A
:10733000121F20F8023BF6D20BE051F8043B00F894
:10734000013B1B0A20F8023B1B0C121F00F8013BFB
:10735000F3D238BF121D521E24BF11F8013B00F8B2
:10736000013BF8D870470268531C036011707047E6
:10737000EFF30980BFF36F8F254B1A681EF0100FD3
:1073800008BF20ED108A20E9F04F106008B44FF0DC
:10739000500072B680F31188BFF34F8FBFF36F8F29
:1073A00062B6FEF71EFE4FF0000080F3118808BCA5
:1073B00019680868B0E8F04F1EF0100F08BFB0EC75
:1073C000108A80F30988BFF36F8F7047104B1968DC
:1073D0000868B0E8F04F80F30988BFF36F8F4FF073
:1073E000000080F3118870470A480068006880F345
:1073F000088862B661B6BFF34F8FBFF36F8F00DFAF
:10740000DFF81400016841F470010160704700006A
:1074100088A6032008ED00E088ED00E081B000F5CB
:10742000E0700268914203D343681A44914202D348
:1074300080680028F5D101B07047DFF86817086848
:1074400090B94FF4805048604FF480324FF0FF30D5
:107450008A60C86008610420DFF84C27DFF84C37E9
:107460004861C2F8BC010B600120704701F10803BC
:1074700013F0070F0EBF0023C3F1080303F0070347
:107480001944D21A8161C26042F001034B60091DA8
:1074900028238B50DFF80C170A69C26170472DE969
:1074A000FC4B074601F1080010F0070F0FBF89469B
:1074B000C0F1080000F0070001EB000902F108012B
:1074C00011F0070F06D002F10800C0F1080000F02B
:1074D000070002441546A5EB090009EB0306A0EBE3
:1074E000030B43F00303C9F80430AE4228BF01F098
:1074F000FFF92879C10758BF01F0FAF9BBF1100F65
:1075000038BF01F0F5F9B869854207D1F8685844E9
:10751000F860BE6140F00100706050E1786985421A
:107520000AD1B8688344C7F808B07E614BF0010007
:10753000706046F80BB042E1686800F00301012971
:1075400040F0AB80C008C0000190C0081F2839D8A7
:10755000AC68D5F80C800090454508BF01F0C8F92B
:10756000A54208BF01F0C4F968680099C008C000CE
:10757000B0EBC10F18BF01F0BBF9009907F128006B
:1075800000EBC100844206D03A699442C0F080808A
:10759000E168A9427CD1A04506D100983968012252
:1075A00082409143396075E0804506D03869804556
:1075B0006ED3D8F80800A8426AD1C4F80C80C8F885
:1075C000084067E0EC68D5F81880AC420CD0A86899
:1075D0003969884222D3C168A94204BFA168A9427F
:1075E0001CD1C460A0601BE005F11402146834B91A
:1075F00005F1100214689CB101E01A46146804F108
:1076000014031968002902BF04F110031868002848
:10761000F3D139698A4228BF106001D201F068F9BC
:10762000B8F1000F36D0E96907F5987000EB8100DA
:107630000268954208D10460A4B9E869796801221A
:1076400082409143796025E03869804508D3D8F8B5
:107650001000A84214BFC8F81440C8F8104001E058
:1076600001F046F9B4B139698C4211D3C4F81880DD
:10767000286928B1884226BF2061846101F038F969
:10768000686938B13969884202D36061846101E078
:1076900001F02EF901982D188344686840084000D5
:1076A00068604BF0010171604FEADB0446F80BB0F3
:1076B0001F2C23D807F1280000EBC4084546BBF176
:1076C000100F38BF01F014F9386820FA04F1C90727
:1076D00005D4012101FA04F404433C6007E0D8F822
:1076E0000800396988422CBF054601F001F9C8F845
:1076F0000860EE60B560C6F80C8060E05FEA1B20B1
:1077000008BF002123D0B0F5803F28BF1F211ED223
:10771000A0F58072120C02F008029040A0F5805192
:10772000090C01F004018840A0F580431B0CC2F154
:107730000E0203F00203521AD21A984002EBD03222
:10774000D01D2BFA00F101F0010101EB420107F518
:10775000987202EB8100F1610022726132617A68F5
:1077600022FA01F3DB0707D4012303FA01F11143E5
:1077700079600660B0611DE002681F291DBF4908DD
:10778000C1F119010BFA01F1594600E002465068B7
:10779000C008C000584516D002F11003CC0F03EB0F
:1077A0008403490018680028F0D13869834204D363
:1077B0001E60B261F660B66001E001F099F809F16F
:1077C0000800BDE8F68B396990688A4228BF884274
:1077D000F3D3C6609660B060F2600020B061EEE75F
:1077E0002DE9FE4F04468B46A5692E4690469946E4
:1077F0003146FFF713FEA8F128020168406801EB4B
:10780000000AAAF1270111F007000EBF0021C1F103
:10781000080101F007010AEB0100A0F12F0706F1B2
:107820001000874238BF374607F1180001905946CB
:10783000002000902046FFF719FE07F1080010F025
:10784000070F18BF01F054F81B20786007F10801FA
:1078500004F5E07090E80C5081E80C50C0F800B0DE
:10786000C0F80480C0F80C9081600198009900E095
:10787000001D07224260491C00F108025245F7D35F
:107880000129D8BF01F034F8B74200F09580BF1B42
:10789000301D311DC05940084000C85147F001015A
:1078A00071604FEAD70BF751BBF11F0F21D804EBE2
:1078B000CB0000F12805A846102F38BF01F018F8BA
:1078C000206820FA0BF1C90705D4012101FA0BF158
:1078D0000843206006E0A868216988422CBF8046E2
:1078E00001F006F8AE60C8F80C60C6F80880F560D4
:1078F0006FE0380A08BF002123D0B0F5803F28BFD1
:107900001F211ED2A0F58072120C02F008029040D6
:10791000A0F58051090C01F004018840A0F58043D6
:107920001B0CC2F10E0203F00203521AD21A984045
:1079300002EBD032D01D27FA00F101F0010101EB7A
:10794000420104EB8102002302F59870F16173613A
:107950003361626822FA01F3DB0707D4012303FADB
:1079600001F1114361600660B0611DE002681F29EA
:107970001DBF4908C1F1190107FA01F1394600E0BC
:1079800002465068C008C000B84216D002F1100389
:10799000C80F03EB8003490018680028F0D1206964
:1079A000834204D31E60B261F660B56011E003B09B
:1079B000BDE8F04F00F09CBF0BE0216990688A425F
:1079C00028BF8842F3D3C6609560B060F2600020A3
:1079D000B06103B0BDE8F08F2DE9F041714F05466D
:1079E0003868884608B9FFF728FDB96801EB080038
:1079F0002F30491E20EA010188457DD205F5D87651
:107A0000B06828B1326889188A4275D2884273D327
:107A100000F072FF01001CBF0C6811F1010F6BD068
:107A20003068201805F5D87230605368984238BF26
:107A300018467060A86960BB286908B1814200D20D
:107A40002961316174610020F06105F12802386814
:107A500068624FF0FF3028620020D260926002F12D
:107A6000080353611361801C10322028F5D34E485F
:107A7000854208BFA4F1280228D055F8040CC0089C
:107A800005EBC002A2F108000A19121A283A0146B1
:107A90001CE005F5E070024600E092687AB31368D6
:107AA00057683B449942F8D1137B1F0727D4AB6931
:107AB0001768BB4223D3D2F804C06744BB421ED22E
:107AC000A444C2F804C0E868A96922182846FFF750
:107AD000CDFC1FE08068C0B103689342FAD1027BFD
:107AE000130712D4026801604368E41844604346F7
:107AF0002846BDE8F041D2E40020BDE8F0812A69C3
:107B0000914238BF29610A19E5E700232246284639
:107B1000FFF766FEE8688045EED2A0EB0800A96991
:107B2000E86001EB0802AA6140F00100506048F0F3
:107B30000300486001F10800BDE8F08138B4194B3A
:107B40001A6882B94FF480525A604FF480344FF073
:107B5000FF329C60DA601A610422134C134D5A61A3
:107B6000C4F8BC211D6011F1400F17D28269AAB17F
:107B7000C368283199420BD200F5E0710C68A2422B
:107B800003D34D682C44A24202D389680029F5D161
:107B9000C16999423CBF4FF0FF31C16132BC002046
:107BA00070470000ACAF03206CA003206859883CEC
:107BB0002DE9F84F00258946090AC9F1000B08BFD5
:107BC000002323D0B1F5803F28BF1F231ED2A1F58B
:107BD0008072120C02F008029140A1F580531B0C38
:107BE00003F004039940A1F58044240CC2F10E0275
:107BF00004F00204D21A121BA14002EBD132D11DB3
:107C000029FA01F303F0010303EB4203074607F5EA
:107C1000987858F8230030B31F2B0FBF4C465C08F0
:107C2000C4F1190409FA04F4AC46594600E06400B2
:107C30004268D208D200A2EB09028A4203D21100A4
:107C4000054600F06881426910304FEAD47B50F855
:107C50002B00002A1CBF824294460028E7D18B46A5
:107C60006046B0BBBDBB012000FA03F35B00584285
:107C700003437868034000F04D81584203405B1E87
:107C8000180B00F01000C340590901F00801CB4067
:107C90009A0802F00402D3405C0804F002040818B9
:107CA000E3401018C3F3400620183044F3401B187B
:107CB00058F823000DE008464168C908C900A1EB47
:107CC000090159453CBF8B46054601690029F2D19F
:107CD00040690028F0D1002D00F01C81B868A0EBAD
:107CE0000900834580F0168138698542C0F0108113
:107CF0006868C008C00009EB0B01884218BF00F09B
:107D0000F7FD05EB0906B54280F00281EC68D5F875
:107D100018A0AC420CD0A8683969884222D3C16847
:107D2000A94204BFA168A9421CD1C460A0601BE0A5
:107D300005F11402146834B905F1100214689CB1FD
:107D400001E01A46146804F114031968002902BFFF
:107D500004F1100318680028F3D139698A4228BF5A
:107D6000106001D200F0C4FDBAF1000F36D0E9690D
:107D700008EB81000268954209D10460200014D10B
:107D8000E8697968012282409143796026E0386988
:107D9000824508D3DAF81000A84214BFCAF814408C
:107DA000CAF8104001E000F0A3FDBCB1386984427C
:107DB00012D3C4F818A0286930B13969884226BFA7
:107DC0002061846100F094FD686938B139698842A6
:107DD00002D36061846101E000F08AFDBBF1100F05
:107DE0000CD2D94449F003006860291D281D50F8C1
:107DF000090040F0010041F8090088E049F0030063
:107E000068604BF0010070604FEADB0046F80BB091
:107E10001F281DD807EBC00101F12804396821FA99
:107E200000F2D207A34605D4012202FA00F008436B
:107E3000386006E0A068396988422CBF834600F0AC
:107E400057FDA660CBF80C60C6F808B0F4605EE0A1
:107E50005FEA1B2008BF002123D0B0F5803F28BF78
:107E60001F211ED2A0F58072120C02F00802904071
:107E7000A0F58051090C01F004018840A0F5804371
:107E80001B0CC2F10E0203F00203521AD21A9840E0
:107E900002EBD032D01D2BFA00F101F0010101EB11
:107EA0004201F16100227261326108EB81007A685F
:107EB00022FA01F3DB0707D4012303FA01F111438E
:107EC00079600660B0611DE002681F291DBF490886
:107ED000C1F119010BFA01F1594600E00246506860
:107EE000C008C000584518D002F11003CC0F03EBB6
:107EF0008403490018680028F0D13869834204D30C
:107F00001E60B261F660B66001E000F0F1FC13E1C2
:107F100000F0EEFC0DE18B46A3E6396990688A42D9
:107F200028BF8842F1D3C6609660B060F26000203E
:107F3000B061ECE72DE9F84F064688467168484283
:107F40000140491E080B00F01000C1404A0902F030
:107F50000802D1408B0803F00403D9404D0805F016
:107F600002051018E9401818C1F34004281806F556
:107F7000987A2044E14009185AF821104868C0084E
:107F8000C0000D46A0EB080909E001464868C0089A
:107F9000C000A0EB080048453CBF81460D4608697B
:107FA0000028F2D149690029F0D130698542C0F03A
:107FB000BE806868C00808EB090BC000584518BFB0
:107FC00000F096FC05EB08008542009080F0AF8041
:107FD000EF68AC69AF420CD0A8683169884222D3FF
:107FE000C168A94204BFB968A9421CD1C760B86082
:107FF0001BE005F11402176837B905F11002176884
:108000009FB101E01A46176807F1140319680029A7
:1080100002BF07F1100318680028F3D131698A42C2
:1080200028BF106001D200F063FC002C31D0E96958
:108030000AEB81000268954208D107608FB9E869B0
:108040007168012282409143716022E0306984426C
:1080500005D32069A84214BF6761276101E000F0E1
:1080600047FCB7B13069874211D3BC61286930B190
:108070003169884226BF3861876100F039FC686940
:1080800038B13169884202D37861876101E000F03C
:108090002FFCB9F1100F0BD24BF003006860291DC3
:1080A000281D50F80B0040F0010041F80B003DE0A6
:1080B00048F00301696049F00100291D41F80800FA
:1080C000009840F80990D6F808804FEAD80BBBF129
:1080D000200F28BF00F00CFCB8F1000F22D006EBF7
:1080E000CB00776900F12804A246B8F1100F38BF21
:1080F00000F0FEFB306820FA0BF1C90705D401211E
:1081000001FA0BF10843306006E0A068316988424B
:108110002CBF824600F0ECFBA760CAF80C70C7F8D1
:1081200008A0FC60C6F808900098706104E000F0B8
:10813000DFFB0020BDE8F28F05F10800BDE8F28FFB
:108140002DE9FE4F0546AFF30080F52DDFF89C6763
:1081500080F004810B2D31BF10250B35ED08ED00AB
:108160003068EC08E04010F0030F46D0C04300F048
:108170000100041906F1280000EBC408E700D8F854
:1081800008506868C008C000B84218BF00F0B0FBD3
:10819000D5F80890454508BF00F0AAFB4D4508BF3B
:1081A00000F0A6FB6868C008C000B84218BF00F025
:1081B0009FFBC84507D13168012000FA04F421EA89
:1081C000040434600DE03069814508D3D9F80C000F
:1081D000A84204D1C8F80890C9F80C8001E000F06A
:1081E00087FB47F003006860291D281D05F108047E
:1081F000C05940F00100C851F8E0B168A94280F0D0
:10820000BE80002800F0A1804FF0010808FA04F1B8
:10821000490000FA04F4484201430C406042044023
:10822000641E200B00F01000C440610901F0080139
:10823000CC40A20802F00402D440630803F0020319
:108240000818DC401018C4F3400718183818FC4010
:10825000241806F1280000EBC40AE700DAF80890B9
:10826000D9F80400C008C000B84218BF00F040FBB5
:10827000D9F808B0D14508BF00F03AFBD94508BF8E
:1082800000F036FBD9F80400C008C000B84218BF9F
:1082900000F02EFBDA4506D1316808FA04F421EA31
:1082A000040434600DE03069834508D3DBF80C002A
:1082B000484504D1CAF808B0CBF80CA001E000F0A2
:1082C00017FB45F00300C9F804007F1B09F1040106
:1082D00047F00100485109EB05000190C751B4680F
:1082E0004FEAD40ABAF1200F28BF00F001FB34B3E3
:1082F000CDF800A006F12800756900EBCA0AD34644
:10830000102C38BF00F0F4FA3168009821FA00F21E
:10831000D30704D408FA00F00843306007E0DAF825
:108320000800316988422CBF834600F0E1FACAF8A0
:108330000850CBF80C50C5F808B0C5F80CA0B760D1
:1083400009F108040198706150E07068C0B32946D3
:108350003046FFF7EFFD040011D047E015F1400F64
:1083600028BF4FF0FF350AD20B35ED087068ED00DD
:1083700028B129463046FFF71BFC040036D1B0680F
:10838000A8421DD3411B726910290AD3501970618C
:10839000B16041F001034360415045F00305556071
:1083A0000BE00021B1607161131D40F003015160C9
:1083B000111D095841F00101195002F1080415E09E
:1083C000F06885420DD2401BB169F0604A19B26174
:1083D00040F00100506045F003054D6001F10804D4
:1083E00004E029463046FFF7F7FA0446AFF3008071
:1083F0002046FFF7EEBA002800D170472DE9FC4770
:10840000A0F10805AFF30080DFF8E064326995421F
:10841000C0F05982686800F00301012900F053821E
:10842000C1084FEAC109C10705EB090839D42C6816
:1084300010F0030F00F04982604205449542A144C8
:10844000C0F041827069854200F0C780E408202CAA
:108450005ED2D5F80CA0AF68554508BF00F048FAC9
:10846000BD4208BF00F044FA6868C008C000B0EB25
:10847000C40F18BF00F03CFA06F1280000EBC4005E
:10848000874205D031698F423FD3F968A9423CD178
:10849000BA452CD13068012101FA04F420EA040421
:1084A0003460454580F00F82D8F80440E00740F181
:1084B0000A82A00700F16881B069804540F0A08081
:1084C000F068B5618144C6F80C9049F0010068601D
:1084D0007069854202D100207061B060F069484542
:1084E00080F0F38100213046FFF728FBEDE1824563
:1084F00006D03069824508D3DAF80800A84204D1D2
:10850000C7F80CA0CAF80870CBE700F0F1F9C8E78B
:10851000EC68AF69AC420BD0A868904223D3C16825
:10852000A94204BFA168A9421DD1C460A0601CE09B
:1085300005F114031C6834B905F110031C68A4B1DB
:1085400001E063461C6804F1140CDCF800100029FB
:1085500002BF04F1100CDCF800000028F1D19342B6
:1085600028BF196001D200F0C3F9002F99D0E96942
:1085700006F5987000EB81000268954209D104600D
:10858000200011D1E8697168012282409143716035
:1085900087E73069874205D33869A84214BF7C61F8
:1085A0003C6101E000F0A4F9002C3FF47AAF31699E
:1085B0008C42AAD3A761286928B1884226BF2061CE
:1085C000846100F095F9686900283FF46AAF316969
:1085D00088429AD36061846163E798F8040000F0F0
:1085E000030003287FF45DAFC6F8089049F001014D
:1085F000D8F8040040084000C8F8040069600AE0A8
:10860000706980450AD1B06875618144C6F80890E8
:1086100049F00100686045F8099056E1E408E4007B
:10862000A144E408202C3AD2D8F80CA0D8F808705D
:10863000D04508BF00F05CF9B84508BF00F058F914
:10864000D8F80400C008C000B0EBC40F18BF00F099
:108650004FF906F1280000EBC400874207D03169CA
:108660008F42C0F08480F968414540F08080BA456F
:1086700007D13068012101FA04F420EA04043460CF
:1086800077E0824506D031698A4570D3DAF8080070
:1086900040456CD1C7F80CA0CAF8087069E0D8F85A
:1086A0000C40D8F8187044450DD0D8F8080031694E
:1086B000884222D3C168414504BFA16841451CD10D
:1086C000C460A0601BE008F11402146834B908F11A
:1086D000100214689CB101E01A46146804F11403F6
:1086E0001968002902BF04F1100318680028F3D1AB
:1086F00031698A4228BF106001D200F0F9F8002FDA
:1087000037D0D8F81C1006F5987000EB810002688D
:1087100090450AD10460200012D1D8F81C0071687D
:10872000012282409143716023E03069874205D382
:108730003869404514BF7C613C6101E000F0D8F825
:10874000BCB131698C4212D3A761D8F8100028B1AE
:10875000884226BF2061846100F0CAF8D8F814006E
:1087600038B13169884202D36061846101E000F070
:10877000BFF849F00100686045F8099070698542CA
:108780000BD1C6F80890A0E064086400C8F8044063
:1087900049F00100686045F809904FEAD907202F99
:1087A00022D206F1280000EBC704A046B9F1100F51
:1087B00038BF00F09DF8306820FA07F1C90705D4EA
:1087C000012101FA07F70743376006E0A068316925
:1087D00088422CBF804600F08BF8A560C8F80C508A
:1087E000C5F80880EC6070E05FEA192008BF00213E
:1087F00023D0B0F5803F28BF1F211ED2A0F5807284
:10880000120C02F008029040A0F58051090C01F012
:1088100004018840A0F580431B0CC2F10E0203F056
:108820000203521AD21A984002EBD032D01D29FA14
:1088300000F101F0010101EB420106F5987202EB33
:10884000810000226A612A61E961726822FA01F3FB
:10885000DB0707D4012303FA01F1114371600560BE
:10886000A8611DE002681F291DBF4908C1F1190157
:1088700009FA01F1494600E002465068C008C0000C
:10888000484526D002F11003CC0F03EB84034900C6
:1088900018680028F0D13069834204D31D60AA61B2
:1088A000ED60AD6001E000F023F8306A401E3062F8
:1088B0000BD1D6F8C80100E080680028FCD14FF049
:1088C000FF30306201E000F013F8AFF30080BDE844
:1088D000F387316990688A4228BF8842E3D3C56034
:1088E0009560A860EA600020A861DEE76CA0032024
:1088F000012000F017B800000749086808B10020FF
:1089000070470648C008C00008600549C908C9008A
:10891000091A0160704700BF94B10320B7D103204A
:10892000B0F1032080B5AFF30080024A1100182097
:10893000ABBEFBE726000200000108100902030A93
:1089400011182019120B04050C131A2128302922A2
:108950001B140D06070E151C232A313839322B241F
:108960001D160F171E252C333A3B342D261F272E9C
:10897000353C3D362F373E3F3F3F3F3F3F3F3F3F38
:108980003F3F3F3F3F3F3F3F0000000001000000EE
:1089900002000000040000000800000010000000B9
:1089A00020000000400000008000000000010000E6
:1089B0000002000000040000000800000010000099
:1089C000002000000040000000000000FFFFFFFF4B
:1089D000FDFFFFFFF9FFFFFFF1FFFFFFE1FFFFFFDB
:1089E000C1FFFFFF81FFFFFF01FFFFFF01FEFFFF50
:1089F00001FCFFFF01F8FFFF01F0FFFF01E0FFFFB7
:108A000001C0FFFF0180FFFF4DFFFFFF4EFFFFFF93
:108A10004FFFFFFF51FFFFFF52FFFFFF54FFFFFF1C
:108A200055FFFFFF56FFFFFF58FFFFFF59FFFFFFF6
:108A30005BFFFFFF5CFFFFFF5DFFFFFF5FFFFFFFCF
:108A400060FFFFFF62FFFFFF63FFFFFF64FFFFFFA9
:108A500066FFFFFF67FFFFFF69FFFFFF6AFFFFFF82
:108A60006BFFFFFF6DFFFFFF6EFFFFFF70FFFFFF5C
:108A700071FFFFFF72FFFFFF74FFFFFF75FFFFFF36
:108A800077FFFFFF78FFFFFF79FFFFFF7BFFFFFF0F
:108A90007CFFFFFF7EFFFFFF7FFFFFFF80FFFFFFE9
:108AA00082FFFFFF83FFFFFF85FFFFFF86FFFFFFC2
:108AB00087FFFFFF89FFFFFF8AFFFFFF8CFFFFFF9C
:108AC0008DFFFFFF8EFFFFFF90FFFFFF91FFFFFF76
:108AD00093FFFFFF94FFFFFF95FFFFFF97FFFFFF4F
:108AE00098FFFFFF9AFFFFFF9BFFFFFF9CFFFFFF29
:108AF0009EFFFFFF9FFFFFFFA1FFFFFFA2FFFFFF02
:108B0000A3FFFFFFA5FFFFFFA6FFFFFFA8FFFFFFDB
:108B1000A9FFFFFFAAFFFFFFACFFFFFFADFFFFFFB5
:108B2000AFFFFFFFB0FFFFFFB1FFFFFFB3FFFFFF8E
:108B3000B4FFFFFFB6FFFFFFB7FFFFFFB8FFFFFF68
:108B4000BAFFFFFFBBFFFFFFBDFFFFFFBEFFFFFF41
:108B5000C0FFFFFFC1FFFFFFC2FFFFFFC4FFFFFF1A
:108B6000C5FFFFFFC7FFFFFFC8FFFFFFC9FFFFFFF4
:108B7000CBFFFFFFCCFFFFFFCEFFFFFFCFFFFFFFCD
:108B8000D0FFFFFFD2FFFFFFD3FFFFFFD5FFFFFFA7
:108B9000D6FFFFFFD7FFFFFFD9FFFFFFDAFFFFFF81
:108BA000DCFFFFFFDDFFFFFFDEFFFFFFE0FFFFFF5A
:108BB000E1FFFFFFE3FFFFFFE4FFFFFFE5FFFFFF34
:108BC000E7FFFFFFE8FFFFFFEAFFFFFFEBFFFFFF0D
:108BD000ECFFFFFFEEFFFFFFEFFFFFFFF1FFFFFFE7
:108BE000F2FFFFFFF3FFFFFFF5FFFFFFF6FFFFFFC1
:108BF000F8FFFFFFF9FFFFFFFAFFFFFFFCFFFFFF9A
:108C0000FDFFFFFFFFFFFFFF00000000010000006D
:108C10000300000004000000060000000700000040
:108C2000080000000A0000000B0000000D0000001A
:108C30000E0000000F0000001100000012000000F4
:108C400014000000150000001600000018000000CD
:108C5000190000001B0000001C0000001D000000A7
:108C60001F00000020000000220000002300000080
:108C7000240000002600000027000000290000005A
:108C80002A0000002B0000002D0000002E00000034
:108C9000300000003100000032000000340000000D
:108CA00035000000370000003800000039000000E7
:108CB0003B0000003C0000003E0000003F000000C0
:108CC000400000004200000043000000450000009A
:108CD0004600000048000000490000004A00000073
:108CE0004C0000004D0000004F000000500000004C
:108CF0005100000053000000540000005600000026
:108D000057000000580000005A0000005B000000FF
:108D10005D0000005E0000005F00000061000000D8
:108D200062000000640000006500000066000000B2
:108D300068000000690000006B0000006C0000008B
:108D40006D0000006F000000700000007200000065
:108D5000730000007400000076000000770000003F
:108D6000790000007A0000007B0000007D00000018
:108D70007E000000800000008100000082000000F2
:108D800084000000850000008700000088000000CB
:108D9000890000008B0000008C0000008E000000A5
:108DA0008F0000009000000092000000930000007F
:108DB0009500000096000000970000009900000058
:108DC0009A0000009C0000009D0000009E00000032
:108DD000A0000000A1000000A3000000A40000000B
:108DE000A5000000A7000000A8000000AA000000E5
:108DF000AB000000AC000000AE000000AF000000BF
:108E0000B1000000B200000000695B002EB25A0001
:108E10005CFB59008A445900B88D5800E6D65700CB
:108E2000142057004269560070B255009EFB540052
:108E3000CC445400FA8D530028D7520056205200DB
:108E400084695100B2B25000E0FB4F000E454F0064
:108E50003C8E4E006AD74D0098204D00C6694C00EC
:108E6000F4B24B0022FC4A0050454A007E8E490075
:108E7000ACD74800DA204800086A470036B34600FD
:108E800064FC450092454500C08E4400EED7430087
:108E90001C2143004A6A420078B34100A6FC40000E
:108EA000D4454000028F3F0030D83E005E213E0096
:108EB0008C6A3D00BAB33C00E8FC3B0016463B0020
:108EC000448F3A0072D83900A0213900CE6A3800A8
:108ED000FCB337002AFD360058463600868F350031
:108EE000B4D83400E2213400106B33003EB43200B9
:108EF0006CFD31009A463100C88F3000F6D82F0043
:108F000024222F00526B2E0080B42D00AEFD2C00C9
:108F1000DC462C000A902B0038D92A0066222A0051
:108F2000946B2900C2B42800F0FD27001E472700DB
:108F30004C9026007AD92500A8222500D66B240063
:108F400004B5230032FE2200604722008E902100EB
:108F5000BCD92000EA222000186C1F0046B51E0074
:108F600074FE1D00A2471D00D0901C00FED91B00FE
:108F70002C231B005A6C1A0088B51900B6FE180085
:108F8000E44718001291170040DA16006E2316000D
:108F90009C6C1500CAB51400F8FE13002648130097
:108FA0005491120082DA1100B0231100DE6C10001F
:108FB0000CB60F003AFF0E0068480E0096910D00A7
:108FC000C4DA0C00F2230C00206D0B004EB60A0030
:108FD0007CFF0900AA480900D891080006DB0700B9
:108FE00034240700626D060090B60500BEFF040041
:108FF000EC4804001A92030048DB020076240200C9
:10900000A46D0100D2B60000000000002E49FFFF51
:109010005C92FEFF8ADBFDFFB824FDFFE66DFCFFDE
:1090200014B7FBFF4200FBFF7049FAFF9E92F9FF65
:10903000CCDBF8FFFA24F8FF286EF7FF56B7F6FFEF
:109040008400F6FFB249F5FFE092F4FF0EDCF3FF77
:109050003C25F3FF6A6EF2FF98B7F1FFC600F1FFFF
:10906000F449F0FF2293EFFF50DCEEFF7E25EEFF88
:10907000AC6EEDFFDAB7ECFF0801ECFF364AEBFF10
:109080006493EAFF92DCE9FFC025E9FFEE6EE8FF9A
:109090001CB8E7FF4A01E7FF784AE6FFA693E5FF21
:1090A000D4DCE4FF0226E4FF306FE3FF5EB8E2FFAA
:1090B0008C01E2FFBA4AE1FFE893E0FF16DDDFFF33
:1090C0004426DFFF726FDEFFA0B8DDFFCE01DDFFBB
:1090D000FC4ADCFF2A94DBFF58DDDAFF8626DAFF44
:1090E000B46FD9FFE2B8D8FF1002D8FF3E4BD7FFCC
:1090F0006C94D6FF9ADDD5FFC826D5FFF66FD4FF56
:1091000024B9D3FF5202D3FF804BD2FFAE94D1FFDC
:10911000DCDDD0FF0A27D0FF3870CFFF66B9CEFF65
:109120009402CEFFC24BCDFFF094CCFF1EDECBFFEE
:109130004C27CBFF7A70CAFFA8B9C9FFD602C9FF76
:10914000044CC8FF3295C7FF60DEC6FF8E27C6FFFE
:10915000BC70C5FFEAB9C4FF1803C4FF464CC3FF87
:109160007495C2FFA2DEC1FFD027C1FFFE70C0FF11
:109170002CBABFFF5A03BFFF884CBEFFB695BDFF98
:10918000E4DEBCFF1228BCFF4071BBFF6EBABAFF21
:109190009C03BAFFCA4CB9FFF895B8FF26DFB7FFAA
:1091A0005428B7FF8271B6FFB0BAB5FFDE03B5FF32
:1091B0000C4DB4FF3A96B3FF68DFB2FF9628B2FFBA
:1091C000C471B1FFF2BAB0FF2004B0FF4E4DAFFF43
:1091D0007C96AEFFAADFADFFD828ADFF0672ACFFCC
:1091E00034BBABFF6204ABFF904DAAFFBE96A9FF54
:1091F000ECDFA8FF1A29A8FF4872A7FF76BBA6FFDD
:10920000A404A6FFD24DA5FF008D2C00E6342C004F
:10921000CCDC2B00B2842B00982C2B007ED42A00AF
:10922000647C2A004A242A0030CC290016742900C4
:10923000FC1B2900E2C32800C86B2800AE132800DD
:1092400094BB27007A632700600B270046B32600F3
:109250002C5B260012032600F8AA2500DE5225000A
:10926000C4FA2400AAA22400904A240076F2230023
:109270005C9A23004242230028EA22000E92220038
:10928000F4392200DAE12100C0892100A631210051
:109290008CD9200072812000582920003ED11F0067
:1092A00024791F000A211F00F0C81E00D6701E007E
:1092B000BC181E00A2C01D0088681D006E101D0095
:1092C00054B81C003A601C0020081C0006B01B00AB
:1092D000EC571B00D2FF1A00B8A71A009E4F1A00C5
:1092E00084F719006A9F19005047190036EF1800DB
:1092F0001C971800023F1800E8E61700CE8E1700F2
:10930000B43617009ADE160080861600662E160008
:109310004CD61500327E150018261500FECD14001F
:10932000E4751400CA1D1400B0C51300966D130037
:109330007C15130062BD1200486512002E0D12004C
:1093400014B51100FA5C1100E0041100C6AC100065
:10935000AC54100092FC0F0078A40F005E4C0F007C
:1093600044F40E002A9C0E0010440E00F6EB0D0093
:10937000DC930D00C23B0D00A8E30C008E8B0C00AB
:1093800074330C005ADB0B0040830B00262B0B00C0
:109390000CD30A00F27A0A00D8220A00BECA0900D9
:1093A000A47209008A1A090070C20800566A0800EF
:1093B0003C12080022BA070008620700EE09070005
:1093C000D4B10600BA590600A001060086A905001E
:1093D0006C51050052F9040038A104001E49040034
:1093E00004F10300EA980300D0400300B6E802004D
:1093F0009C9002008238020068E001004E88010063
:10940000343001001AD8000000800000E627000078
:10941000CCCFFFFFB277FFFF981FFFFF7EC7FEFF95
:10942000646FFEFF4A17FEFF30BFFDFF1667FDFFAA
:10943000FC0EFDFFE2B6FCFFC85EFCFFAE06FCFFC3
:1094400094AEFBFF7A56FBFF60FEFAFF46A6FAFFDA
:109450002C4EFAFF12F6F9FFF89DF9FFDE45F9FFF1
:10946000C4EDF8FFAA95F8FF903DF8FF76E5F7FF09
:109470005C8DF7FF4235F7FF28DDF6FF0E85F6FF1E
:10948000F42CF6FFDAD4F5FFC07CF5FFA624F5FF37
:109490008CCCF4FF7274F4FF581CF4FF3EC4F3FF4D
:1094A000246CF3FF0A14F3FFF0BBF2FFD663F2FF64
:1094B000BC0BF2FFA2B3F1FF885BF1FF6E03F1FF7B
:1094C00054ABF0FF3A53F0FF20FBEFFF06A3EFFF92
:1094D000EC4AEFFFD2F2EEFFB89AEEFF9E42EEFFAB
:1094E00084EAEDFF6A92EDFF503AEDFF36E2ECFFC1
:1094F0001C8AECFF0232ECFFE8D9EBFFCE81EBFFD8
:10950000B429EBFF9AD1EAFF8079EAFF6621EAFFEE
:109510004CC9E9FF3271E9FF1819E9FFFEC0E8FF05
:10952000E468E8FFCA10E8FFB0B8E7FF9660E7FF1D
:109530007C08E7FF62B0E6FF4858E6FF2E00E6FF32
:1095400014A8E5FFFA4FE5FFE0F7E4FFC69FE4FF4C
:10955000AC47E4FF92EFE3FF7897E3FF5E3FE3FF62
:1095600044E7E2FF2A8FE2FF1037E2FFF6DEE1FF79
:10957000DC86E1FFC22EE1FFA8D6E0FF8E7EE0FF91
:109580007426E0FF5ACEDFFF4076DFFF261EDFFFA6
:109590000CC6DEFFF26DDEFFD815DEFFBEBDDDFFBF
:1095A000A465DDFF8A0DDDFF70B5DCFF565DDCFFD5
:1095B0003C05DCFF22ADDBFF0855DBFFEEFCDAFFEC
:1095C000D4A4DAFFBA4CDAFFA0F4D9FF869CD9FF05
:1095D0006C44D9FF52ECD8FF3894D8FF1E3CD8FF1A
:1095E00004E4D7FFEA8BD7FFD033D7FFB6DBD6FF33
:1095F0009C83D6FF822BD6FF68D3D5FF4E7BD5FF49
:109600003423D5FF1ACBD4FF1DFFFFFF1FFFFFFF41
:1096100021FFFFFF23FFFFFF24FFFFFF26FFFFFFC8
:1096200028FFFFFF2AFFFFFF2BFFFFFF2DFFFFFF9C
:109630002FFFFFFF31FFFFFF32FFFFFF34FFFFFF70
:1096400036FFFFFF38FFFFFF3AFFFFFF3BFFFFFF43
:109650003DFFFFFF3FFFFFFF41FFFFFF42FFFFFF17
:1096600044FFFFFF46FFFFFF48FFFFFF49FFFFFFEB
:109670004BFFFFFF4DFFFFFF4FFFFFFF51FFFFFFBE
:1096800052FFFFFF54FFFFFF56FFFFFF58FFFFFF92
:1096900059FFFFFF5BFFFFFF5DFFFFFF5FFFFFFF66
:1096A00061FFFFFF62FFFFFF64FFFFFF66FFFFFF39
:1096B00068FFFFFF69FFFFFF6BFFFFFF6DFFFFFF0D
:1096C0006FFFFFFF70FFFFFF72FFFFFF74FFFFFFE1
:1096D00076FFFFFF78FFFFFF79FFFFFF7BFFFFFFB4
:1096E0007DFFFFFF7FFFFFFF80FFFFFF82FFFFFF88
:1096F00084FFFFFF86FFFFFF88FFFFFF89FFFFFF5B
:109700008BFFFFFF8DFFFFFF8FFFFFFF90FFFFFF2E
:1097100092FFFFFF94FFFFFF96FFFFFF97FFFFFF02
:1097200099FFFFFF9BFFFFFF9DFFFFFF9FFFFFFFD5
:10973000A0FFFFFFA2FFFFFFA4FFFFFFA6FFFFFFA9
:10974000A7FFFFFFA9FFFFFFABFFFFFFADFFFFFF7D
:10975000AEFFFFFFB0FFFFFFB2FFFFFFB4FFFFFF51
:10976000B6FFFFFFB7FFFFFFB9FFFFFFBBFFFFFF24
:10977000BDFFFFFFBEFFFFFFC0FFFFFFC2FFFFFFF8
:10978000C4FFFFFFC6FFFFFFC7FFFFFFC9FFFFFFCB
:10979000CBFFFFFFCDFFFFFFCEFFFFFFD0FFFFFF9F
:1097A000D2FFFFFFD4FFFFFFD5FFFFFFD7FFFFFF73
:1097B000D9FFFFFFDBFFFFFFDDFFFFFFDEFFFFFF46
:1097C000E0FFFFFFE2FFFFFFE4FFFFFFE5FFFFFF1A
:1097D000E7FFFFFFE9FFFFFFEBFFFFFFEDFFFFFFED
:1097E000EEFFFFFFF0FFFFFFF2FFFFFFF4FFFFFFC1
:1097F000F5FFFFFFF7FFFFFFF9FFFFFFFBFFFFFF95
:10980000FCFFFFFFFEFFFFFF000000000200000062
:10981000040000000500000007000000090000002F
:109820000B0000000C0000000E0000001000000003
:1098300012000000130000001500000017000000D7
:10984000190000001B0000001C0000001E000000AA
:10985000200000002200000023000000250000007E
:1098600027000000290000002B0000002C00000051
:109870002E00000030000000320000003300000025
:109880003500000037000000390000003A000000F9
:109890003C0000003E0000004000000042000000CC
:1098A00043000000450000004700000049000000A0
:1098B0004A0000004C0000004E0000005000000074
:1098C0005200000053000000550000005700000047
:1098D000590000005A0000005C0000005E0000001B
:1098E00060000000610000006300000065000000EF
:1098F00067000000690000006A0000006C000000C2
:109900006E00000070000000710000007300000095
:109910007500000077000000780000007A00000069
:109920007C0000007E00000080000000810000003C
:109930008300000085000000870000008800000010
:109940008A0000008C0000008E00000090000000E3
:1099500091000000930000009500000097000000B7
:10996000980000009A0000009C0000009E0000008B
:109970009F000000A1000000A3000000A50000005F
:10998000A7000000A8000000AA000000AC00000032
:10999000AE000000AF000000B1000000B300000006
:1099A000B5000000B7000000B8000000BA000000D9
:1099B000BC000000BE000000BF000000C1000000AD
:1099C000C3000000C5000000C6000000C800000081
:1099D000CA000000CC000000CE000000CF00000054
:1099E000D1000000D3000000D5000000D600000028
:1099F000D8000000DA000000DC000000DD000000FC
:109A0000DF000000E1000000000000000000000096
:109A10000000000000000000000000000000000046
:109A20000000000000000000000000000000000036
:109A30000000000000000000000000000000000026
:109A40000000000000000000000000000000000016
:109A50000000000000000000000000000000000006
:109A600000000000000000000000000000000000F6
:109A700000000000000000000000000000000000E6
:109A800000000000000000000000000000000000D6
:109A900000000000000000000000000000000000C6
:109AA00000000000000000000000000000000000B6
:109AB00000000000000000000000000000000000A6
:109AC0000000000000000000000000000000000096
:109AD0000000000000000000000000000000000086
:109AE0000000000000000000000000000000000076
:109AF0000000000000000000000000000000000066
:109B00000000000000000000000102030405060739
:109B100008090A0B0C0D0E0F10111213141516174D
:109B200018191A1B1C1D1E1F20212223242526273D
:109B300028292A2B2C2D2E2F30313233343536372D
:109B400038393A3B3C3D3E3F40414243444546471D
:109B500048494A4B4C4D4E4F50515253545556570D
:109B600058595A5B5C5D5E5F6061626364656667FD
:109B700068696A6B6C6D6E6F7071727374757677ED
:109B800078797A7B7C7D7E7F8081828384858687DD
:109B900088898A8B8C8D8E8F9091929394959697CD
:109BA00098999A9B9C9D9E9FA0A1A2A3A4A5A6A7BD
:109BB000A8A9AAABACADAEAFB0B1B2B3B4B5B6B7AD
:109BC000B8B9BABBBCBDBEBFC0C1C2C3C4C5C6C79D
:109BD000C8C9CACBCCCDCECFD0D1D2D3D4D5D6D78D
:109BE000D8D9DADBDCDDDEDFE0E1E2E3E4E5E6E77D
:109BF000E8E9EAEBECEDEEEFF0F1F2F3F4F5F6F76D
:109C0000F8F9FAFBFCFDFEFFFFFFFFFFFFFFFFFF80
:109C1000FFFFFFFFFFFFFFFFFFFFFFFFFFFFFFFF54
:109C2000FFFFFFFFFFFFFFFFFFFFFFFFFFFFFFFF44
:109C3000FFFFFFFFFFFFFFFFFFFFFFFFFFFFFFFF34
:109C4000FFFFFFFFFFFFFFFFFFFFFFFFFFFFFFFF24
:109C5000FFFFFFFFFFFFFFFFFFFFFFFFFFFFFFFF14
:109C6000FFFFFFFFFFFFFFFFFFFFFFFFFFFFFFFF04
:109C7000FFFFFFFFFFFFFFFFFFFFFFFFFFFFFFFFF4
:109C8000FFFFFFFFFFFFFFFFFFFFFFFFFFFFFFFFE4
:109C9000FFFFFFFFFFFFFFFFFFFFFFFFFFFFFFFFD4
:109CA000FFFFFFFFFFFFFFFFFFFFFFFFFFFFFFFFC4
:109CB000FFFFFFFFFFFFFFFFFFFFFFFFFFFFFFFFB4
:109CC000FFFFFFFFFFFFFFFFFFFFFFFFFFFFFFFFA4
:109CD000FFFFFFFFFFFFFFFFFFFFFFFFFFFFFFFF94
:109CE000FFFFFFFFFFFFFFFFFFFFFFFFFFFFFFFF84
:109CF000FFFFFFFFFFFFFFFFFFFFFFFFFFFFFFFF74
:109D0000FFFFFFFFFFFFFFFF6DDF030831F20408D5
:109D100031ED0508A5BF05080000000000000000A7
:109D2000141401012C9D0008100A0D00A000FF0072
:109D3000389D0008B8AD00080505010080AD000899
:109D4000050501006CAD00080A0A020044AD0008D8
:109D50000A0A02001CAD00080A0A0200F4AC00085E
:109D60000A0A0200CCAC000804040100B8AC0008E8
:109D70000A0A020090AC0008060601007CAC00084C
:109D80000D0D020054AC00080707010040AC0008AC
:109D90000A0A020018AC00080B0B0200F0AB000826
:109DA00006060100DCAB00080D0D0200B4AB000894
:109DB0000A0A02008CAB00080707010078AB000814
:109DC0000A0A020050AB0008060601003CAB00087E
:109DD0000606010028AB00080606010014AB0008C7
:109DE0000A0A0200ECAA00080A0A0200C4AA000833
:109DF00005050100B0AA0008060601009CAA00089B
:109E00000606010088AA00080707010074AA0008D6
:109E10000A0A02004CAA00080F0F020024AA000838
:109E20000F0F0200FCA900080F0F0200D4A90008C0
:109E30000B0B0200ACA900080D0D020084A900085C
:109E40000D0D02005CA900080D0D020034A90008E8
:109E50000D0D02000CA900080D0D0200E4A8000879
:109E60000D0D0200BCA800081212030080A8000813
:109E70000D0D020058A800080C0C020030A80008C4
:109E80000C0C020008A800080C0C0200E0A7000857
:109E90000C0C0200B8A7000805050100A4A70008E3
:109EA0000505010090A70008050501007CA7000832
:109EB0000505010068A700080D0D020040A7000875
:109EC0000D0D020018A700080E0E0200F0A60008F3
:109ED0000E0E0200C8A600080E0E0200A0A6000882
:109EE0000E0E020078A600080E0E020050A6000812
:109EF0000B0B020028A600080E0E020000A60008A8
:109F00000D0D0200D8A500080D0D0200B0A5000837
:109F10000D0D020088A500080D0D020060A50008C7
:109F20000C0C020038A500080C0C020010A500085B
:109F30000C0C0200E8A400080A0A0200C0A40008F1
:109F40000A0A020098A400080A0A020070A4000885
:109F50000A0A020048A400080A0A020020A4000815
:109F60000A0A0200F8A3000810100200D0A300089B
:109F70000A0A0200A8A300080A0A020080A3000837
:109F80000A0A020058A300080A0A020030A30008C7
:109F90000A0A020008A3000805050100F4A200084F
:109FA00005050100E0A2000805050100CCA200089B
:109FB00005050100B8A200080B0B020090A20008E2
:109FC0000B0B020068A200080B0B020040A2000865
:109FD0000B0B020018A200080B0B0200F0A10008F6
:109FE0000B0B0200C8A100080B0B0200A0A1000887
:109FF0000A0A020078A100080B0B020050A1000819
:10A000000B0B020028A100080B0B020000A10008A6
:10A010000B0B0200D8A000080B0B0200B0A0000838
:10A020000A0A020088A000080B0B020060A00008CA
:10A030000A0A020038A00008000000000000198091
:10A0400019800000E0C0E0C071C071C031803B8069
:10A050001B801F001F000E000E001C007C007800FB
:10A0600000000000000070007000700077007F802A
:10A070007BC071C071C071C071C07BC07F80770030
:10A080007000700070007000000000000700060003
:10A090000C000000E0C0E0C071C071C031803B80A6
:10A0A0001B801F001F000E000E001C007C007800AB
:10A0B00000000000000019801980000071C071C00C
:10A0C00071C071C071C071C071C073C07FC03DC02C
:10A0D00000000000000000000000000000000E0072
:10A0E0001B00000071C071C071C071C071C071C02F
:10A0F00071C073C07FC03DC00000000000000000C0
:10A1000000000000070006000C00000071C071C0D4
:10A1100071C071C071C071C071C073C07FC03DC0DB
:10A120000000000000000000000000001C000C0007
:10A130000600000071C071C071C071C071C071C0F3
:10A1400071C073C07FC03DC000000000000000006F
:10A150000000000000000000000000801EC03F80E2
:10A160003B8073C077C07DC079C03B803F806F006B
:10A1700020000000000000000000000000000000BF
:10A180001C001C001C000000FF80FF80FF800000FE
:10A190001C001C001C00000000000000000000006B
:10A1A0000000000000001980198000001F003F809F
:10A1B0007BC071C071C071C071C07BC03F801F0087
:10A1C00000000000000000000000000000001C80F3
:10A1D000138000001F003F807BC071C071C071C040
:10A1E00071C07BC03F801F00000000000000000025
:10A1F0000000000000000E001B0000001F003F8058
:10A200007BC071C071C071C071C07BC03F801F0036
:10A210000000000000000000000000000700060031
:10A220000C0000001F003F807BC071C071C071C076
:10A2300071C07BC03F801F000000000000000000D4
:10A24000000000000E000600030000001F003F8019
:10A250007BC071C071C071C071C07BC03F801F00E6
:10A2600000000000000000000000000000001C8052
:10A270001380000077807FC079C071C071C071C049
:10A2800071C071C071C071C000000000000000000A
:10A290000000000000000E80070009800F803FC012
:10A2A0003BC071C071C071C071C03B803F801F0056
:10A2B0000000000000000000000000D8D80070700E
:10A2C000707070707070707000000000000000709E
:10A2D000D800707070707070707070700000000046
:10A2E0000000383060007070707070707070707046
:10A2F000000000000000E06030007070707070704E
:10A3000070707070000000000000000000001980F4
:10A31000198000001F003F8071C071C07FC07FC0E6
:10A32000700071C03F801F000000000000000000AE
:10A330000000000000000E001B0000001F003F8016
:10A3400071C071C07FC07FC0700071C03F801F00AE
:10A3500000000000000000000000000007000600F0
:10A360000C0000001F003F8071C071C07FC07FC023
:10A37000700071C03F801F0000000000000000005E
:10A38000000000000E000600030000001F003F80D8
:10A3900071C071C07FC07FC0700071C03F801F005E
:10A3A00000000000000000000000000000000000AD
:10A3B000000000001E003F007B80710070007000F4
:10A3C00071007B803F001E001E0006003C00000064
:10A3D0000000000000000000000000001E783FFCAC
:10A3E000638E078E0FFE3BFE738073CE7FFC3C783E
:10A3F000000000000000000000000C00120012002D
:10A400000C0000001F003F80638007801F803B809E
:10A41000738073807F803DC000000000000000005A
:10A420000000000000003300330000001F003F80E8
:10A43000638007801F803B80738073807F803DC076
:10A4400000000000000000000000000000003900D3
:10A45000270000001F003F80638007801F803B8033
:10A46000738073807F803DC000000000000000000A
:10A470000000000000000E001B0000001F003F80D5
:10A48000638007801F803B80738073807F803DC026
:10A4900000000000000000000000000007000600AF
:10A4A0000C0000001F003F80638007801F803B80FE
:10A4B000738073807F803DC00000000000000000BA
:10A4C000000000001C000C00060000001F003F8080
:10A4D000638007801F803B80738073807F803DC0D6
:10A4E00000000000000000000000000000001F004D
:10A4F0003F807380738077007700778073C071C06E
:10A5000070E074E07FE07780000000000000000051
:10A51000000000000000700070007F807FC07FE0BE
:10A5200070E070E070E07FE07FC07F8070007000BE
:10A5300000000000000000000380030006007070AF
:10A54000707038E01DC01DC00F800F80070007002D
:10A5500007000700070007000000000000000000DF
:10A560000CC00CC0000070707070707070707070F3
:10A57000707070707070707078F03FE03FE00F8026
:10A58000000000000000000007000D800000707057
:10A5900070707070707070707070707070707070BB
:10A5A00078F03FE03FE00F80000000000000000076
:10A5B00003800300060070707070707070707070AF
:10A5C000707070707070707078F03FE03FE00F80D6
:10A5D00000000000000000000E0006000300707084
:10A5E000707070707070707070707070707070706B
:10A5F00078F03FE03FE00F80000000000000000026
:10A600000000000000080FCC1FF83FF0387870F809
:10A6100071B8733876387C3878703FF07FE0CFC0FF
:10A6200040000000000000000000000000000000EA
:10A6300000000000210073803F001E001E003F004C
:10A6400073802100000000000000000000000000F6
:10A650000CC00CC0000007801FE03FF0387070385D
:10A66000703870387038703838703FF01FE00780ED
:10A6700000000000000000000E4009C0000007803C
:10A680001FE03FF0387070387038703870387038AC
:10A6900038703FF01FE0078000000000000000005D
:10A6A000038006C0000007801FE03FF0387070385C
:10A6B000703870387038703838703FF01FE007809D
:10A6C0000000000000000000038003000600078077
:10A6D0001FE03FF03870703870387038703870385C
:10A6E00038703FF01FE0078000000000000000000D
:10A6F00007000300018007801FE03FF038707038CA
:10A70000703870387038703838703FF01FE007804C
:10A7100000000000000000000E4009C00000707042
:10A7200078707C707C707E7076707770737073F068
:10A7300071F071F070F07070000000000000000017
:10A740000000000000007F807FE07FE070F070700C
:10A75000FE70FE707070707070F07FE07FE07F8040
:10A760000000000000000000D8D800707070707009
:10A7700070707070707070700000000070D80070A1
:10A780007070707070707070707070700000000089
:10A790003830607070707070707070707070707041
:10A7A00000000000E0703070707070707070707039
:10A7B00070707070000000001980198000007FE048
:10A7C0007FE07FE0700070007FE07FE07FE070005E
:10A7D00070007FE07FE07FE00000000000000000EC
:10A7E00007000D8000007FE07FE07FE070007000D8
:10A7F0007FE07FE07FE0700070007FE07FE07FE03F
:10A8000000000000000000000380030006007FE05D
:10A810007FE07FE0700070007FE07FE07FE070000D
:10A8200070007FE07FE07FE000000000000000009B
:10A830000E00060003007FE07FE07FE07000700004
:10A840007FE07FE07FE0700070007FE07FE07FE0EE
:10A850000000000000000000000000000000078071
:10A860001FE03FE038F070607000700070007060B2
:10A8700038F03FE01FE00780078001800F000000F4
:10A8800000000000000000000007FF800FFF800EA6
:10A89000FF801CE0001CE00038FF8038FF803FFF95
:10A8A000807FE0007FE000E0FF80E0FF80C0FF806D
:10A8B0000000000000000000000000000300048011
:10A8C00004800F800F800F801DC01DC01DC038E0A8
:10A8D0003FE03FE07FF070707070E03800000000F3
:10A8E000000000000CC00CC000000F800F800F8023
:10A8F0001DC01DC01DC038E03FE03FE07FF070701C
:10A900007070E03800000000000000000E4009C038
:10A9100000000F800F800F801DC01DC01DC038E0DB
:10A920003FE03FE07FF070707070E03800000000A2
:10A930000000000007000D8000000F800F800F80D6
:10A940001DC01DC01DC038E03FE03FE07FF07070CB
:10A950007070E03800000000000000000380030079
:10A9600006000F800F800F801DC01DC01DC038E085
:10A970003FE03FE07FF070707070E0380000000052
:10A98000000000000E00060003000F800F800F8003
:10A990001DC01DC01DC038E03FE03FE07FF070707B
:10A9A0007070E038000000000000000000000000AF
:10A9B00000000000000000000E000E000E0000006D
:10A9C0000E000E001E003C007800700071C073C0C5
:10A9D0003F801F000000000000007030D860186049
:10A9E00030C01980D980730C031C061C0C2C0C4C35
:10A9F000187E180C0000000000000000000000009D
:10AA0000000030607060F0C031C0318033003338F6
:10AA1000066C060C0C1C18381870307C0000000006
:10AA2000000000000000000000001860386078C0DE
:10AA300018C0198019801B0C031C061C062C0C4C1A
:10AA40000C7E180C00000000000000000000000058
:10AA500000000000000000000000660033003B80A2
:10AA60001DC01DC03B8033006600000000000000D8
:10AA7000000000000000003C66666666663C000060
:10AA800000000000000000000000003070F03030D6
:10AA90003030000000000000000000000000000056
:10AAA0000000000000000000000000007818F00026
:10AAB0000000000000000000707070000000000046
:10AAC000000000000000000000003FC07FC0FD80CB
:10AAD000FD80FD807D803D800D800D800D800D808E
:10AAE0000D800D800D800D800D80000000000000A5
:10AAF000000000000000000073807380738073808A
:10AB000073807380738073807F807F80700070009B
:10AB1000700070000000001C1830000000000000F1
:10AB2000000000000000000000000070D81830187D
:10AB3000D87000000000000000000000000000705D
:10AB4000D8183870E0F80000000000000000000095
:10AB50000000000000000E000E000E007FC07FC04D
:10AB60007FC00E000E000E0000007FC07FC07FC0BF
:10AB70000000000000000000000000384444443899
:10AB8000000000000000000000000000FFC0FFC047
:10AB900000000000000000000000000000000000B5
:10ABA00000000000000000000000000000000000A5
:10ABB000000000000000000000000F8030606030E6
:10ABC0004F10888888888F08890888884890603066
:10ABD00030600F8000000000000000000000000056
:10ABE0000000000000007C7C7C00000000000000F1
:10ABF0000000000000000000000000007FC07FC0D7
:10AC00007FC001C001C001C001C000000000000001
:10AC10000000000000000000000000000000000034
:10AC2000000000000000198033007700EE00EE0005
:10AC300077003300198000000000000000000000D1
:10AC400000000078CC0C7CCCCC7C00000000000024
:10AC5000000000000000000000000F803060603045
:10AC600047908CC89808980898088CC8479060301E
:10AC700030600F800000000000000000000000CCE9
:10AC8000CC000000000000000000000000000000F8
:10AC90000000000000003C007E00630060003800FF
:10ACA0007E00CF00C380E18071803F001E0007005E
:10ACB000630073003F001E00000000606060606081
:10ACC0006060000000606060606060600000000024
:10ACD0000000E0C071C071C03B803B801F007FC09E
:10ACE0007FC00E007FC07FC00E000E00000000007D
:10ACF0000000000000000000000000000000210033
:10AD00007F80FFC07380618061807380FFC07F801F
:10AD10002100000000000000000000000000000012
:10AD200000001E003F00738073807000FE00FE0074
:10AD3000380038007000FC80FFC047800000000031
:10AD40000000000000000000000000800100010081
:10AD50001F003F807BC072007400740075C079C012
:10AD60003F801F00100010001000200000000000B5
:10AD700000007070700020207070707070707070C3
:10AD800000000000000000000000000000000000C3
:10AD9000000000006DDF030831F2040831ED050802
:10ADA000A5BF050800000000000000001414010108
:10ADB000B8AD0008100A0D0020007E00C4AD0008E8
:10ADC0000000000005050100C8BD000805050100E0
:10ADD000B4BD0008090902008CBD00080A0A02007F
:10ADE00064BD00080A0A02003CBD000811110300FE
:10ADF00000BD00080D0D0200D8BC000804040100CD
:10AE0000C4BC000806060100B0BC0008060601002C
:10AE10009CBC00080707010088BC00080B0B02005F
:10AE200060BC0008050501004CBC000806060100D6
:10AE300038BC00080505010024BC00080505010018
:10AE400010BC00080A0A0200E8BB00080A0A020057
:10AE5000C0BB00080A0A020098BB00080A0A0200E8
:10AE600070BB00080A0A020048BB00080A0A020078
:10AE700020BB00080A0A0200F8BA00080A0A020009
:10AE8000D0BA00080A0A0200A8BA00080A0A02009A
:10AE900080BA0008070701006CBA00080707010024
:10AEA00058BA00080B0B020030BA00080B0B020066
:10AEB00008BA00080B0B0200E0B900080B0B0200F7
:10AEC000B8B90008121203007CB900080D0D020089
:10AED00054B900080D0D02002CB900080D0D020038
:10AEE00004B900080D0D0200DCB800080C0C0200CB
:10AEF000B4B800080B0B02008CB800080E0E02005C
:10AF000064B800080D0D02003CB8000805050100FA
:10AF100028B800080A0A020000B800080D0D020057
:10AF2000D8B700080B0B0200B0B700080F0F0200E3
:10AF300088B700080D0D020060B700080E0E020071
:10AF400038B700080C0C020010B700080E0E020003
:10AF5000E8B600080D0D0200C0B600080C0C020097
:10AF600098B600080B0B020070B600080D0D020029
:10AF700048B600080D0D020020B6000811110300AC
:10AF8000E4B500080C0C0200BCB500080D0D020071
:10AF900094B500080A0A02006CB500080606010014
:10AFA00058B500080505010044B500080606010073
:10AFB00030B500080B0B020008B500080A0A0200B1
:10AFC000E0B4000806060100CCB400080A0A02003A
:10AFD000A4B400080B0B02007CB400080A0A0200AB
:10AFE00054B400080B0B02002CB400080B0B020039
:10AFF00004B4000806060100F0B300080B0B0200C1
:10B00000C8B300080B0B0200A0B30008050501003F
:10B010008CB300080505010078B300080A0A020095
:10B0200050B30008050501003CB3000811110300EE
:10B0300000B300080B0B0200D8B200080B0B020093
:10B04000B0B200080B0B020088B200080B0B020024
:10B0500060B20008070701004CB200080A0A0200AB
:10B0600024B200080606010010B200080B0B020013
:10B07000E8B100080B0B0200C0B100080F0F02007E
:10B0800098B100080B0B020070B100080B0B020016
:10B0900048B100080909020020B1000807070100B3
:10B0A0000CB1000804040100F8B000080707010013
:10B0B000E4B000080B0B0200BCB000080000000068
:10B0C000000000000000000000007840FFC0FFC04A
:10B0D0008780000000000000000000000000000069
:10B0E00000000000000000E0F03030303030381C4C
:10B0F0001C3830303030F0E000000060606060608C
:10B100006060606060606060606060600000000EB1
:10B110001E181818181838707038181818181E0EBD
:10B120000000000000000000000000007F007F0021
:10B1300007000E001C001C00380070007F007F001C
:10B1400000000000000000000000000000000000FF
:10B1500000000000E0E0E0E071C071C031803B80A1
:10B160001B801F001F000E000E001C007C007800DA
:10B1700000000000000000000000000071C03B80E3
:10B180003B801F000E000E001F003B803B8071C003
:10B1900000000000000000000000000000000000AF
:10B1A00000000000E38EE38E638C77DC76DC36D81B
:10B1B0003EF83C781C701C7000000000000000008D
:10B1C00000000000000000000000000071C071C01D
:10B1D00071C03B803B801B001F001F000E000E0053
:10B1E000000000000000000000000000000000005F
:10B1F0000000000071C071C071C071C071C071C029
:10B2000071C073C07FC03DC000000000000000009E
:10B21000000000307070FCFC7070707070707C3CCE
:10B22000000000000000000000000000000000001E
:10B230003F007F80738078003E001F00078073808E
:10B240007F803F00000000000000000000000000C0
:10B250000000767E78707070707070700000000072
:10B260000000000000000000000000001DC03FC002
:10B270007BC071C071C071C071C07BC03FC01DC0B8
:10B2800001C001C001C001C00000000000000000BA
:10B290000000000077007F807BC071C071C071C06A
:10B2A00071C07BC07F8077007000700070007000FC
:10B2B0000000000000000000000000001F003F80B0
:10B2C0007BC071C071C071C071C07BC03F801F0066
:10B2D000000000000000000000000000000000006E
:10B2E0000000000077807FC079C071C071C071C05C
:10B2F00071C071C071C071C000000000000000008A
:10B30000000000000000000000000000000000003D
:10B310000000779E007FFF0079E70071C70071C7CA
:10B320000071C70071C70071C70071C70071C70005
:10B33000000000000000000000000000000000709D
:10B3400070707070707070707070707000000000BD
:10B3500000000000000070007000700071C0738079
:10B3600077007E007E007F0077007380738071C05D
:10B37000000000000000000000000070700070700D
:10B3800070707070707070707070F0E0000000701D
:10B3900070007070707070707070707000000000DD
:10B3A00000000000000070007000700077807FC017
:10B3B00079C071C071C071C071C071C071C071C0FD
:10B3C000000000000000000000000000000000007D
:10B3D000000000001DC03FC07BC071C071C071C0C3
:10B3E00071C07BC03FC01DC001C071C07F803F00E5
:10B3F0000000003C7C70FCFC7070707070707070AD
:10B40000000000000000000000000000000000003C
:10B410001F003F8071C071C07FC07FC0700071C0CD
:10B420003F801F000000000000000000000000003E
:10B43000000001C001C001C01DC03FC07BC071C081
:10B4400071C071C071C07BC03FC01DC00000000052
:10B4500000000000000000000000000000000000EC
:10B460001E003F007B8071007000700071007B80C7
:10B470003F001E000000000000000000000000006F
:10B48000000070007000700077007F807BC071C08A
:10B4900071C071C071C07BC07F8077000000000068
:10B4A000000000000000000000000000000000009C
:10B4B0001F003F80638007801F803B807380738004
:10B4C0007F803DC00000000000000000000000E0A0
:10B4D00060300000000000000000000000000000DC
:10B4E000000000000000000000000000000000005C
:10B4F000000000000000000000000000000000004C
:10B5000000000000FFC0FFC00000000000000E00AF
:10B510000E001F001B003B80318071C00000000046
:10B52000000000000000000000000000000000001B
:10B53000000000F8F8F838383838383838383838F3
:10B5400038F8F8F8000000C0C0606060607030300B
:10B5500030301818000000000000007C7C7C707007
:10B560007070707070707070707C7C7C0000000077
:10B5700000007FC07FC07FC0038007000E001E0058
:10B580001C0038007000FFC0FFC0FFC000000000BA
:10B59000000000000000000000007070707038E0D3
:10B5A0001DC01DC00F800F800700070007000700A7
:10B5B000070007000000000000000000000000007D
:10B5C000000070E070E039C019801F800F000F008C
:10B5D0000F001F80198039C070E070E0000000008B
:10B5E00000000000000000000000000000E1C38037
:10B5F000E1C380E3E38073670073670077770077C8
:10B6000077007637007637003E3E003E3E003C1E17
:10B61000003C1E00000000000000000000000000D0
:10B62000000000000000E038E0387070707070704A
:10B6300038E038E01DC01DC01DC00F800F800F8096
:10B64000000000000000000000000000000070701A
:10B6500070707070707070707070707070707070EA
:10B6600078F03FE03FE00F800000000000000000A5
:10B67000000000000000FFE0FFE0FFE00E000E0011
:10B680000E000E000E000E000E000E000E000E004A
:10B6900000000000000000000000000000001F800B
:10B6A0003FC07FE070E070007F003FC00FE000E02F
:10B6B00070E07FE03FC01F8000000000000000003D
:10B6C0000000000000007FC07FE07FF070707070AD
:10B6D0007FF07FE07F8073C071E070E070F0707881
:10B6E00000000000000000000000000000000FC08B
:10B6F0001FE03FF03870703870387038713873F868
:10B7000039F83FF01FF00FB80010000000000000F3
:10B710000000000000007F807FC07FE070E070E0EC
:10B720007FE07FC07F80700070007000700070004C
:10B730000000000000000000000000000000078082
:10B740001FE03FF0387070387038703870387038DB
:10B7500038703FF01FE0078000000000000000008C
:10B76000000000000000707078707C707C707E704B
:10B7700076707770737073F071F071F070F07070B4
:10B780000000000000000000000000000000783C05
:10B79000783C7C7C7C7C7C7C76DC76DC76DC76DCC5
:10B7A000739C739C739C711C0000000000000000DF
:10B7B0000000000000007000700070007000700059
:10B7C000700070007000700070007FC07FC07FC08C
:10B7D000000000000000000000000000000070F009
:10B7E00071E071C0738077007F007F807B8071C0C3
:10B7F00071C070E070707070000000000000000008
:10B8000000000000000003800380038003800380A9
:10B81000038003800380E380E380FF807F003E009D
:10B8200000000000000000000000007070707070E8
:10B830007070707070707070000000000000000088
:10B840000000707070707070707070707FF07FF0BA
:10B850007FF0707070707070707070700000000019
:10B860000000000000000000000007C01FF03FF0D3
:10B8700038787030700071F871F871F838383FF826
:10B880001FF007C0000000000000000000000000E2
:10B8900000007FC07FC07FC0700070007F807F800D
:10B8A0007F80700070007000700070000000000069
:10B8B000000000000000000000007FE07FE07FE06B
:10B8C000700070007FE07FE07FE0700070007FE03C
:10B8D0007FE07FE0000000000000000000000000AA
:10B8E00000007F807FE07FE070F07070707070709B
:10B8F0007070707070F07FE07FE07F80000000006B
:10B900000000000000000000000007801FE03FE092
:10B9100038F07060700070007000706038F03FE0C8
:10B920001FE0078000000000000000000000000091
:10B9300000007FC07FE07FF0707070707FE07FC09C
:10B940007FE0707070707FF07FE07FC000000000CB
:10B95000000000000000000000000F800F800F803A
:10B960001DC01DC01DC038E03FE03FE07FF070709B
:10B970007070E038000000000000000000000000CF
:10B98000000000000001F80007FE001E0F0019DB98
:10B990000033FB803639806E39806C31806C3180A9
:10B9A0006C73006C770067FE0037B8003801C01E6A
:10B9B00007800FFF0003FC000000000000001F00D4
:10B9C0003F8079C071C003C007800F000E000E00D9
:10B9D00000000E000E000E0000000000000000003D
:10B9E00000000000000000000000400070007E0029
:10B9F0001F8003C003C01F807E0070004000000055
:10BA00000000000000000000000000000000000036
:10BA1000000000007FC07FC07FC0000000007FC02A
:10BA20007FC07FC000000000000000000000000098
:10BA300000000000000000000000004001C00FC036
:10BA40003F00780078003F000FC001C000400000B8
:10BA50000000000000000000000000000000383876
:10BA600038000000003838380818300000000000A6
:10BA70000000383838000000003838380000000076
:10BA80000000000000001E003F0073007380738000
:10BA9000738073803F801F80038073003F001E000F
:10BAA00000000000000000000000000000001E0078
:10BAB0003F007380738073803F001E0033007380EB
:10BAC000738073803F001E00000000000000000033
:10BAD0000000000000007F807F80038007000600D8
:10BAE0000E000C001C001C00380038003800380024
:10BAF00000000000000000000000000000001F0027
:10BB00003F80338070007E007F007380738073807D
:10BB1000738033803F001E00000000000000000022
:10BB20000000000000001F001F00380030003E0031
:10BB30003F00738003800380038073803F001E00FA
:10BB400000000000000000000000000000000700EE
:10BB50000F000F001F00370037006700C700FFC04D
:10BB6000FFC0070007000700000000000000000001
:10BB70000000000000001E003F00738073800380FF
:10BB80000F000F0003800380738073803F001E004E
:10BB900000000000000000000000000000001E0087
:10BBA0003F00738073800380070007000E001C00B5
:10BBB0001C0038007F807F80000000000000000033
:10BBC00000000000000006000E003E007E006E0037
:10BBD0004E000E000E000E000E000E000E000E00B5
:10BBE00000000000000000000000000000001E0037
:10BBF0003F00330073807380738073807380738021
:10BC0000738033003F001E000000000000000000B1
:10BC10000000001818303030307060606060C0C0C4
:10BC20000000000000000000000000000000000014
:10BC300000707070000000000000000000000000B4
:10BC400000007C7C7C000000000000000000000080
:10BC500000000000000000000070707010306000F4
:10BC6000000000000000000000000E000E000E00AA
:10BC70007FC07FC07FC00E000E000E0000000000DD
:10BC8000000000000000000000000030B4FC30782C
:10BC9000CC00000000000000000000000000006078
:10BCA000707030383838383838383838307070601C
:10BCB00000000018383830707070707070707070DC
:10BCC0003030381800000070707070700000000094
:10BCD00000000000000000000000000000000F0055
:10BCE0003FC039C039C01D800F001F003FB073F046
:10BCF00071E071F03FF81F1000000000000000002C
:10BD00000000000000000000003C180066300066E3
:10BD100030006660006660003CC00000C00001802A
:10BD200000019E0003330003330006330006330096
:10BD30000C1E0000000000000000000000000000D9
:10BD400008003E007F00EB80E800E8007C003F0038
:10BD50000F800B80EB80EB807F003E000800080026
:10BD6000000000000000000000000CC00CC01980A2
:10BD7000FFC0FFC019803B803300FFC0FFC033000D
:10BD800066006600000000000000000000000000E7
:10BD90000000770077007700770077000000000050
:10BDA0000000000000000000000000000000000093
:10BDB0000000000000000070707070707070202033
:10BDC0000070707000000000000000000000000023
:10BDD00000000000000000000000000047F288435F
:10BDE0002DE9F04FC358AFB00990002B40F02F82DF
:10BDF00047F20943C35C002B00F0528200F0E4FFDD
:10BE0000002840F0668247F22043099AD358099DE2
:10BE100047F20841012047F288426854AB50099B21
:10BE200003F5E9442368002B00F0C087079347F22D
:10BE30007443099CE05801F053F90D90002800F07C
:10BE40004F8247F21843E358002B40F3468247F2F3
:10BE5000184301460020E31808900B936D4B0A939A
:10BE6000034601EBC3110A9B80220EA81B6898476A
:10BE70000DF1480E19E03EF9103C0EF1100E9B003A
:10BE80001BB22EF8203C2EF81E3C2EF81C3C2EF83F
:10BE90001A3C2EF8183C2EF8163C2EF8143C2EF8BE
:10BEA000123C32AB734500F0AC803EF90E0C3EF90B
:10BEB0000C5C3EF9062C3EF90A1C40EA0503564F7D
:10BEC00002EB000A56183EF9089C0B433EF9048C1D
:10BED00007FB06F63EF902CC49EA030305EB08042A
:10BEE00002920CEB0007134301964CF2DF4241F241
:10BEF000511648EA030318FB02FB06FB04F441F663
:10BF00007E020CEB01065CEA0303444B05FB024591
:10BF1000434A5C44009506EB0A0502FB07F742F230
:10BF2000A15202FB05F503FB06563E4B03FB0A55E7
:10BF3000A1D03EF910BCBB19019A2F440EF1100E8E
:10BF400002EB050A0BEB09051644009A6D03C9EBD9
:10BF50000B0B02EB0508AD1A43F20B024FEA4B3B09
:10BF600010FB027740F68E1204EB0B09C4EB0B04B6
:10BF70001CFB023C44F2B313BDF8082008EB070099
:10BF8000C7EB080712FB03AB46F2542300F58060B1
:10BF900007F5806711FB036605EB0C0104EB0B034F
:10BFA000CCEB050509EB0602CBEB040BC6EB09064F
:10BFB00001F5806105F5806502F5806206F5806611
:10BFC00003F580630BF5806BC012DB12FF122EF8B5
:10BFD000200CC9122EF81C3CED122EF8127CD21245
:10BFE0002EF81A1CF6122EF8185C4FEAEB2B2EF8DE
:10BFF0001E2C2EF8146C32AB2EF816BC73457FF451
:10C0000054AF0DF1380EDDF81C800823F346C4460A
:10C0100002932AE0B4030020FDADFFFF3BC1FFFF08
:10C0200033E3FFFF84F3FFFFBBF9003010335B11F4
:10C03000803383F30803DBB28CF800308CF80830CF
:10C040008CF810308CF818308CF820308CF82830B0
:10C050008CF830308CF83830029B0BF1020B0CF16D
:10C06000010C013B029300F0ED85BBF910E0BBF938
:10C070002010BBF930904EEA0102BBF94050BBF9E9
:10C08000504049EA0202BBF96030BBF970002A4314
:10C090000094019022431A430243C5D0024604464D
:10C0A000944F01EB03084A44BBF900A01646009ADE
:10C0B00002EB0E0004EB0E02344607FB02F741F2DE
:10C0C00051120444049742F2A15702FB08F841F6CA
:10C0D0007E0207FB04F40AEB0507C5EB0A0501FB2A
:10C0E00002814CF2DF420695834D13FB02F343F2CB
:10C0F0000B0205FB00407D03049F4344039507EBBF
:10C10000000A009D7D4F1EFB02A24D4407FB064422
:10C110007B4E1746059206FB05F5039E01EB060ACA
:10C12000049E28440AEB070E2644069F2C440EF575
:10C13000003E324646F25425039E4FEAAE4E4FEA89
:10C140004738711A0EF1800E40F68E16BDF8047055
:10C1500019FB05441FFA8EFE17FB0622BDF800707E
:10C160000FFA8EF544F2B31617FB060015F47F4F55
:10C1700003EB0807C3EB080340F032855FFA8EFE3D
:10C18000059D8CF800E0C5EB0A0606F50036B614EE
:10C190008036B6B235B215F47F4F40F04D85F6B219
:10C1A0003D198CF8386005F50035AD148035ADB219
:10C1B0002EB216F47F4F40F03985EDB23C1B8CF85F
:10C1C000085004F50034A4148034A4B225B215F448
:10C1D0007F4F40F02585E5B21C188CF8305004F5EF
:10C1E0000034A4148034A4B225B215F47F4F40F07B
:10C1F0001185E4B21B1A8CF8104003F500339B1430
:10C2000080339BB218B210F47F4F40F0FD84D8B257
:10C210008B188CF8280003F500339B1480339BB2F5
:10C2200018B210F47F4F40F0E984DBB28A1A8CF820
:10C23000183002F500339B1480339BB21AB212F40B
:10C240007F4F40F0D584DBB28CF8203004E747F212
:10C2500008420146825C002A7FF4E1AD47F20A42BF
:10C260008A5C042A0ED8DFE812F02D0257029D03E3
:10C2700005004D00DA0740F1F98447F294420121AC
:10C2800009988154099E47F28441013B47F2884452
:10C29000725800203351013A72502FB0BDE8F08F30
:10C2A00000F032FFA8B9099947F2204447F28442CE
:10C2B0000B598A589A423FF7AAAD08460EA901F0D9
:10C2C0000FFE30B99DF83830D92B02D1099B1B598C
:10C2D0009DE501202FB0BDE8F08F0DA802F012F807
:10C2E000099C002147F2884347F20842E358A154D1
:10C2F0002146B3E733E3FFFF84F3FFFF3BC1FFFFBA
:10C30000FDADFFFFD907B8D4099E47F2204147F29F
:10C310008C427458B058E41A00F0E2FE47F29043A1
:10C320000D900546F05800F0DBFE072C0E9000F350
:10C33000318506F5E9431A6802EBC40A631047F237
:10C340000C41099CDB0061580029049140F3AB814A
:10C3500003F5827305F120010AF1400ADFF8B4B356
:10C36000D318029100F120010193E84B00910AF1EA
:10C370008006029A504603969DE8220095F83C708C
:10C38000403015F804EC20320BEB870710F880CC16
:10C390000BEB8E0E0435D7F8D0442031DEF8D06890
:10C3A000D7F8D070DEF8D0EC34441F4403EB2444BB
:10C3B0009E4407EB0C0904EB0C08F44499F8D89060
:10C3C00098F8D8809CF8D8C002F83F8C02F8409CBE
:10C3D00002F83ECC10F87FCC07EB0C0904EB0C08FC
:10C3E000F44499F8D89098F8D8809CF8D8C002F80E
:10C3F0003C9C02F83B8C02F83ACC10F878CC07EB66
:10C400000C0904EB0C08F44499F8D89098F8D880FB
:10C410009CF8D8C001F8409C01F83F8C01F83ECC54
:10C4200010F877CC67446444E64497F8D87094F8E1
:10C43000D84001F83C7C01F83B4C9EF8D84001F80C
:10C440003A4C95F8397015F807EC0BEB870710F8A4
:10C450007ECC0BEB8E0ED7F8D044DEF8D068D7F840
:10C46000D070DEF8D0EC34441F4403EB24449E44E7
:10C4700007EB0C0904EB0C08F44499F8D89098F8F1
:10C48000D8809CF8D8C002F8378C02F8389C02F8A3
:10C4900036CC10F87DCC07EB0C0904EB0C08F44407
:10C4A00099F8D89098F8D8809CF8D8C002F8349CB5
:10C4B00002F8338C02F832CC10F876CC07EB0C097A
:10C4C00004EB0C08F44499F8D89098F8D8809CF8BC
:10C4D000D8C001F8389C01F8378C01F836CC10F838
:10C4E00075CC67446444E64497F8D87001F8347C0E
:10C4F00094F8D8709EF8D84001F8337C01F8324C9B
:10C5000095F83A7015F806EC0BEB870710F87CCC21
:10C510000BEB8E0ED7F8D044DEF8D068D7F8D07089
:10C52000DEF8D0EC34441F4403EB24449E4407EB74
:10C530000C0904EB0C08F44499F8D89098F8D880CA
:10C540009CF8D8C002F82F8C02F8309C02F82ECC50
:10C5500010F87BCC07EB0C0904EB0C08F44499F8B9
:10C56000D89098F8D8809CF8D8C002F82C9C02F893
:10C570002B8C02F82ACC10F874CC07EB0C0904EBD6
:10C580000C08F44499F8D89098F8D8809CF8D8C052
:10C5900001F8309C01F82F8C01F82ECC10F873CCE8
:10C5A0006444E644674497F8D8C094F8D8709EF87D
:10C5B000D84001F82CCC01F82B7C01F82A4C95F8D6
:10C5C0003B7015F805EC0BEB870710F87ACC0BEBFA
:10C5D0008E0ED7F8D044DEF8D068D7F8D070DEF8E9
:10C5E000D0EC34441F4403EB24449E4407EB0C0975
:10C5F00004EB0C08F44499F8D89098F8D8809CF88B
:10C60000D8C002F8278C02F8289C02F826CC10F833
:10C6100079CC07EB0C0904EB0C08F44499F8D8909A
:10C6200098F8D8809CF8D8C002F8249C02F8238C93
:10C6300002F822CC10F872CC07EB0C0904EB0C08C2
:10C64000F44499F8D89098F8D8809CF8D8C001F8AC
:10C65000289C01F8278C01F826CC10F871CC644492
:10C66000E644674494F8D8C09EF8D84097F8D8704C
:10C6700001F8224C039C01F823CCA04201F8247C51
:10C680007FF47CAE029A0AF5C07A40320292009A98
:10C6900040320092019A02F5C0720192049A013A66
:10C6A00004927FF464AE0DA801F02CFE0EA801F0F8
:10C6B00029FE099C47F29442002147F28843A15485
:10C6C000E358DFE5099D47F2204147F28C426C5860
:10C6D000A858E41A00F004FD47F20C4105F5E943BF
:10C6E00006460E906D581A68002D02EBC404DDDD7D
:10C6F000074B1F46214630463B6808229847013DBC
:10C7000004F1400406F10806F4D1CFE7309A00089E
:10C71000B403002038890008099E47F2204147F2FF
:10C720008C427158B058CD1A00F0DAFC47F20C4236
:10C7300006F5E9430E90B4581968002C01EBC501C9
:10C74000B4DD00F12002DFF858B2944B91F880700C
:10C75000013C087802F120020BEB870791F840605A
:10C76000184401F1C001D7F8D0500BEB8606054400
:10C7700095F8D85002F8405CD7F8D074D6F8D05865
:10C780003D4400EB254595F8D85002F83F5CD6F8BB
:10C79000D05C284490F8D80002F83E0C11F83F7C99
:10C7A00011F8BF0C0BEB870711F87F6C1844D7F812
:10C7B000D0500BEB8606054495F8D85002F83C5C47
:10C7C000D7F8D074D6F8D0583D4400EB254595F8FD
:10C7D000D85002F83B5CD6F8D05C284490F8D800DA
:10C7E00002F83A0C11F83E7C11F8BE0C0BEB8707EF
:10C7F00011F87E6C1844D7F8D0500BEB8606054430
:10C8000095F8D85002F8385CD7F8D074D6F8D058DC
:10C810003D4400EB254595F8D85002F8375CD6F832
:10C82000D05C284490F8D80002F8360C11F83D7C12
:10C8300011F8BD0C0BEB870711F87D6C1844D7F885
:10C84000D0500BEB8606054495F8D85002F8345CBE
:10C85000D7F8D074D6F8D0583D4400EB254595F86C
:10C86000D85002F8335CD6F8D05C284490F8D80051
:10C8700002F8320C11F83C7C11F8BC0C0BEB87076A
:10C8800011F87C6C1844D7F8D0500BEB86060544A1
:10C8900095F8D85002F8305CD7F8D074D6F8D05854
:10C8A0003D4400EB254595F8D85002F82F5CD6F8AA
:10C8B000D05C284490F8D80002F82E0C11F83B7C8C
:10C8C00011F8BB0C0BEB870711F87B6C1844D7F8F9
:10C8D000D0500BEB8606054495F8D85002F82C5C36
:10C8E000D7F8D074D6F8D0583D4400EB254595F8DC
:10C8F000D85002F82B5CD6F8D05C284490F8D800C9
:10C9000002F82A0C11F83A7C11F8BA0C0BEB8707E5
:10C9100011F87A6C1844D7F8D0500BEB8606054412
:10C9200095F8D85002F8285CD7F8D074D6F8D058CB
:10C930003D4400EB254595F8D85002F8275CD6F821
:10C94000D05C284490F8D80002F8260C11F8397C05
:10C9500011F8B90C0BEB870711F8796C1844D7F86C
:10C96000D0500BEB8606054495F8D85002F8245CAD
:10C97000D7F8D074D6F8D0583D4400EB254595F84B
:10C98000D85002F8235CD6F8D05C284490F8D80040
:10C9900002F8220C7FF4DAAE88E600BF309A000875
:10C9A00038890008099D47F2204147F28C426C58B3
:10C9B000A858E41A00F094FB47F20C4105F5E9424F
:10C9C000E3000E9069581268002901917FF76EAE5E
:10C9D00003F14005843300F12006DFF88CB2D7184C
:10C9E0001544A04B05F180023C4629460295009271
:10C9F000324694F83CE0403114F8048C20320BEBC2
:10CA00008E0E11F880CC0BEB88080434DEF8D004CD
:10CA1000D8F8D058DEF8D0E0D8F8D08C28449E441E
:10CA200003EB204098440EEB0C0A00EB0C09C444C5
:10CA30009AF8D8A099F8D8909CF8D8C002F83F9CF2
:10CA400002F840AC02F83ECC11F87FCC6044E044E0
:10CA5000E6449EF8D8C090F8D8E098F8D80002F8DC
:10CA60003CCC02F83BEC02F83A0C94F839E014F8AC
:10CA7000078C0BEB8E0E11F87ECC0BEB8808DEF8E2
:10CA8000D004D8F8D058DEF8D0E0D8F8D08C2844BC
:10CA90009E4403EB204098440EEB0C0A00EB0C097B
:10CAA000C4449AF8D8A099F8D8909CF8D8C002F855
:10CAB000379C02F838AC02F836CC11F87DCCE04453
:10CAC0006044E64490F8D8C09EF8D8E098F8D800C2
:10CAD00002F833CC02F834EC02F8320C94F83AE065
:10CAE00014F8068C0BEB8E0E11F87CCC0BEB88083F
:10CAF000DEF8D004D8F8D058DEF8D0E0D8F8D08CE2
:10CB000028449E4403EB204098440EEB0C0A00EBB3
:10CB10000C09C4449AF8D8A099F8D8909CF8D8C0C9
:10CB200002F82F9C02F830AC02F82ECC11F87BCC26
:10CB30006044E044E6449EF8D8C090F8D8E098F805
:10CB4000D80002F82CCC02F82BEC02F82A0C94F84E
:10CB50003BE014F805CC0BEB8E0E0BEB8C0CDEF8E7
:10CB6000D004DCF8D058DEF8D0E02844DCF8D08CD3
:10CB70009E4411F87ACC03EB204098440EEB0C0A4B
:10CB800000EB0C09C4449AF8D8A09CF8D8C099F8D6
:10CB9000D89002F828AC02F8279C02F826CC11F8AD
:10CBA00079CC6044E644E0449EF8D8C090F8D8E0E0
:10CBB00098F8D80002F824CC02F8220C009802F869
:10CBC00023EC81427FF415AF019A4036029D07F5B0
:10CBD0008077013A05F5807501927FF403AF65E532
:10CBE000002DACBF4FF0FF0E4FF0000EFFF7C8BA9C
:10CBF000002AACBFFF230023FFF726BB0028ACBFF1
:10CC0000FF230023FFF712BB0028ACBFFF2000204A
:10CC1000FFF7FEBA002DACBFFF240024FFF7EABAED
:10CC2000002DACBFFF250025FFF7D6BA002EACBF04
:10CC3000FF250025FFF7C2BA002DACBFFF26002656
:10CC4000FFF7AEBA089B0799013340311A460893A3
:10CC50000B9B07911B689A42BFF63FAB0D99134699
:10CC6000FFF7FFB8309A000838890008099C47F29E
:10CC7000204147F28C426558A058ED1A00F030FA76
:10CC800047F290430D900646E05800F029FA072D30
:10CC90000E9075DC04F5E943196801EBC5026B10D1
:10CCA00047F20C44099DDB002C59002C05947FF7BA
:10CCB000FAAC7F33341D013ADFF808B1CB18039486
:10CCC000041D029204933E4B049F04F1200202993A
:10CCD00007F14008039E01F1080C8E46019200976F
:10CCE000009A043418F8011F043612F8015F0BEBA8
:10CCF00081011EF8010F0BEB85050092D1F8D024BD
:10CD0000D5F8D078D1F8D010D5F8D05C3A44194491
:10CD100003EB22421D4401EB000A02EB0009284408
:10CD20009AF8D8A090F8D80099F8D89006F808ACEE
:10CD300006F8079C06F8060C1CF8010F0244014493
:10CD4000054491F8D80092F8D81095F8D82004F846
:10CD5000080C04F8062C04F8071C019AA242BFD163
:10CD6000039A20320392049A02F580720492029A86
:10CD700002F580720292059A013A0592A4D192E4DA
:10CD8000099B05F0070203F5E943196801EBC202AC
:10CD9000403284E7099B04F0070A03F5E9431A6867
:10CDA00002EBCA0A0AF1800AFFF7C8BA47F27C43CD
:10CDB000099AD05800F094F920600790FFF737B82F
:10CDC000309A0008388900082DE9F04FB84B97B029
:10CDD000834610221B68002112A8984747F240435F
:10CDE0005BF80320002A40F3F48047F24843002117
:10CDF000DFF8C8A218460D9102915BF803300BEBE7
:10CE000000010A91002B40F3DE8047F2744247F2A2
:10CE10002D3100230A985A44994698460C920BEB00
:10CE2000010205930B92029A0390D2010192039B97
:10CE300047F2B83553F8044F03930BEB04070C9BF0
:10CE40002601186800F04CF98446089047F2253016
:10CE5000A30016A9384441F6C2420793CB1890F8B4
:10CE600000E041F6FE410BEB060053F8103C724423
:10CE7000214405444B440BEB82025BF821402968B6
:10CE8000526804910992049A05999342CDF83CC0E6
:10CE90000C4480F2E08047F2BC321258944280F297
:10CEA000DA8047F2C03247F2C431069302440144AB
:10CEB00012680868049200F013F92968069B049A26
:10CEC00001FB0431119002FB01050BEB060147F257
:10CED000783604930E443268934249DA47F27C3242
:10CEE0005258944244DA47F2843001F5E74208444C
:10CEF00012680068069200F0F3F83168049B069A05
:10CF000001FB0434109002FB04F4061931D085B300
:10CF1000015B019A0898674B8418864601987E2227
:10CF20001B682EF80010A91CA01C984762493F22DC
:10CF300002E0013A00F0A78011F8013D34F8133007
:10CF4000002BF6D009995D4801EB4201024433B150
:10CF5000B1F800E010781EFB03F324F810305245BE
:10CF6000A1F1020105D012F8013D34F81330EEE7CB
:10CF700000260F9B13B10FA801F0C4F915B111A839
:10CF800001F0C0F916B110A801F0BCF90B9B029A90
:10CF90001B780132012B02925FD047F21D3309F159
:10CFA00001093B441B78994561D00A9B08F10108AF
:10CFB000019A1B688032434501923FF738AF47F230
:10CFC000404252F80B200D99013191420D91FFF62C
:10CFD00019AF47F22D331BF80320012A70D0002A25
:10CFE00035D047F22E3047F2F83347F22131012A8B
:10CFF0001BF800000BEB80055844EC58405C0444DF
:10D00000EC5024D047F22F30022A1BF800000BEB23
:10D0100080055844EC58405C0444EC5017D047F26B
:10D020003030032A1BF800000BEB80055844EC5805
:10D03000405C0444EC500AD047F231321BF8022025
:10D040000BEB82005A44C458525C2244C250002068
:10D0500017B0BDE8F08F002537E716AA079B1344E9
:10D060001A4653F8103C013342F8103C9DE747F252
:10D070002133059A3B4401321B7805929A4209D02C
:10D080004FF0000991E709990C4801EB4201238810
:10D0900002445CE716AA079B134453F8102C4A4439
:10D0A0004FF0000943F8102CCDF814907DE700BF35
:10D0B000B8030020B40300207889000838890008EC
:10D0C00047F22E3347F2F83100201BF803300BEB08
:10D0D00083035A5801325A5017B0BDE8F08F00BF91
:10D0E000084AD169536B013110B4D16103EBC0041C
:10D0F00013F83020013203F8302060685DF8044BEB
:10D100000830704754A4032047F278432DE9F04FCC
:10D11000804695B0C058FFF7E3FF47F240431290B6
:10D1200058F80330002B40F31E8347F2404400239D
:10D1300047F2344247F23841254647F27444089397
:10D1400047F24840264604931C4608EB0203DFF8EA
:10D15000B894C3460D9308EB0103099308EB000351
:10D160000A9308EB05030E9308EB06030B930D9B44
:10D170001B6823B1099B1B68002B00F06D860A9A7F
:10D180001368002B40F3E282002C40F0DF82049B06
:10D1900005920C93DB010693059B47F232351A4644
:10D1A00052F8043F1C4600930B9B05921868FFF74A
:10D1B00097FF0BEB040347F2253441F6C2421E46AB
:10D1C0000193DBF8243035443444C3F30721139032
:10D1D00095F80080069D247800EB050A4FF4507501
:10D1E000224405FB08110BEB82020BEB8101526814
:10D1F000D1F8BC580292002DC0F2DD824FF450628B
:10D20000DBF8287002FB08B808EB050292F8BC6C4A
:10D21000BF1B002FCBF8287040F3A183C6F1200676
:10D22000F341CBF82430002D40F0A4822946009A27
:10D2300047F2643047F23634129D0BEB820201262E
:10D240001044019A2244144602681144029A016073
:10D25000128812FB01F20499AAF80020695C227876
:10D2600000914FF4507101FB02F84FF4506101FB43
:10D2700002B20192C3F3072242440BEB8202D2F8BE
:10D28000BC48002CC0F22881019A224492F8BC5C70
:10D290007F1B002FCBF8287040F37B81C5F1200263
:10D2A00063FA02F2CBF82420231114F00F0450D0BB
:10D2B000002B00F00B819F193F2F00F34382009A4F
:10D2C000B24240F30481921B9342A8BF1346002B45
:10D2D00000F0FD80721E0020CB4E991809EB02036E
:10D2E000494413F8012F8B422AF81200F9D1DBF8D8
:10D2F00028200123C4F11005DBF82410121BA340E1
:10D3000021FA05F0002A03F1FF35CBF8282005EAC1
:10D31000000540F37B81C4F12003D941CBF82410F0
:10D3200006EB8404236DAB4202DDD4F890301D443B
:10D33000029BF25D33F8173013FB05F52AF8125003
:10D340007E1C402E00F09F80DBF82430DBF8287034
:10D3500090E70F2B40F09780302E00F3F381009B75
:10D36000B34240F3B6809B1B102BA8BF1023002BA9
:10D3700000F0AF8019F80620012B06F101012AF810
:10D38000124000F0A680A04A022B515C06F1020276
:10D390002AF8114000F09D809B49032B895C06F11F
:10D3A00003022AF8114000F094809749042B895C0D
:10D3B00006F104022AF8114000F08B809249052BF7
:10D3C000895C06F105022AF8114000F0828019F804
:10D3D0000200062B4FF0000206F106012AF8102089
:10D3E00077D019F80100072B06F107012AF8102061
:10D3F0006FD019F80100082B06F108012AF8102057
:10D4000067D019F80100092B06F109012AF810204C
:10D410005FD019F801000A2B06F10A012AF8102042
:10D4200057D019F801000B2B06F10B012AF8102038
:10D430004FD019F801000C2B06F10C012AF810202E
:10D4400047D019F801000D2B06F10D012AF8102024
:10D450003FD019F801000E2B06F10E012AF810201A
:10D4600037D019F801100F2B06F10F072AF81120F9
:10D470003FF466AF7E1C19F807300022402E2AF8D0
:10D4800013207FF461AF009BB3420ADD591E731E67
:10D49000002049444B4413F8012F99422AF8120006
:10D4A000F9D1049913A8129B069A5E544B1C803242
:10D4B0001C460493069200F025FF0A9B0C991A68FB
:10D4C000631A9A423FF768AE00243FE137464E4E5A
:10D4D0000DE706F10F0733E7083F002FCBF8287060
:10D4E00040F3CE804FEA3362CBF8242023463946FE
:10D4F0000FE04FEAF272CBF824202B1B43440BEBD6
:10D500008303D3F8BC3D002B3FDADBF82420DBF8A3
:10D51000281001395D42C2F3C0340029CBF828102D
:10D52000E7DCDBF800200DF147015846904770BB5F
:10D530009DF84770FF2F00F0D880DBF800300DF128
:10D5400047015846984710BB9DF84730FF2B00F025
:10D55000DD811904DBF82830DBF82420C3F11F0E2D
:10D56000584262FA0EF203F1200E103392B2CBF859
:10D57000283042EA076747EA010303FA00F023FA7A
:10D580000EF30343CBF82430B7E71C468CE6FF24A8
:10D59000B3E70DF14703584619460393DBF8003013
:10D5A000984700287FF480AE9DF84770DBF8003084
:10D5B000FF2F00F05F8103995846984700287FF4B9
:10D5C00073AE9DF84730FF2B079300F0C782190414
:10D5D000DBF82800DBF824202B18C0F1000E00F146
:10D5E00020051030C3F12003CBF8280062FA03F3C2
:10D5F0009BB243EA0763194301FA0EF3E9400B4378
:10D60000CBF8243050E600BF388900080DF14703FD
:10D61000584619460393DBF80030984770BB9DF8D5
:10D620004730FF2B0793DBF8003000F04881039967
:10D630005846984710BB9DF84720FF2A00F01184F8
:10D640001004DBF82820DBF8243004EB020E5142F2
:10D6500002F1200C1032CEF1200ECBF8282063FA14
:10D660000EF3079A9BB243EA0263034303FA01F104
:10D6700023FA0CF30B43CBF8243051E6FF254FE699
:10D680000DF14703584619460393DBF800309847DD
:10D69000002852D19DF84730FF2B0793DBF800306C
:10D6A00000F09281039958469847002845D19DF88B
:10D6B0004750FF2D00F026832904DBF82830DBF8E3
:10D6C0002420C3F11805584203F11007EA4103F181
:10D6D0002005079B92B242EA0362114301FA00F26D
:10D6E000E9400A43CBF8242000E7DBF800200DF1E5
:10D6F00047015846904700287FF449AF9DF84700FE
:10D7000000283FF41AAF9BF82120042A3FF415AFFC
:10D71000531C0BEB0201DBB28BF82130042B487752
:10D72000C349CBF8001000F09482911C0BEB03026C
:10D73000BF4B8BF82110577701E7DBF82420DBF88B
:10D740002870D3E613A8012400F0DCFD089A09989C
:10D7500001320368114608920E9A013B1268036079
:10D760008A423FF704AD12A800F0CCFD002015B0AE
:10D77000BDE8F08F0122C5F110017F1BAA4023FAFA
:10D7800001F1002FCBF8287002F1FF3201EA02020A
:10D79000039240F384811146C5F12002D341CBF8B6
:10D7A000243009EB85052A6D8A427FF740ADD5F814
:10D7B000905029443BE5DBF82870083F002FCBF858
:10D7C000287040F337814FEA3363CBF824304FF4AD
:10D7D000507202FB08F80DE04FEAF3732246CBF8D3
:10D7E0002430B21A42440BEB8202D2F8BC5D002D09
:10D7F000BFF619AD013F6E42C3F3C034002FCBF822
:10D800002870E9DCDBF800300DF1470158469847F5
:10D8100050BB9DF84750FF2D00F07981DBF8007078
:10D820000DF147015846B847F0B99DF84770FF2FF2
:10D8300000F08E823B04DBF828702246DBF82410CF
:10D84000C7F11F047842E14107F12004103789B283
:10D85000CBF8287041EA05652B4303FA00F0E3405A
:10D860000343CBF82430BCE7DBF82430FF22DBF89D
:10D870002870B6E703995846984700287FF414ADFE
:10D880009DF84700002800F0C6809BF82120042A5C
:10D8900000F0C180531C0BEB0201DBB28BF821308E
:10D8A000042B48776249CBF8001000F024820BEB80
:10D8B000030102325E4B8BF821204F777BE6039900
:10D8C0005846984700287FF4D9AE9DF847000028B5
:10D8D00000F06D819BF82120042A00F06881531C20
:10D8E0000BEB0201DBB28BF82130042B4877504957
:10D8F000CBF8001000F0EB8202320BEB03014C4B33
:10D900008BF821209DF81C204A7790E6DBF8002058
:10D910000DF14701584603939047039B00287FF47D
:10D9200036AE9DF847E0BEF1000F7DD09BF8211088
:10D93000042979D04A1C0BEB0100D2B28BF82120CC
:10D94000042A80F81DE03A48CBF800006CD0881C0F
:10D950005A444FF47F018BF821005377FAE50DF11B
:10D960004704DBF80030584621469847002855D137
:10D970009DF84780DBF80030B8F1FF0F00F0998187
:10D98000214658469847002848D19DF84770FF2FF8
:10D9900000F061813904DBF82870DBF82430F219DB
:10D9A000784207F120041037C2F12002CBF828702A
:10D9B000D3419BB243EA08630B4303FA00F0E34010
:10D9C0000343CBF824302EE40399584698470028A7
:10D9D0007FF4B3AE9DF84700002800F074829BF8F6
:10D9E0002120042A00F06F82531C0BEB0201DBB2F2
:10D9F0008BF82130042B48770D49CBF8001000F04C
:10DA00005F8202320BEB0301094B8BF821209DF85A
:10DA10001C204A7746E6DBF80030CCE5DBF8243002
:10DA2000DBF82870FFF7FFBB4FF47F0192E500BFE2
:10DA300099A405080DF14704DBF80030584621464B
:10DA40009847002840F000819DF84730FF2B039352
:10DA5000DBF8003000F0D180214658469847002876
:10DA600040F0F2809DF84760FF2E00F0A380320462
:10DA7000DBF82870DBF82430C7F11800039C7942EA
:10DA8000C34107F1200010379BB243EA04631343FC
:10DA900003FA01F1C3400B43CBF8243097E60DF1B4
:10DAA0004704DBF80030584621469847002840F0EC
:10DAB0009B819DF84780DBF80030B8F1FF0F00F044
:10DAC0006D81214658469847002840F08D819DF889
:10DAD0004760FF2E00F08E813004DBF82870DBF801
:10DAE0002430EC197A4207F120061037C4F12004E3
:10DAF0000399CBF82870E3419BB243EA08630343E0
:10DB000003FA02F2F3401343CBF8243049E6DBF882
:10DB100000300DF147015846984700287FF4A4AE25
:10DB20009DF8470000283FF479AE9BF82120042A95
:10DB30003FF474AE531C0BEB0201DBB28BF82130C7
:10DB4000042B4877C349CBF8001000F0B3810232B0
:10DB50005B440F468BF821205D7761E603995846B8
:10DB6000DBF80030984700287FF49EAB9DF8470013
:10DB7000002800F0AF819BF82120042A00F0AA8140
:10DB8000531C0BEB0201DBB28BF82130042B4877DE
:10DB9000B049CBF8001000F09D8102325B444FF495
:10DBA0007F018BF821209DF81C205A7710E5DBF8C7
:10DBB00000303CE52146DBF8003058469847002805
:10DBC00042D19DF8470000286DD09BF82110042910
:10DBD00069D04B1C0BEB0102DBB28BF82130042B1C
:10DBE00050779C4ACBF800205DD002315B444FF463
:10DBF0007F028BF821105E773AE721465846984716
:10DC000010BB9DF8470000284AD09BF82120042A29
:10DC100046D0531C0BEB0201DBB28BF82130042BF6
:10DC200048778C49CBF8001038D002320BEB030157
:10DC30005846884B8BF821209DF80C204A772146C6
:10DC4000984700283FF40EAFDBF82430DBF828704B
:10DC5000BDE5804B73E42146DBF800305846984719
:10DC600000287FF4DBAE9DF84700F8B19BF8212037
:10DC7000042A1BD0531C0BEB0201DBB28BF82130C2
:10DC8000042B48777349CBF800100FD002325B4465
:10DC90004FF47F018BF821205F777CE66D4BDBE64C
:10DCA000DBF80030D8E64FF47F02E1E64FF47F0165
:10DCB00071E621465846984700287FF4AFAE9DF89C
:10DCC0004700E0B19BF82120042A18D0531C0BEB2D
:10DCD0000201DBB28BF82130042B48775D49CBF889
:10DCE00000100AD00BEB030102325A4B8BF82120B3
:10DCF00081F81D8044E6574B5DE4564B40E6DBF867
:10DD000000303DE603995846DBF80030984700287C
:10DD10007FF413AD9DF84700002800F08D809BF83C
:10DD20002120042A00F08880531C0BEB0201DBB297
:10DD30008BF82130042B48774649CBF800107BD074
:10DD400002325B444FF47F018BF821205D77B4E40D
:10DD5000DBF800300DF147015846984700287FF462
:10DD600083AD9DF8470000286CD09BF82120042A41
:10DD700068D0531C0BEB0201DBB28BF82130042B73
:10DD800048773449CBF800105CD0911C0BEB0302B0
:10DD90004FF47F038BF8211057774CE52146584606
:10DDA000984708BB9DF84700002850D09BF82120D9
:10DDB000042A4CD0531C0BEB0201DBB28BF8213050
:10DDC000042B48772349CBF800103ED00BEB03011E
:10DDD0000232204B58468BF8212081F81D802146C5
:10DDE000984700283FF473AEDBF82430FF21DBF8BE
:10DDF0002870D6E42146DBF80030584698470028C2
:10DE0000F2D19DF84700D0B19BF82120042A16D00A
:10DE1000531C0BEB0201DBB28BF82130042B48774B
:10DE20000C49CBF800100AD002325B444FF47F005B
:10DE30008BF821205E7750E64FF47F013DE44FF4EC
:10DE40007F004AE64FF47F03F5E4024B39E6DBF846
:10DE5000003036E699A40508584600F06DFAFFF741
:10DE60008EB903995846DBF800300F9298470F9A05
:10DE700000287FF403AC9DF847E0BEF1000F1BD0F3
:10DE80009BF82110042917D04B1C0BEB0100DBB2CF
:10DE90008BF82130042B80F81DE01048CBF80000EF
:10DEA0000AD002315B444FF47F008BF821105A777F
:10DEB000FFF7C7BB094FB3E44FF47F00FFF7C1BBC7
:10DEC000064BFFF7EFBBDBF80030FFF7EBBB034B74
:10DED000FFF7ADBB4FF47F01FFF77ABB99A40508AC
:10DEE0002DE9F04F044683B00D460026236801A9B2
:10DEF0002046984718B113E02368984780B99DF8E9
:10DF0000043001A92046FF2BF6D103E09DF8043030
:10DF1000FF2B09D1236801A9204698470028F5D096
:10DF2000012003B0BDE8F08F002BDFD0CC2B2B708D
:10DF3000F6D04AD9DA2B40F21381DD2B00F017819D
:10DF4000EE2B00F0B980DB2B00F0438123680DF14C
:10DF50000301204698470028C8D1236801A920461C
:10DF600098470028C2D19DF803809DF8043043EA09
:10DF70000828A8F10208B8F1000FB7DDA2699045A2
:10DF80004FF000031ADD217FC2EB0808002940F0A2
:10DF90007481E36867684FF4805201A9A068B847AC
:10DFA000002800F06D81E3680246A06190451844A6
:10DFB000019BE06063614FF00003E4DC6369C8EB40
:10DFC00002024344A261636190E7C72B00F24F81D4
:10DFD000C52BA6D2C32B40F2BC800DF103072368EA
:10DFE00020463946984700289AD1236801A920463F
:10DFF0009847002894D19DF803909DF8043043EA97
:10E000000929A9F10209B9F1100F7FF76FAF236851
:10E0100001A920469847002882D19DF80420C2F328
:10E02000001302F00F0202EB8303072B8DF804307C
:10E030003FF676AF03EB03124FF001012344804615
:10E0400002F1300A224483F82C10A24482F83400F2
:10E050000AF1050B0AF1150A226839462046904755
:10E0600000287FF45DAF9DF803200BF8012BD3450A
:10E070009044F1D1B8F1FF0FA9F111093FF750AF6A
:10E08000C8453FF74DAF9DF8043004EB0323BC3384
:10E09000B8F1000F00F0218103EB080A02E0D3453C
:10E0A00000F01B8103F1010B1946226820469047BE
:10E0B0005B460028F3D033E723680DF103012046C7
:10E0C000984700287FF42CAF236801A92046984781
:10E0D00000287FF425AF9DF803209DF8043043EA23
:10E0E00002230D2B7FF71CAFA2694FF00B08904560
:10E0F0004FF000031ADD217FC2EB0808002940F031
:10E10000C480E36867684FF4805201A9A068B847EB
:10E11000002800F0BD80E3680246A06190451844E5
:10E12000019BE06063614FF00003E4DC6769C8EBCA
:10E130000202236801A94744A2612046676198470B
:10E1400000287FF4EDAE9DF80430012B7FF4E8AE9B
:10E15000CCE6C02BBFF4E5AE012B3FF4E1AEF5E613
:10E16000D82BBFF4DEAECF2B3FF6DAAED9E60DF1F9
:10E170000307236820463946984700287FF4D0AE2D
:10E18000236801A92046984700287FF4C9AE9DF86E
:10E1900003209DF8043043EA0223042B7FF4C0AE31
:10E1A000394623682046984700287FF4B9AE236893
:10E1B00001A92046984700287FF4B2AE47F23443C5
:10E1C0009DF803109DF80420234442EA01221A60BE
:10E1D0008CE60DF10307236820463946984700284E
:10E1E0007FF49EAE236801A92046984700287FF45B
:10E1F00097AE9DF803A09DF8043043EA0A2AAAF1DD
:10E20000020ABAF1000F75DD23680DF10201204604
:10E21000984700287FF484AE9DF8023003F00F0188
:10E220001A0903298DF802103FF67AAE04EBC110EB
:10E2300047F2081941F6C24381440B4409F104082E
:10E2400004EB8303C3F804803ABB09F1020809F127
:10E25000820905E09DF8043028F8023FC84546D001
:10E26000236801A9204698470028F3D058E6C82B18
:10E270003FF456AE03B0BDE8F08FE660267789E63E
:10E28000A269002A7FF47BAE30E6E660267739E7A4
:10E29000A269002A7FF42BAF42E6DFF864B00BF1ED
:10E2A000400912E0236801A92046984700287FF41E
:10E2B00037AE1BF8012F9DF803109DF80430D945A7
:10E2C00043EA012328F812300ED02368394620464D
:10E2D000984700287FF424AEE4E7C8EB0909B9F1B8
:10E2E000100F3FF794AE01E6AAF1810A89E7AAF17F
:10E2F000410A86E7BAF1000F3FF4F8AD10E600BF1F
:10E300003789000803680B4A30B4044653F8085CA8
:10E31000506B10F83530012B03D9D16909B101399F
:10E32000D1610022013B00F835301046226030BC3C
:10E33000704700BF54A40320F0B5054683B04FF4E6
:10E34000FA6405E09DF80730FF2B0DD0013C07D0A3
:10E350002B680DF107012846264698470028F1D082
:10E360000124204603B0F0BD2B680DF107012846BB
:10E37000984704460028F3D19DF80730FF2B02D1BF
:10E38000013EF1D1ECE747F23C46AA59D032934224
:10E39000E6D147F21C32114B47F264302146AA5CA9
:10E3A00010271B68284492009847AB5947F2344124
:10E3B00047F23842013347F23040695803F007030F
:10E3C0002C50A95028463946AB51AF6200F008F8EE
:10E3D0003946284600F004F8C3E700BFB803002020
:10E3E0002DE9F0410123846AC1F11005466A641ADF
:10E3F0008B4026FA05F582B0013B002C0246846270
:10E4000005EA030508DDC1F12001284666FA01F19D
:10E41000516202B0BDE8F0810C4603680DF10701BE
:10E420000646984728BB9DF807803368B8F1FF0F70
:10E4300021D00DF1070130469847D0B99DF80770FB
:10E44000FF2F38D0B16A2846726A631801F120059F
:10E450004C421031C3F12003B162DA4192B242EA78
:10E46000086242EA074303FA04F4EB402343736271
:10E47000CFE7FF20CDE70DF1070130469847002890
:10E48000F7D19DF80700A0B196F82110042910D00B
:10E490004A1C7718184BD2B2042A86F821207877C4
:10E4A0003360C6D00231324486F8211082F81D80D4
:10E4B000BFE73368BDE70DF1070133683046984781
:10E4C0000028D6D19DF807000028BBD096F821205F
:10E4D000042AB7D0531CB118DFF81CE0DBB2042BC0
:10E4E00086F821304877C6F800E0ABD002323344DA
:10E4F00086F821205F77A5E799A405080101000DA2
:10E500000400000048F30508020A010304000000AB
:10E5100098E805080304010306000000D8EB05088D
:10E52000070900040800000084970508060C010292
:10E5300008000000A89705080A0A00030B00000065
:10E5400090490508090A01030A000000C4490508AA
:10E55000020401030300000044F00508050D010357
:10E560000600000080920508050D0003060000006B
:10E57000A8920508050602030800000080CF0508E0
:10E580000706010708000000CCC405080303000BC0
:10E590000400000010EE050804020008040000005A
:10E5A00048F005080202010B04000000D0F2050843
:10E5B000060B010307000000DCA50508070A00039D
:10E5C0000800000090780508040A01030800000014
:10E5D00084CB0508060A01030800000098AC050872
:10E5E000070A000308000000B8780508070A0003BE
:10E5F00008000000E0780508070A00030800000092
:10E6000008790508070A00030800000030790508AA
:10E61000060A010308000000B8AC0508070A000359
:10E620000800000058790508070A000308000000E8
:10E63000807905080207010604000000D8ED0508EE
:10E640000308000604000000B0D105080707010612
:10E650000800000084B9050807050107080000004C
:10E6600098CB05080707010608000000A0B90508B7
:10E67000070A000308000000A8790508090A00033A
:10E680000A000000F84905080A0A00030A00000011
:10E690002C4A0508070A010308000000D079050884
:10E6A0000A0A00030B000000604A0508080A01037B
:10E6B0000A000000F8790508060A010307000000B7
:10E6C000D8AC0508050A010306000000F8AC0508EF
:10E6D0000A0A00030B000000944A0508070A010318
:10E6E00009000000207A0508020A01030400000066
:10E6F000A4E80508060A00030700000018AD050895
:10E70000080A010309000000487A0508050A010308
:10E710000600000038AD05080A0A01030C000000DD
:10E72000C84A0508080A01030A000000707A0508B3
:10E730000A0A00030B000000FC4A0508070A01034F
:10E7400008000000987A05080A0A01030B0000007F
:10E75000304B0508070A010308000000C07A0508CD
:10E76000070A000307000000E87A0508060A00030C
:10E770000600000058AD0508070A01030900000063
:10E78000107B0508090A000309000000644B050816
:10E790000C0A00030C0000009C1C0508090A000379
:10E7A00009000000984B0508080A00030800000053
:10E7B000387B0508060A00030600000078AD05084E
:10E7C000040D01030600000060C20508060B0103EA
:10E7D0000700000000A60508040D01030600000064
:10E7E0007CC20508060501030800000080D3050867
:10E7F0000701000E070000004CF0050804030102A9
:10E800000700000018EE05080807000609000000D0
:10E81000BCB90508070A010309000000607B050870
:10E820000807000608000000D8B90508080A000318
:10E8300009000000887B05080807000608000000A2
:10E84000F4B90508040A000304000000ACCB050875
:10E85000080A000609000000B07B0508060A01034B
:10E860000800000098AD0508020A0103030000003B
:10E87000B0E80508030D00030400000098C2050875
:10E88000060A010307000000B8AD0508020A0103EB
:10E8900003000000BCE805080B0701060D0000009E
:10E8A0002876050806070106080000007CC905084F
:10E8B000080700060900000010BA0508070A01064B
:10E8C00009000000D87B0508080A000609000000BE
:10E8D000007C0508040701060500000090D4050827
:10E8E0000707FF06060000002CBA0508050AFF030B
:10E8F00004000000D8AD0508060701060800000066
:10E9000094C90508070700060700000048BA050873
:10E910000B0700060B0000005476050808070006E8
:10E920000700000064BA0508070A00060700000097
:10E93000287C05080507000606000000ACC905088C
:10E94000050D010307000000D0920508020D030326
:10E9500007000000D0D50508050D000307000000E2
:10E96000F89205080603010808000000A8EA050857
:10E970000101000D040000004CF30508020A010625
:10E9800004000000C8E805080609010408000000AA
:10E9900068C00508090AFF0308000000CC4B050801
:10E9A0000908FF0508000000507C0508080A00035C
:10E9B00008000000787C0508020B03040700000033
:10E9C00050E80508070D000308000000A8420508EC
:10E9D000050201030700000020EE05080A0A0003F3
:10E9E0000A000000004C05080404000305000000B4
:10E9F000E0EB0508050500070500000090D30508B9
:10EA00000704000708000000C0D105080402000840
:10EA10000400000050F005080A0A00030A00000084
:10EA2000344C0508050201040700000028EE050823
:10EA30000304010405000000E8EB050807080106CF
:10EA40000800000098A9050804060003050000005E
:10EA500070E605080506FF030500000094CF0508D1
:10EA6000040302020700000030EE0508060A010652
:10EA700008000000F8AD0508070B000309000000BE
:10EA8000206A05080202010904000000D4F205080A
:10EA90000304020C07000000F0EB05080306010365
:10EAA000050000007CE605080504000305000000E1
:10EAB00088E605080505000705000000A0D3050845
:10EAC000090A01030B000000684C0508090A01034C
:10EAD0000B0000009C4C05080C0A00030C00000011
:10EAE000D81C0508060A01060800000018AE050833
:10EAF0000A0D00000A0000003C0F05080A0D000086
:10EB00000A000000800F05080A0C00010A0000003E
:10EB1000141D05080A0C00010A000000501D05081C
:10EB20000B0CFF010A00000058F60408090D000054
:10EB30000A000000C40F05080D0AFF030D000000C5
:10EB4000480305080B0D00030B000000CCEB040884
:10EB5000060D01000700000020930508060D0100C6
:10EB60000700000048930508070C0001070000009B
:10EB700090570508060C010107000000CC97050816
:10EB8000050DFF000400000070930508050D00004E
:10EB90000400000098930508060CFF010400000023
:10EBA000F0970508050CFF01040000001498050803
:10EBB000090A00030A000000D04C0508080C0101F6
:10EBC0000A000000C05705080A0D00000B000000F5
:10EBD000081005080A0D00000B0000004C10050885
:10EBE0000A0C00010B0000008C1D05080A0C000136
:10EBF0000B000000C81D05080A0C00010B000000F6
:10EC0000041E0508070701060800000080BA050871
:10EC10000A0C00020B000000401E0508070D010051
:10EC200009000000DC420508070D01000900000092
:10EC300010430508070C010109000000F057050802
:10EC4000070C01010900000020580508080D00000C
:10EC50000800000044430508070A010308000000FB
:10EC6000A07C0508070A010309000000C87C05080C
:10EC7000080B0002090000004C6A0508080B00029E
:10EC800009000000786A0508080A0003090000006E
:10EC9000F07C0508080A000309000000187D05083B
:10ECA000080A000309000000407D0508080B000267
:10ECB00009000000A46A05080E0700060E00000007
:10ECC00088540508080A000608000000687D050849
:10ECD000080B000208000000D06A0508080B0002BB
:10ECE00008000000FC6A0508080A0003080000008C
:10ECF000907D0508080A000308000000B87D05089B
:10ED0000050BFF020300000024A60508040B000207
:10ED100003000000B4C70508060AFF030300000053
:10ED200038AE0508050AFF030300000058AE0508C9
:10ED3000080A000309000000E07D0508060A010337
:10ED40000800000078AE0508080B0002090000006A
:10ED5000286B0508080B000209000000546B050829
:10ED6000080A000309000000087E0508080A0003DD
:10ED700009000000307E0508080A000309000000B1
:10ED8000587E05080708010608000000B8A9050814
:10ED9000080900050900000038980508060B010263
:10EDA0000800000048A60508060B01020800000044
:10EDB0006CA60508060A01030800000098AE0508C5
:10EDC000060A010308000000B8AE0508070E00029D
:10EDD0000700000058330508070D01030900000073
:10EDE00078430508090DFF0307000000901005088F
:10EDF0000207010603000000E0ED0508060A000313
:10EE000006000000D8AE0508040A00030400000054
:10EE1000C0CB05080E0A00030E0000009003050891
:10EE20000E0700060E000000BC540508070C000188
:10EE30000700000050580508070AFF0306000000FD
:10EE4000807E0508080C00010800000080580508B5
:10EE5000060C0001060000005C980508060A000385
:10EE600006000000F8AE0508070D000308000000CA
:10EE7000AC430508060201030700000038EE050850
:10EE8000060201030700000040EE05080502010428
:10EE90000700000048EE0508050301030700000015
:10EEA000B4EA05080202030307000000D8F20508CF
:10EEB0000304020207000000F8EB05080303020D3B
:10EEC0000700000050EE05080503010307000000DD
:10EED000C0EA05080603010207000000CCEA0508A5
:10EEE0000A0A00030A000000044D0508060A01068C
:10EEF0000800000018AF05080A07FF060800000018
:10EF0000BCA40508040200080400000054F0050831
:10EF1000060201080700000058EE05080C02000870
:10EF20000D00000094E6050803030103040000003F
:10EF300060EE0508030301030400000068EE050805
:10EF40000303010B0400000070EE05080503020333
:10EF500007000000D8EA05080503010307000000C8
:10EF6000E4EA05080503010B07000000F0EA0508C4
:10EF7000060D010308000000C0930508060D0103FB
:10EF800008000000E89305080404030708000000D7
:10EF900000EC05080B02010B0D000000A0E60508BF
:10EFA0000F0A000310000000ACE804080305000786
:10EFB00003000000D4E80508030500070300000073
:10EFC000E0E80508060AFF030200000038AF050864
:10EFD000080AFF0307000000A87E0508070A0003CF
:10EFE00007000000D07E05080C06FF030D0000009E
:10EFF000809805080A0A00030A000000384D050839
:10F000000B0A00030C0000007C1E0508070A000321
:10F0100008000000F87E0508090A00030900000046
:10F020006C4D05080A0B00030A000000283805088B
:10F03000070C000308000000B0580508070201098A
:10F040000800000008EC0508060AFF0302000000A3
:10F0500058AF05080202010904000000DCF20508AF
:10F06000080D000208000000E0430508090401073C
:10F070000B000000D4CB0508050D000205000000C0
:10F08000109405080704010708000000D0D1050806
:10F090000708010508000000D8A9050806090104B1
:10F0A0000800000084C005080609010408000000EB
:10F0B000A0C00508070B010308000000806B0508CD
:10F0C000060A00030700000078AF0508060A0003DF
:10F0D0000700000098AF05080709000407000000BA
:10F0E000A49805080101000C0400000050F3050875
:10F0F000010A010204000000ECE805080304010213
:10F100000500000010EC0508070A000207000000D7
:10F11000207F0508060C000107000000C8980508BC
:10F120000A0A00020A000000A04D0508080A0102B0
:10F130000A000000487F05080104010203000000E6
:10F1400058F00508040E0102060000009CBA0508EC
:10F15000040E000206000000B8BA05080505010209
:10F1600008000000B0D305080707000508000000EC
:10F17000D4BA05080203000A0400000060F2050882
:10F180000401000804000000E0F205080102010A81
:10F1900004000000E4F20508060B0102070000006D
:10F1A00090A60508060A010207000000B8AF05088E
:10F1B000030A010207000000E8CB0508060A010265
:10F1C00007000000D8AF0508070A0002070000008A
:10F1D000707F0508070A000207000000987F0508F5
:10F1E000070A000207000000C07F0508070A0002A6
:10F1F00007000000E87F0508060A0102070000007A
:10F20000F8AF0508060A01020700000018B005085B
:10F21000070A000207000000108005080107010529
:10F2200004000000E8ED05080208000504000000E5
:10F2300018EC05080707010508000000F0BA0508EA
:10F240000704010708000000E0D1050807070105D1
:10F25000080000000CBB0508050A010207000000B9
:10F2600038B005080A0A00020A000000D44D05085B
:10F27000090A000209000000084E0508060A0102FA
:10F280000700000058B005080A0A01020A00000041
:10F290003C4E0508080A01020900000038800508F4
:10F2A000060A01020700000078B00508050A0102FD
:10F2B0000600000098B005080A0A01020B000000D1
:10F2C000704E0508070A0102090000006080050869
:10F2D000010A010203000000F8E80508050A00021F
:10F2E00006000000B8B00508070A01020800000087
:10F2F00088800508050A010206000000D8B005084C
:10F300000A0A01020C000000A44E0508080A0102C6
:10F310000A000000B0800508090A01020B00000085
:10F32000D84E0508060A010207000000F8B00508DB
:10F330000B0A01020B000000B81E0508060A0102B4
:10F340000800000018B10508050A010207000000C6
:10F3500038B10508070AFF0206000000D88005083A
:10F36000060A01020800000058B10508090A000257
:10F37000090000000C4F05080C0A00020C000000F8
:10F38000F41E0508080A00020800000000810508B4
:10F39000070A00020800000028810508070A000289
:10F3A0000600000050810508040D0202060000005E
:10F3B000B4C20508060B010207000000B4A6050848
:10F3C000040D000206000000D0C205080605010277
:10F3D00008000000C0D305080701000D0700000069
:10F3E0005CF00508040302020700000078EE05083F
:10F3F000080700050900000028BB0508070A0102EC
:10F4000009000000788105080807000508000000D1
:10F4100044BB0508080A000209000000A081050895
:10F42000080700050800000060BB0508040A000288
:10F4300004000000FCCB0508080A000509000000D4
:10F44000C8810508060A01020800000078B1050815
:10F45000010A01020300000004E90508030DFF0290
:10F4600003000000ECC20508060A010207000000C4
:10F4700098B10508010A01020300000010E905081F
:10F480000A0701050C000000E0A4050806070105B5
:10F4900008000000C4C905080807000508000000AE
:10F4A0007CBB0508070A010509000000F08105087A
:10F4B000080A000509000000188205080407010574
:10F4C00004000000A0D405080507000506000000A0
:10F4D000DCC90508050AFF0204000000B8B10508F0
:10F4E0000607010508000000F4C905080707000524
:10F4F0000700000098BB05080A0700050A00000085
:10F5000004A5050806070005060000000CCA05084A
:10F51000070A0005070000004082050805070005EE
:10F520000500000024CA0508040D020206000000C0
:10F5300008C30508010D030207000000E0D5050817
:10F54000040D01020600000024C30508060201089C
:10F550000800000080EE05080101000C0400000016
:10F5600054F305080109010504000000FCEA050840
:10F570000608010307000000E4C40508070A0002AA
:10F580000700000068820508080800040700000062
:10F59000F8A90508070A0002070000009082050884
:10F5A000010B0303070000005CE80508060D0102DB
:10F5B000080000003894050803020202070000005A
:10F5C00060F005080A0A00020A000000404F050822
:10F5D0000504000205000000ACE60508040500066D
:10F5E000050000001CE905080704000708000000EA
:10F5F000F0D105080401000804000000E8F2050845
:10F600000A0A00020A000000744F05080501010300
:10F610000700000064F20508040301030500000070
:10F6200088EE0508070800040800000018AA05086D
:10F630000306010205000000B8E605080406000202
:10F6400005000000C4E605080403020207000000EC
:10F6500090EE0508060A010508000000D8B105086B
:10F66000070B000208000000AC6B0508010201074F
:10F6700004000000ECF205080304020B0700000080
:10F6800020EC05080306000205000000D0E605088E
:10F69000040401020500000028EC0508040500062A
:10F6A0000500000028E905080A0A00020A00000017
:10F6B000A84F05080A0A00020A000000DC4F0508EE
:10F6C0000A0A01020B00000010500508060A010595
:10F6D00007000000F8B10508090C0000090000004F
:10F6E000301F0508090C0000090000006C1F050808
:10F6F000090C000009000000A81F0508090C000003
:10F7000009000000E41F0508090C000009000000C2
:10F7100020200508090C0000090000005C200508F5
:10F720000C0A00020C000000982005080A0D0102D6
:10F730000A000000D4100508060C010007000000B4
:10F74000EC980508060C0100070000001099050858
:10F75000060C01000700000034990508050C0100A3
:10F760000700000058990508040CFF000300000082
:10F77000FCC40508040C00000300000014C50508C3
:10F78000050CFF00030000007C990508030C000035
:10F79000030000002CC50508090A0002090000004A
:10F7A00044500508080C01000A000000E058050854
:10F7B000090C01000B000000D4200508090C010011
:10F7C0000B00000010210508090C01000B000000CF
:10F7D0004C210508090C01000B00000088210508D8
:10F7E000090C01000B000000C421050807070105F2
:10F7F00008000000B4BB0508090C01010B00000063
:10F8000000220508060C010008000000A099050868
:10F81000060C010008000000C4990508060C010050
:10F8200008000000E8990508060C01000800000027
:10F830000C9A0508070C0000080000001059050884
:10F84000060A01020700000018B20508060A0102B4
:10F850000800000038B20508080A0002090000008C
:10F86000B8820508080A000209000000E0820508C5
:10F87000080A00020900000008830508080A0002BF
:10F880000900000030830508080A00020900000092
:10F8900058830508080A0002090000008083050853
:10F8A0000E0700050F000000F0540508080A0005C7
:10F8B00008000000A8830508080A000208000000EC
:10F8C000D0830508080A000208000000F883050834
:10F8D000080A00020800000020840508080A000247
:10F8E0000800000048840508040AFF020300000025
:10F8F00010CC0508040B000103000000CCC705086C
:10F90000060AFE020300000058B20508030A0002BE
:10F910000300000024CC0508080A000208000000CB
:10F9200070840508060A01020800000078B2050884
:10F93000080A00020800000098840508080A00026E
:10F9400008000000C0840508080A00020800000042
:10F95000E8840508080A0002080000001085050870
:10F96000080A00020800000038850508070700059E
:10F9700008000000D0BB05080809000408000000CA
:10F98000309A0508060A01020800000098B205082E
:10F99000060B010108000000D8A60508060A0102AE
:10F9A00008000000B8B20508060A010208000000BD
:10F9B000D8B20508070E00010700000090330508C3
:10F9C000070D01020900000014440508070D00029C
:10F9D0000700000048440508010701050300000076
:10F9E000F0ED0508060A000206000000F8B205085E
:10F9F000040A00020300000038CC05080D0A0102C9
:10FA00000F000000D80305080E0700050F000000D6
:10FA100024550508050C010007000000549A05084C
:10FA2000060A00020600000018B30508070C0000D3
:10FA30000800000040590508070C000006000000FF
:10FA400070590508060A00020500000038B30508D1
:10FA5000070D0002070000007C44050806020102B1
:10FA60000700000098EE05080602010207000000EA
:10FA7000A0EE0508050101030700000068F2050873
:10FA80000502010207000000A8EE050801020302BA
:10FA900007000000F0F2050803030202070000005F
:10FAA000B0EE05080303020C07000000B8EE0508DD
:10FAB000050301020700000008EB0508050301012A
:10FAC0000700000014EB05080A0A00020A00000003
:10FAD00078500508060A01050800000058B305081B
:10FAE0000807000508000000ECBB05080401000839
:10FAF00004000000F4F205080601000807000000F9
:10FB00006CF205080C0100080D000000C0EE0508AD
:10FB1000020301020400000070F205080203010262
:10FB20000400000074F205080203010A040000004A
:10FB300078F205080403020206000000C8EE05087A
:10FB40000403010206000000D0EE05080403010AC8
:10FB500006000000D8EE0508070C000208000000AF
:10FB6000A0590508070C000208000000D05905083C
:10FB70000303020606000000E0EE05080902020A7F
:10FB80000D00000034E905080E0A00020F00000015
:10FB900020040508030501060300000040E90508EC
:10FBA00003050106030000004CE90508050AFE02F2
:10FBB0000200000078B30508080AFF0207000000F1
:10FBC00060850508060B000107000000FCA605087B
:10FBD0000B0600020D000000789A05080A0A0002D0
:10FBE0000A000000AC5005080B0A00020C000000DF
:10FBF0003C220508060B01010700000020A70508AC
:10FC0000080A000209000000888505080A0B0002A6
:10FC10000900000060380508070B0002070000001B
:10FC2000D86B0508070101080800000064F005080A
:10FC3000050AFE020200000098B305080102010750
:10FC400004000000F8F20508080E0100080000009A
:10FC5000C8330508090501050B00000004C40508A8
:10FC6000050E000005000000807605080705010567
:10FC7000080000004CCC050807070105080000003B
:10FC800008BC0508060801040800000044C5050872
:10FC9000070800040800000038AA0508070B010245
:10FCA00008000000046C0508050A000206000000B8
:10FCB000B8B30508050A000206000000D8B305081D
:10FCC00007090003070000009C9A050801010019BC
:10FCD0000700000058F305080214030507000000A0
:10FCE00060CC0508060802050A0000005CC505088E
:10FCF0000E1100070F000000E4A704080B17020410
:10FD00000F000000B0870408121401051400000061
:10FD1000D42D04081214010513000000882E0408D5
:10FD2000020802050600000030EC0508081B020569
:10FD30000B000000B4B90408081B01050B0000000B
:10FD400020BA040809090305100000001062050824
:10FD50000E0D010C1000000038D504080405011632
:10FD60000800000058E9050807020011070000001C
:10FD700038EC050802030316080000007CF20508B1
:10FD80000B1602050E000000F09304080D14010587
:10FD90000F000000907A0408061403050F0000000D
:10FDA000782205080D1401050F0000001C7B0408D3
:10FDB0000D1400050F000000A87B04080E140005B8
:10FDC0000F000000347C04080E1400050F00000032
:10FDD000C07C04080D1401050F0000004C7D0408D0
:10FDE0000B1402050F0000000C9E04080D14010501
:10FDF0000F000000D87D04080D1401050F0000005D
:10FE0000647E0408020E030B08000000B0D405084D
:10FE10000410010B0800000058AA05080D0E010B84
:10FE20001000000038CA04080D07010F1000000080
:10FE3000585505080D0E010B100000009CCA04085F
:10FE40000C1401050E000000849E04081214010524
:10FE5000140000003C2F04081214000512000000DA
:10FE6000F02F04080C1402050F000000FC9E04088B
:10FE70001314010515000000700C04080F1402058E
:10FE800013000000005304080B1402050E000000CC
:10FE9000749F04080A1402050D000000F8C304084A
:10FEA0001514010516000000DCF603080D14020508
:10FEB00011000000F07E0408021402050600000094
:10FEC00074CC05080B1400050D000000EC9F04081D
:10FED0000D1402050F0000007C7F04080A140205BF
:10FEE0000C0000005CC40408141402051800000093
:10FEF000380D04080F14020513000000A053040875
:10FF00001414010516000000000E04080C1402056C
:10FF10000E00000064A0040816140105170000007C
:10FF2000B8F703080D1402050F000000088004084C
:10FF30000C1401050E000000DCA004080C140005E0
:10FF40000C00000054A104080C140205110000006C
:10FF5000CCA104081214000512000000A43004080B
:10FF600017140005180000006CE2030810140005C7
:10FF70001000000040540408101400050F00000099
:10FF8000E05404080D1400050D00000094800408DE
:10FF9000071903050B000000C0C404080B16020576
:10FFA0000E00000074940408071901050B000000FE
:10FFB00024C504080B0A020510000000B42205083D
:10FFC0000D02001A0D000000C0D405080705030546
:10FFD0000E00000088CC05080F0E010B1200000077
:10FFE00010B004080F140205120000008055040828
:10FFF0000F0E010B1000000080B004080F14010563
:020000040801F1
:1000000012000000205604080E0E010B1000000024
:1000100000CB04080714000507000000FCE80408F2
:100020000F14010B12000000C05604080D14020545
:1000300011000000208104080214020506000000DF
:100040009CCC05080519FF0507000000F8F304081B
:100050000B1402050D00000044A20408021402055E
:1000600006000000B0CC0508150E020B19000000B8
:10007000606104080D0E020B1100000064CB04083F
:100080000F0E010B11000000F0B004080F13020B5B
:1000900012000000346304080F13010B120000006B
:1000A000CC630408070E020B0800000000340508AA
:1000B0000A0E000B0C000000680405080814000577
:1000C000080000004CE904080D0E020B11000000AE
:1000D000C8CB04080D0E000B0D0000002CCC04084A
:1000E000140E000B14000000AC8104080C0E000B71
:1000F0000D000000D8DF04080D13000B0D000000F8
:10010000608A04080B0E000B0B0000002CE00408B2
:10011000081B02050C0000008CBA0408021A060530
:100120000E00000040C30508081B02050C0000007B
:10013000F8BA04080C05021010000000F8B3050816
:1001400001010019070000005CF305080214030B0D
:1001500007000000C4CC05080C1102070F000000C6
:1001600028C304080F1400050F000000605704089E
:100170000E0E00090F00000090CC04080E140005BC
:100180000F00000038820408021606080E00000066
:10019000E4C705080D1A010510000000AC2B040887
:1001A000070404050E00000000D205081414000521
:1001B00015000000C80E0408080A01050B00000025
:1001C000B0850508080A010D0A000000D885050859
:1001D0000D07010F100000008C55050807020011E3
:1001E0000700000040EC050814140005150000008D
:1001F000900F04080A0203060E00000064E90508D7
:10020000080801070A00000078AA05080E0F010B74
:100210001000000050BD0408080D01050A00000090
:10022000B0440508080D01050A000000E444050873
:10023000070504050E000000D8CC05080B13020BBF
:100240000F00000088AB04080E1700051000000026
:1002500014510408020303110800000080F205088D
:10026000050604180E000000A8CF0508050C0105BE
:100270000A000000C09A0508090A01050B000000E9
:10028000E0500508080A010D0A0000000086050874
:10029000141400051400000058100408141400057C
:1002A00015000000201104081514010517000000B6
:1002B00094F803080B13020B0E000000FCAB0408BB
:1002C000121900001200000084F103081219000046
:1002D0001200000068F2030812180001120000006A
:1002E00004FC03081218000112000000DCFC0308E3
:1002F00013180001120000005CE30308131900004A
:100300001200000098D603081814FF051900000019
:100310004CE40308131901051500000094D70308E5
:100320000B1902000E0000007C6E04080B1902007D
:100330000E000000146F04080B1802010E000000EC
:10034000F07404080B1802010E0000008075040808
:100350000819FE000600000088C5040808190000FE
:1003600006000000ECC504080B18FE0106000000A2
:10037000107604080618000106000000A0F6040824
:100380001114000513000000583104080F18020171
:1003900013000000DC180408141901001600000006
:1003A00090D8030814190100160000008CD9030826
:1003B00014180101160000003CE50308141801019F
:1003C000160000002CE603081418010116000000B6
:1003D0001CE703080D0D010C1000000094D5040863
:1003E000141601041600000070F903080C1902002D
:1003F00011000000AC6F04080C190200110000008D
:10040000447004080C18020111000000A0760408D2
:100410000C180201110000003077040810190000C8
:100420000F000000E81104080C1402050E00000083
:10043000BCA204080D14020510000000C4820408C8
:100440000F14010512000000005804080F140105E4
:1004500012000000A05804080F140105120000004B
:10046000405904080F1301061200000064640408D8
:100470000F14010512000000E05904080F140105D3
:1004800012000000805A04081C0E010B1D00000021
:10049000081504080E13010B10000000E88A040878
:1004A0000E14010510000000508304080E1401050D
:1004B00010000000DC8304080E1401051000000089
:1004C000688404080E14010510000000F484040878
:1004D0000815FE040600000080E00408081500046A
:1004E00006000000D4E004080C14FD05060000001E
:1004F00034A304080714FF05060000009CE9040863
:100500000F14010511000000205B04080D13020602
:1005100011000000708B04080F1401051100000089
:10052000C05B04080F14010511000000605C0408A2
:100530000F14010511000000005D04080F130106EF
:1005400011000000FC6404080F14010511000000F4
:10055000A05D04080E0F010B10000000BCBD0408D4
:100560000F10010A11000000109804080D15020474
:1005700011000000A07204080D1502041100000013
:10058000347304080D14020511000000808504086E
:100590000D140205110000000C8604080D1A000459
:1005A0000D000000642C04080F1902051200000061
:1005B000B01204080E1900050D000000F4360408FE
:1005C000020E020B06000000D0D405080C14000532
:1005D0000C000000ACA3040807140005070000008D
:1005E000ECE904081C1401051E00000098C403086F
:1005F0001B0E010B1D000000CC1504080C18010196
:100600000E000000C07704080B1400050C00000069
:1006100024A40408101800010F0000009C1904080D
:100620000D1800010D000000DC4904080B14000542
:100630000B0000009CA404080E1900050F00000028
:10064000A43704080B0402050E00000074C5050859
:100650000B0402050E0000008CC505080A02030603
:100660000E00000070E905080B0402050E000000F2
:10067000A4C50508020406050E00000068F0050880
:10068000060604050E000000BCCF05080506051887
:100690000E000000D0CF05080A0302060E0000007D
:1006A000D0D305080B0603030E000000E49A0508EA
:1006B00012140105130000000C3204080B13020B86
:1006C0000F00000070AC04080F0E000B0F000000BC
:1006D00060B10408070200110700000048EC05089B
:1006E0000B0201110D000000DCE6050818020111E3
:1006F0001A000000BCC5050804050205080000003A
:100700007CE90508040501050800000088E90508E2
:10071000040501160800000094E905080705030513
:100720000B000000ECCC0508070502050B000000DB
:1007300000CD0508070502160B00000014CD0508C2
:100740000C18020510000000507804080C1902056E
:1007500010000000DC7004080606030C0D00000009
:10076000E4CF0508140303161A00000018B40508A6
:100770001C1401051E000000B0C50308050A010D88
:100780000600000038B40508050A010D0600000047
:1007900058B405080A14FD050300000050C60408FB
:1007A0000F14FF050E000000405E04080B15010445
:1007B0000D00000090990408160D00051A000000B5
:1007C000007A04081214010513000000C032040866
:1007D00016140105180000004CFA03080C1601035A
:1007E0000F000000F8940408101301061100000027
:1007F000946504081116010613000000781304081C
:100800000D1601060F000000FC6104080D02011224
:1008100010000000E0D405080A14FD0503000000E4
:10082000B4C60408020303110800000084F205089E
:100830000F1B01020F000000B4FD03081208010D98
:1008400015000000E8F60408091C00020A00000078
:10085000988604080D08010D0F00000038340508C3
:100860000D0E020B0F000000F4CC04080E1001095D
:100870000F000000D0B104080D1000090F000000A7
:1008800040B204080D1502050F000000C8730408EB
:100890000A1400050C00000018C704080A1400051B
:1008A0000C0000007CC704080D1200070D000000BA
:1008B000109A04080101000D0400000060F305080F
:1008C000020900040200000020EB050804040004F3
:1008D0000500000050EC05080709010407000000AE
:1008E000089B0508070C000307000000005A0508D4
:1008F0000A0900040A000000406205080909000412
:1009000009000000706205080204000402000000F3
:100910006CF00508040B000404000000FCC7050887
:10092000040B00040400000014C8050804030004BC
:1009300004000000E8EE05080707010508000000B4
:1009400024BC05080204010B0400000070F0050837
:10095000040200090400000074F005080202010B03
:1009600004000000FCF20508070B0004070000006B
:10097000306C050807090004070000002C9B0508DF
:100980000409020407000000F8CF05080709000465
:1009900007000000509B050807090004070000003D
:1009A000749B05080809000407000000989B0508CF
:1009B0000709000407000000BC9B050807090004A4
:1009C00007000000E09B050806090004070000007E
:1009D000BCC005080709000407000000049C0508C6
:1009E0000709000407000000289C0508020601070B
:1009F00004000000F0EE05080208010704000000F2
:100A000058EC0508070801040800000098AA05082A
:100A1000070401070800000010D2050807080104B8
:100A200008000000B8AA0508060900040600000036
:100A3000D8C00508090901040B000000A0620508E0
:100A40000A09000409000000D06205080709000433
:100A5000070000004C9C05080A090004090000007A
:100A60000063050809090004090000003063050857
:100A70000709000407000000709C0508070900042E
:100A800007000000949C0508090900040900000003
:100A90006063050809090004090000009063050867
:100AA00004090004040000000CD005080709000434
:100AB00006000000B89C05080909000409000000B0
:100AC000C06305080709000407000000DC9C050856
:100AD0000C0900040C000000E84005080A090004A5
:100AE0000A000000F06305080A090004090000007C
:100AF000206405080709000407000000009D0508A0
:100B00000B0900040A00000020410508090900043F
:100B100008000000506405080609000406000000F3
:100B2000F4C00508060900040700000010C105080C
:100B30000909000408000000806405080909000490
:100B400009000000B06405080D0900040C00000055
:100B50001C1C05080909000409000000E0640508E0
:100B60000809000408000000249D05080809FF0486
:100B700007000000489D0508040B00040500000064
:100B80002CC8050805090104070000002CC1050850
:100B9000040B00040500000044C805080807010410
:100BA0000800000040BC05080701000E0600000018
:100BB00078F00508040401020600000060EC050856
:100BC00008070006080000005CBC050808090004CE
:100BD000080000006C9D05080707000607000000DC
:100BE00078BC05080809000408000000909D05086D
:100BF000070700060700000094BC0508040900046C
:100C00000400000020D005080809000608000000C4
:100C1000B49D05080809000408000000D89D0508D7
:100C2000040900040400000034D00508030B00048C
:100C3000030000005CC80508070900040700000065
:100C4000FC9D0508040900040400000048D00508C4
:100C50000C0700060C000000AC760508080700062B
:100C600008000000B0BC05080707000607000000E8
:100C7000CCBC05080809000608000000209E0508F5
:100C80000809000608000000449E05080507000644
:100C9000050000003CCA0508060700060600000023
:100CA00054CA050804090004040000005CD00508CB
:100CB0000807000608000000E8BC05080707000652
:100CC0000700000004BD05080B0700060B0000002C
:100CD000D8760508070700060700000020BD0508B4
:100CE0000709000607000000689E050805070006C2
:100CF000060000006CCA0508040B00040400000094
:100D000074C80508020D030308000000F0D50508AB
:100D1000040B0004040000008CC805080703010749
:100D200008000000E8E605080101000D04000000CD
:100D300064F3050802090006020000002CEB050818
:100D4000060901040700000048C105080809FF045E
:100D5000070000008C9E050805080105070000003B
:100D6000D4C505080809000407000000B09E050866
:100D7000020B03040800000068E80508050B0004E6
:100D80000600000044A70508040201040600000054
:100D90007CF005080A0900040A0000001065050837
:100DA0000504000405000000F4E60508040500073A
:100DB00004000000A0E9050808040007080000007E
:100DC00020D20508040200090400000080F0050894
:100DD0000A0900040A000000406505080502010434
:100DE00006000000F8EE05080304010405000000F9
:100DF00068EC050807070105080000003CBD050870
:100E00000405000404000000ACE905080406000421
:100E10000400000000E705080403010306000000C9
:100E200000EF05080809000608000000D49E050828
:100E3000070B0004060000005C6C050802020108B4
:100E40000400000000F305080303010D0400000086
:100E500008EF050803060104040000000CE705087C
:100E6000040400040400000070EC050804050007F9
:100E700004000000B8E90508090901040A0000009F
:100E800070650508090901040A000000A06505084D
:100E90000B0900040A000000584105080609000675
:100EA0000600000064C105080A0D000009000000EA
:100EB000181105080A0D0000090000005C11050862
:100EC0000A0C000109000000F02205080A0C0001CC
:100ED000090000002C2305080A0B0002090000008D
:100EE000983805080A0D000009000000A011050847
:100EF0000C0900040C000000904105080A0C0004D5
:100F00000900000068230508070D00000700000025
:100F100018450508070D0000070000004C450508AE
:100F2000070C000107000000305A0508080CFF02FA
:100F300007000000605A0508040D000004000000CE
:100F40005CC30508040D00000400000078C3050818
:100F5000060CFF0104000000F89E0508040B0002C7
:100F600004000000A4C805080909000409000000E5
:100F7000D06505080A0C00010A000000A42305083A
:100F80000A0D000009000000E41105080A0D000028
:100F900009000000281205080A0C000109000000E1
:100FA000E02305080A0C0001090000001C240508C4
:100FB0000A0B000209000000D038050806060106E9
:100FC0000800000070D005080A0B000309000000AB
:100FD00008390508090D0000080000006C1205081A
:100FE000090D000008000000B0120508090C0001FE
:100FF0000800000058240508090B00020800000042
:1010000040390508080D000008000000804505086B
:1010100007090004070000001C9F050807090004D9
:1010200007000000409F0508080B000208000000B0
:10103000886C0508080B000208000000B46C050865
:10104000080A00030800000028860508080A0003B3
:101050000800000050860508080900040800000088
:10106000649F0508080A0003080000007886050848
:101070000D0700060C000000C0550508070A000611
:1010800007000000A0860508070B0002070000000B
:10109000E06C0508070B0002070000000C6D050856
:1010A000070A000307000000C88605080909FF04B5
:1010B0000700000000660508050BFF0204000000A1
:1010C00068A70508050BFF02040000008CA70508AF
:1010D000060AFF030400000078B4050804090004B0
:1010E0000400000084D00508070900040700000080
:1010F000889F0508080A000308000000F08605081C
:10110000070B000207000000386D0508070B0002FE
:1011100007000000646D0508070A000307000000CF
:1011200018870508070A0003070000004087050824
:101130000709000407000000AC9F05080706010529
:1011400008000000ECC505080709000507000000BD
:10115000D09F0508080B000208000000906D0508EC
:10116000080B000208000000BC6D0508080A000317
:10117000080000006887050808090004080000004E
:10118000F49F0508070D000207000000B44505089C
:10119000080B000408000000E86D0508080B0004B7
:1011A00007000000146E0508040700060400000094
:1011B000F0D40508070900040700000018A005087E
:1011C0000509FF040400000080C105080D090004A2
:1011D0000D0000005C1C05080D0700060C00000057
:1011E000F4550508060C0001060000003CA00508A7
:1011F000070AFF030600000090870508090B00029C
:101200000800000078390508080CFF0107000000FD
:10121000905A0508050A00030600000098B4050866
:10122000060B010407000000B0A705080602010331
:101230000700000010EF0508060301030700000087
:1012400038EB0508050201040600000018EF050848
:10125000050301030600000044EB05080202010437
:101260000300000004F30508030301030500000068
:1012700020EF05080203010C0400000088F20508B5
:10128000050301030600000050EB050805030103F8
:10129000060000005CEB05080A09FF0409000000D5
:1012A00030660508080900060800000060A005086F
:1012B0000907FF060700000028A505080402000929
:1012C0000400000084F00508070200090600000081
:1012D00078EC05080D0200090C00000000D5050897
:1012E000020400040200000088F005080204000463
:1012F000020000008CF005080204000B0200000050
:1013000090F00508040400040500000080EC0508C6
:10131000040400040500000088EC05080404000B28
:101320000500000090EC0508070B01040700000011
:10133000406E0508070B0104070000006C6E0508ED
:101340000405020507000000C4E905080A02010BB4
:101350000C000000D0E905080F0900040F00000090
:1013600030F704080205000702000000F0EF05084E
:101370000205000702000000F8EF05080609FE0458
:10138000010000009CC105080809000407000000D6
:1013900084A00508060A000306000000B8B405088A
:1013A0000B0500040C000000D8B405080A09FF046E
:1013B00009000000606605080B0900040B0000002E
:1013C000C8410508070A000307000000B8870508A0
:1013D0000809000408000000A8A005080B0BFF0482
:1013E00009000000DC080508070A000407000000E7
:1013F000E0870508070201080800000098EC0508CE
:101400000609FE0401000000B8C105080202010837
:101410000400000008F30508080D010207000000A1
:10142000E8450508080501070A00000028CD050861
:10143000050D00020500000060940508060501077F
:1014400007000000E0D305080607010607000000BA
:1014500084CA0508060801050700000004C605083F
:1014600006080005070000001CC60508070A01045D
:1014700007000000088805080709000406000000AE
:10148000CCA005080709000406000000F0A005082C
:101490000609000406000000D4C105080101000D82
:1014A0000400000068F30508010A000302000000C0
:1014B000DCE9050802030103040000008CF20508C2
:1014C000070A00030800000030880508060D010225
:1014D00008000000889405080A0A00030A000000BA
:1014E00014510508090A00030900000048510508C5
:1014F000010301030200000090F20508040B010340
:1015000004000000BCC80508040B00030400000030
:10151000D4C805080404000304000000A0EC05087A
:10152000070701050900000058BD05080203010B6B
:101530000400000094F20508040100090400000002
:101540000CF305080102020B0400000010F305086B
:10155000070D0103080000001C460508060A0103E8
:1015600008000000F8B40508050A0203080000009E
:1015700018B50508060A01030800000038B505087B
:10158000060A01030800000058B50508080A000310
:101590000800000058880508070A0003080000003A
:1015A00080880508070A000308000000A8880508CD
:1015B000060A01030800000078B50508060A0103C1
:1015C0000800000098B50508070A0003080000009D
:1015D000D0880508010602070400000028EF05086E
:1015E0000207010704000000F8ED050807080104E0
:1015F00009000000D8AA0508070301070900000038
:1016000018E705080708010409000000F8AA050802
:10161000060A000307000000B8B505080A0A01031E
:101620000C0000007C5105080A0A00030B000000B2
:10163000B0510508060A010308000000D8B50508E6
:101640000A0A00030A000000E4510508080A010321
:1016500009000000F8880508060A010307000000D9
:10166000F8B50508060A01030700000018B60508CA
:101670000A0A00030A00000018520508080A0103BC
:101680000900000020890508030A01030400000086
:101690003CCD0508060A00030700000038B605081F
:1016A000080A01030900000048890508050A01032A
:1016B0000700000058B605080C0A00030D000000E2
:1016C00094240508090A01030A0000004C52050889
:1016D0000A0A00030A00000080520508060A0103F6
:1016E0000800000078B605080B0A00030B00000094
:1016F000D0240508080A01030800000070890508C5
:10170000060A00030700000098B60508070A000350
:101710000700000098890508080A01030900000075
:10172000C08905080A0A00030A000000B45205082F
:101730000D0A00030E000000B0040508090A0003AA
:101740000A000000E8520508090A00030900000029
:101750001C530508070A000307000000E889050874
:10176000030C01030400000034C60508050A010348
:1017700008000000B8B60508030C000304000000D0
:101780004CC60508080701030900000074BD0508E0
:101790000701000E0700000094F005080403010291
:1017A0000500000030EF05080807000609000000EA
:1017B00090BD0508090A0003090000005053050800
:1017C0000807000607000000ACBD0508080A000372
:1017D00009000000108A050807070006080000003D
:1017E000C8BD0508040A00030400000050CD050828
:1017F000080A000609000000388A0508080A0003E4
:1018000008000000608A0508030A000303000000C6
:1018100064CD0508030DFF030300000094C3050811
:10182000070A000308000000888A0508040AFF036D
:101830000400000078CD05080D0700060D0000002B
:10184000285605080807000609000000E4BD050841
:10185000070700060800000000BE0508090A000688
:101860000900000084530508080A0006090000006A
:10187000B08A0508040700060500000010D5050819
:1018800005070006050000009CCA0508050AFF03BD
:1018900004000000D8B6050808070006080000008C
:1018A0001CBE0508080700060800000038BE050831
:1018B0000C0700060C000000047705080707000667
:1018C0000800000054BE0508080A000608000000D1
:1018D000D88A05080607FF0605000000B4CA0508F7
:1018E000030B000304000000ECC80508010D04030D
:1018F0000900000000D60508030B000304000000E7
:1019000004C905080702010709000000A8EC050842
:101910000101000D040000006CF30508010A000637
:1019200002000000E8E905080609010308000000BC
:10193000F0C10508080A000308000000008B050834
:101940000607010508000000CCCA0508080A0003C4
:1019500008000000288B0508010B040409000000A2
:1019600074E80508050C00030600000014A1050832
:10197000030201030400000098F00508090A0103AE
:101980000B000000B8530508060500030500000021
:10199000F0D305080405000704000000F4E9050879
:1019A0000904FF07090000008CCD050804010009A7
:1019B0000400000014F30508090A01030B000000ED
:1019C000EC530508050101030600000098F2050824
:1019D000040501030500000000EA050807070105EA
:1019E0000900000070BE05080407000305000000A0
:1019F00020D50508040700030500000030D50508C0
:101A0000040301030500000038EF0508080A00067A
:101A100008000000508B0508060B010307000000BA
:101A2000D4A70508010202080400000018F3050805
:101A30000303010D0400000040EF05080407000344
:101A40000500000040D5050805050003040000005E
:101A500000D4050804050007040000000CEA05088E
:101A60000B0A00030B0000000C2505080B0A0003FD
:101A70000B000000482505080B0A00030B000000BE
:101A800084250508050A010607000000F8B60508C8
:101A90000A0D00000B000000F41205080A0D0000FA
:101AA0000B000000381305080A0C00010B000000B1
:101AB000C02505080A0D00000B0000007C13050876
:101AC0000A0C00010B000000FC2505080A0D0000AF
:101AD0000B000000C01305080D0A00030D000000F4
:101AE000F80405080A0D00030A00000004140508A4
:101AF000060D010007000000B0940508060D010066
:101B000007000000D8940508060C0101070000003A
:101B100038A10508060C0101070000005CA10508BA
:101B2000040D000004000000B0C30508040D00000F
:101B300004000000CCC30508050C000104000000EF
:101B400080A10508030C01010400000064C605081B
:101B5000080A010309000000788B0508090D01003F
:101B60000A000000481405080A0D00000A000000E1
:101B70008C1405080A0D00000A000000D0140508A6
:101B80000A0C00010A000000382605080A0D0000B2
:101B90000A000000141505080A0C00010A000000E4
:101BA00074260508060601050900000098D00508FE
:101BB0000A0C00020A000000B0260508080D01000A
:101BC0000900000050460508080D0100090000004A
:101BD00084460508080C010109000000C05A0508E8
:101BE000080C010109000000F05A0508090D000069
:101BF0000900000058150508060A01030800000046
